:100000000C94F4500C9425510C9425510C942551CA
:100010000C9425510C9425510C9425510C94255188
:100020000C9425510C9425510C9425510C94255178
:100030000C94E6860C9425510D9477130D94BB1007
:100040000C9425510D94681B0C9425510C9425514A
:100050000C9425510C9425510C9425510C94E37665
:100060000C9425510C9462630C9425510C942551E9
:100070000C9425510C9451BC0C9425510C94255191
:100080000D94C5150C9425510C9425510C942551B3
:100090000C941E630C9425510C9425510C942551FD
:1000A0000C9425510C9425510D949F0D0C942551C1
:1000B0000C9425510D94810D0C9425510C942551CF
:1000C0000C9425510C9425510C9425510D94410DFF
:1000D0000C9425510C9425510C9425510C942551C8
:1000E0000C942551000000000000000000000000FA
:1000F0000000000000000000000000000000000000
:10010000A55AB44B3B3082018CAD7365D5E91568B7
:10011000150343036C03A803CD031D0444048204A8
:10012000B9040E0545056F0582059705AA05BE05AC
:10013000CE05DE05EF05210645065A0675069E0624
:10014000AF06BE06D3061B073F078D071403A207A1
:10015000B707C107C907D607E307F00703080D086B
:100160001A0827083408430855087D08E5084B0994
:100170006C09D609DF09E709EF09F7092A0A460AD7
:10018000590A620ABA0AE10A2B0B820B290C5B0C92
:10019000BD0C130D3F0D630D810DE30D030E460ED7
:1001A000AD0EE80E340F880FA30FCC0FED0F1B1010
:1001B00041107510C4102011CA11D0111403DA11A6
:1001C000E811F611FF11081217121C122912301231
:1001D0003912721281128C1295129D121403A412FC
:1001E000AD12BF12D212E312F31202130D13191340
:1001F000241336134713571368137B138613140302
:1002000093139D13B013C1131403E213EC13FE13E5
:100210000A141A1422143514481455146114741451
:1002200084149214A414B314C514D514E614F7144A
:10023000FD140F151B1523153415461552155915A8
:10024000611568156D1579158B1591159B15A815F8
:10025000AC15B915BF15CD151403D015E215F11560
:100260001F162B163A1614036816791687169B1656
:100270009F16B016BD16CE161403DD16F016021723
:100280001217221737174117511760176C177C1771
:100290009117A017AA17BF17CD17DF17F01701186E
:1002A0001218231834183A1844184C1851185C18AE
:1002B00065186B187318A918DE18F118FA180D19BB
:1002C00021193D196B19BB19DC19331A911AF41A4B
:1002D0004B1B941BBD1BE21BE91B061C511C8E1CF7
:1002E0000C1D511DBC1DED1D761EBE1EFD1E311FB9
:1002F000461F9E1FC31F1D20A0203821D221362259
:10030000C0223F23D1233A24422448244F241403FB
:1003100055245C24F71469247E248F249E24AB2466
:10032000BA24CA24DE241403EC24FD24082518254D
:10033000262539254D255C25692576258225952597
:10034000A725BA25C625D425DB25EF2503261126AA
:10035000232637264C265E26662694269D26E826EA
:10036000F8260A271A2729273E2714035027622731
:1003700077278A279D27AE27C227D627EB27FC277A
:100380000A281E282A283D284F285C286F28842800
:100390009928AE28C328D3281403E628F8280C2966
:1003A0002029302943295729622971298129942933
:1003B0001403A429B729C829DD29EE29FF29122A07
:1003C000272A3A2A4D2A612A722A872A9A2AAD2A8E
:1003D000BF2AD32AE82AFA2A0D2B202B332B442BB1
:1003E000532B652BAB2BFD2B382C7B2CBA2CF72CED
:1003F000312D5E2DA82DCC2D452EDB2EFE2E272F48
:100400005D2F6A2F7A2F8A2F9F2FC92FDC2F2C3038
:10041000333037300050726F626C656D6120656EED
:10042000636F6E747261646F2C206E6976656C61A7
:100430006369AD6E205A20666F727A6F7361202EE9
:100440002E2E004E6976656C616369AD6E20666123
:100450006C6C6964612E20496D7072657369AD6E54
:100460002063616E63656C6164612E0043616C653D
:100470006E7461646F72657320646573616374691F
:100480007661646F7320706F7220656C2074656D87
:10049000706F72697A61646F72206465207365673A
:1004A0007572696461642E0043AD6469676F2047AB
:1004B000206C616D696E61646F207061726120757E
:1004C0006E206E6976656C206469662E0043AD64AB
:1004D00069676F2047206C616D696E61646F207081
:1004E00061726120756E206E6976656C2064696644
:1004F0006572656E74652E205675656C7665206133
:10050000206C616D696E617220656C206D6F646531
:100510006C6F206465206E7565766F2E0043AD6448
:1005200069676F2047206C616D696E61646F207030
:10053000617261206E7565766F206669726D776194
:1005400072652E0043AD6469676F2047206C616D52
:10055000696E61646F2070617261206E7565766F7F
:10056000206669726D776172652E204163747561D2
:100570006C697A6120656C206669726D776172655D
:100580002E0043AD6469676F2047206C616D696E12
:1005900061646F207061726120756E207469706F84
:1005A00020646520696D707265736F726120646983
:1005B000662E436F6E742E3F0043AD6469676F20F3
:1005C00047206C616D696E61646F2070617261209B
:1005D000756E6120696D707265736F7261206469F8
:1005E000666572656E74652E205675656C7665203D
:1005F00061206C616D696E617220656C206D6F6445
:10060000656C6F206465206E7565766F2E00507581
:100610006C736120656C206469616C20706172612B
:100620002070726563616C656E746172206C61200C
:10063000626F7175696C6C61207920636F6E74698B
:100640006E75652E0050756C736120656C20646951
:10065000616C2070617261206465736361726761AF
:100660007220656C2066696C616D656E746F0079CF
:100670002070726573696F6E6120656C20646961BA
:100680006C00496E74726F64756369722066696C80
:10069000616D656E746F00436F6C6F72206E6F20BA
:1006A000686F6D6F679A6E656F0046696C2E206E7D
:1006B0006F20696E74726F64756369646F00436163
:1006C0006D62696F20636F72726563746F0043615E
:1006D0006D6269616E646F20636F6C6F720043615D
:1006E0006D62696F20636F72726563746F21004180
:1006F00062726520656C2074656E736F722079205C
:1007000072657469726120656C2066696C616D65E3
:100710006E746F206D616E75616C6D656E74652EA3
:100720000053652064657363617267AD20636F6E0B
:10073000209A7869746F20656C2066696C616D65BC
:100740006E746F3F0041637475616C697A612070EB
:100750006F72206661766F722E004E7565766F201F
:100760006669726D7761726520646973706F6E6916
:10077000626C653A004573706572616E646F2061EA
:100780002071756520736520656E6672A265206CA8
:100790006120736F6E64612050494E444100506F78
:1007A00072206661766F72206573706572610053A6
:1007B000696E206D6F76696D69656E746F00457343
:1007C000706572616E646F206F7264656E65732E02
:1007D0002E2E005365206E65636573697461207504
:1007E0006E612074656D70657261747572612061EF
:1007F0006D6269656E746520656E746520323120A6
:100800007920323643207920756E20736F706F72B5
:1008100074652072A26769646F2E005265616C690D
:100820007A61206C612063616C696272616369AD99
:100830006E2058595A207072696D65726F2E00468D
:10084000616C6CAD206C61206E6976656C6163696A
:10085000AD6E2E2053656E736F72206E6F206675BD
:100860006E63696F6E612E20526573746F732065BD
:100870006E20626F7175696C6C613F2045737065A5
:1008800072616E646F2072657365742E00507265BC
:1008900063616C656E74617220626F7175696C6CF6
:1008A0006100446973742E20656E2059206465735D
:1008B0006465206D696E00497A717569657264615D
:1008C000004465726563686100446573762E206D2F
:1008D000656469646100446573762E206C696765A0
:1008E000726100446573762E2073657665726100CF
:1008F0005B303B305D2070756E746F206F66667381
:10090000657400416A75737461722D5A0054726186
:1009100073657261205BE46D5D0046726F6E746199
:100920006C205BE46D5D0044657265636861205B0B
:10093000E46D5D00497A71756965726461205BE4FC
:100940006D5D0045737461626C65636572207465EA
:100950006D702E3A00436172726F73205A20697A6B
:10096000712E2F6465722E206573748A6E206172F9
:1009700072696261206D8A78696D6F3F0043616CB6
:10098000696272616E646F2058595A2E20476972ED
:100990006120656C206469616C20706172612073F4
:1009A0007562697220656C206578747275736F72F8
:1009B00020686173746120746F636172206C6F735F
:1009C00020746F706573207375706572696F7265DE
:1009D000732E2044657370759A732068617A206362
:1009E0006C69632E0043616C696272616E646F2092
:1009F0005A2E204769726120656C206469616C2001
:100A00007061726120737562697220656C2065780F
:100A1000747275736F7220686173746120746F6390
:100A20006172206C6F7320746F70657320737570C2
:100A30006572696F7265732E2044657370759A7361
:100A40002068617A20636C69632E0046616C6C6F6C
:100A5000206465206C612063616C69627261636906
:100A6000AD6E2064652050494E4441004C612063C6
:100A7000616C696272616369AD6E2050494E444198
:100A8000206573748A2066696E616C697A6164613D
:100A90002079206163746976612E2053652070751A
:100AA000656465206465736163746976617220654D
:100AB0006E20656C206D656E7520436F6E6669678C
:100AC0007572616369AD6E202D3E2043616C2E20EE
:100AD00050494E4441004578747275736F72004DF1
:100AE0006F766572205A004D6F7665722059004D01
:100AF0006F7665722058004C8A6D696E6120252ED4
:100B000037730A5A206F66667365743A20252B3155
:100B10002E33666D6D0A2563436F6E74696E756161
:100B2000720A2563526573657400436172676120C0
:100B30007072696D65726F20656C2066696C616D9D
:100B4000656E746F2E0053656C656363696F6E61CB
:100B50002066696C616D2E3A0043616E63656C615D
:100B60007200456A65637574617220656C2041731B
:100B7000697374656E746520626F72726172612050
:100B80006C6F732076616C6F72657320646520638F
:100B9000616C696272616369AD6E206163747561D5
:100BA0006C6573207920636F6D656E7A61728A203F
:100BB0006465206E7565766F2E0050726563616C9A
:100BC000656E742E20626F7175696C6C612E2045A4
:100BD000737065726120706F72206661766F722E1D
:100BE00000436F6C6F636120656C2066696C616D9A
:100BF000656E746F20656E20656C20657874727503
:100C0000736F722C206C7565676F207072657369E5
:100C10006F6E6120656C206469616C207061726127
:100C2000206361726761726C6F2E00436F6C6F633B
:100C30006120656C2066696C616D656E746F2065FE
:100C40006E20656C207072696D6572207475626FBC
:100C5000206465206C61204D4D552C206C756567B6
:100C60006F2070726573696F6E6120656C206469B6
:100C7000616C2070617261206361726761726C6F78
:100C80002E004C6120696D707265736F7261206314
:100C90006F6D656E7A61728A206120696D7072690C
:100CA0006D697220756E61206C696E656120656E7C
:100CB000207A69672D7A61672E2047697261206505
:100CC0006C206469616C2068617374612071756562
:100CD000206C61206C696E656120616C63616E637C
:100CE00065206C6120616C74757261206F7074692D
:100CF0006D612E204D697261206C617320666F7486
:100D00006F732064656C206D616E75616C20284383
:100D100061706974756C6F2064652063616C6962D1
:100D200072616369AD6E292E0053656C65636369FA
:100D30006F6E61206C612074656D70657261747591
:100D400072612061646563756164612061207475FE
:100D5000206D6174657269616C2E004573636F6705
:100D60006520756E2066696C616D656E746F2070AC
:100D7000617261206C612043616C696272616369B8
:100D8000AD6E206465206C61205072696D65726182
:100D9000204361706120792073656C65636369AD80
:100DA0006E616C6F20656E20656C206D656E7520C0
:100DB000656E2070616E74616C6C612E00566F7987
:100DC00020612063616C6962726172206C612064D1
:100DD000697374616E63696120656E747265206CFD
:100DE000612070756E7461206465206C6120626F93
:100DF0007175696C6C612079206C61207375706508
:100E0000726669636965206465206C612062617344
:100E1000652E005365207265636F6D69656E646150
:100E20002063616C6962726172205A2E20456A6586
:100E300063757461726C6F2061686F72613F0052FC
:100E40006574697261206C61206C616D2E2064652F
:100E500020616365726F206465206C61206261733C
:100E6000652E004573748A206C61206C8A6D696EF2
:100E70006120736F627265206C6120626173653FEF
:100E8000004C656520656C206D616E75616C207924
:100E90002072657375656C766520656C2070726F65
:100EA000626C656D612E2044657370759A732C2099
:100EB0007265696E69636961206C6120696D707229
:100EC00065736F7261207920636F6E74696E7561EE
:100ED00020636F6E20656C204173697374656E7456
:100EE000652E005465726D696E61646F2E204665D3
:100EF0006C6963657320696D70726573696F6E6587
:100F00007321005369656D70726520707565646545
:100F100073206163636564657220616C206173692D
:100F20007374656E74652064657364652043616CD9
:100F3000696272616369AD6E202D3E2041736973F1
:100F400074656E7465005369207469656E657320FD
:100F5000706C616E636861732064652061636572A3
:100F60006F2061646963696F6E616C65732C2063C7
:100F7000616C696272612073757320616A75737444
:100F8000657320656E20416A7573746573202D202A
:100F9000416A7573746573204857202D20506C6129
:100FA0006E6368617320616365726F2E004C696DBA
:100FB000706961206C612073757065726669636920
:100FC00065206465206C6120626173652C20792046
:100FD0006C7565676F2070726573696F6E612065EF
:100FE0006C206469616C2E005175696572657320AF
:100FF0007265706574697220656C20C06C74696D6F
:101000006F207061736F20706172612072652D2096
:10101000616A7573746172206C61206469737461B4
:101020006E63696120626F7175696C6C612D6261BC
:1010300073653F0053656C656363696F6E61206C17
:10104000612074656D706572617475726120706184
:1010500072612070726563616C656E746172206C80
:101060006120626F7175696C6C61207175652073A8
:101070006520616A757374652061207475206D61E7
:1010800074657269616C2E004573746120656C2013
:1010900066696C616D656E746F206361726761640F
:1010A0006F3F0041686F72612070726563616C65AB
:1010B0006E7461729A206C6120626F7175696C6CDC
:1010C00061207061726120504C412E00566F792072
:1010D000612068616365722043616C69627261635B
:1010E00069AD6E205A2061686F72612E0041686F91
:1010F000726120726574697261206C612070727512
:10110000656261206465206C61206C8A6D696E6126
:1011100020646520616365726F2E00526574697288
:1011200061206C6F7320736F706F727465732064CD
:101130006520656E76A26F207072696D65726F2E84
:10114000004861729A206C612063616C696272610F
:101150006369AD6E2058595A2E205075656465201C
:10116000746172646172206861737461203234202A
:101170006D696E2E005072696D65726F2C2068610A
:10118000726520656C2053656C667465737420709D
:1011900061726120636F6D70726F626172206C6F3B
:1011A000732070726F626C656D6173206465206D71
:1011B0006F6E74616A65206D8A7320636F6D756EE2
:1011C00065732E00486F6C612C20736F79207475E5
:1011D00020696D707265736F7261204F7269676903
:1011E0006E616C2050727573612069332E205175C9
:1011F000696572657320717565207465206775A2D5
:1012000065206120747261766573206465206C616D
:1012100020636F6E6669677572616369AD6E3F00CA
:10122000486F6C612C20736F7920747520696D7024
:101230007265736F7261204F726967696E616C20AD
:1012400050727573612069332E205465206775696B
:1012500061729A20612074726176657320646520E2
:10126000756E2062726576652070726F6365736F4C
:1012700020646520636F6E6669677572616369AD2E
:101280006E2C20656E20656C20717565207365205D
:1012900063616C69627261728A20656C20656A653F
:1012A000205A2E2044657370759A732C20657374D0
:1012B00061728A73206C6973746F2070617261202F
:1012C000696D7072696D69722E005061757361008D
:1012D00046532061636369AD6E004465742E2061DE
:1012E000746173636F2066004175746F6361726728
:1012F0002E66696C2E0046696E2066696C2E00436E
:10130000756368696C6C6F0056656C6F63696461C6
:10131000642056656E74004261736500436F6D70A2
:10132000726F622E76656E74004D6F64656C6F002F
:10133000426F7175696C6C61005072696D65726F96
:1013400020646573636172676120656C2066696CF7
:10135000616D656E746F2C206C7565676F207265AA
:101360007069746520657374612061636369AD6E33
:101370002E00436F6D70726F626163696F6E65738B
:10138000004420626F7175696C6C6100416C66612C
:101390006265746F004F7264656E617200546965B6
:1013A0006D706F005461726A2E2053440043616D6A
:1013B0006269617220656C206964696F6D610043C8
:1013C000616D62696F20646520626F7175696C6C14
:1013D0006100436F6E6669677572616369AD6E2007
:1013E00048570050727565626120646520636172C0
:1013F000676100417061676172206D6F746F726523
:1014000073004D6F76657220656A65730054656D73
:1014100070657261747572610043616C2E20504971
:101420004E44410052657365742063616C69627259
:101430002E2058595A004D6F737472617220656E78
:101440006473746F70730043616C69627261636985
:10145000AD6E2050494400436F72722E20646520A7
:101460006C612063616D61004E6976656C612E2050
:101470004D616C6C6120426173650043616C69620F
:10148000726172205A0043616C6962726172205805
:10149000595A004173697374656E74650050726FB8
:1014A00062616E646F2066696C616D656E746F0059
:1014B000496E74722E20746F646F732066696C2E8F
:1014C0000052657469726120656C2066696C616D9B
:1014D000656E746F20646520696E6D656469617402
:1014E0006F0052656E6F6D627261720043616C2EA7
:1014F000207072696D657261206361702E005365A2
:101500006C656363696F6E6172004C8A6D696E61B0
:1015100020646520616365726F00536F706F727431
:10152000650046616C6C6F7320746F74616C6573D9
:10153000204D4D5500526567697374726F20646564
:101540002066616C6C6F73004573746164A2737480
:10155000696361730043616C696272616369AD6E56
:10156000004361726761206175746F2E2066696C3B
:10157000616D2E00496E74726F64756369722066C6
:10158000696C2E0044657363617267612066696CE3
:101590002E00436172676172206120626F7175690C
:1015A0006C6C610050726563617267612061204DEF
:1015B0004D55004E6F20686179207461726A6574C0
:1015C00061205344004D656E75207461726A6574C4
:1015D00061205344005265616E7564617220696DCB
:1015E000707265732E0050617573617220696D7041
:1015F00072657369AD6E004C6973746F00436F6EF2
:101600006A756E746F206E6F206C6973746F005012
:10161000726563616C656E74617200416A757374A2
:10162000617200416A7573746520656E2076697613
:101630006F205A00566F6C766572206120696D705C
:1016400072696D6972004D6F6E69746F72697A614B
:10165000720041736973742E00556E612076657A4D
:1016600000536F6E69646F00416C746F0053656E58
:10167000736F722046696C2E0043616D62696172FE
:101680002066696C616D656E746F00466C756A6F7B
:101690000056656C6F636964616400436F6D702E02
:1016A00020696D616E6573004E2F44005A2D73657D
:1016B0006E736F72206E722E004D616C6C61004310
:1016C0006F6E6669677572616369AD6E005369001C
:1016D000446574656E657220696D7072657369AD7D
:1016E0006E0056657269662E206172636869766F56
:1016F000004172636869766F20696E636F6D706C0C
:1017000065746F2E20436F6E74696E75617220640C
:101710006520746F646F73206D6F646F733F008416
:1017200041637475616C697A6172004D656E7520F4
:101730007072696E636970616C0045737065726187
:101740006E646F20656E667269616D69656E746F37
:10175000206465206C612062617365207920626F6E
:101760007175696C6C612E00496E696369617220E4
:1017700053656C667465737400496E746572636159
:101780006D626961646F0056656E74732E206672B7
:101790006F6E742F697A7175692E00456A65004C09
:1017A0006F6E67697475642064656C20656A650096
:1017B000506F6C6561207375656C74610046696E6D
:1017C000206E6F20616C63616E7A61646F004669A0
:1017D0006E20646520636172726572610046696E95
:1017E000616C65732064652063617272657261006B
:1017F0004572726F7220646520636F6E657869ADA3
:101800006E00426173652F43616C656E7461646F35
:1018100072004E6F2068617920636F6E657869ADE4
:101820006E0043616C656E7461646F722F546572F3
:101830006D6973746F7200436F6E74726F6C613A8E
:10184000004572726F722053656C66746573742103
:101850000053656E736F722064652066696C2E009C
:1018600056656E742E6675736F723A0056656E74A7
:101870002E20642E206675736F723A0043616C6986
:101880006272617220706F732E696E696369616C38
:101890000046616C6C6F2053656C667465737400F0
:1018A000546F646F206269656E00436F6D70726F74
:1018B00062616E646F2073656E736F72657300434F
:1018C0006F6E74726F6C206675736F7200436F6E0B
:1018D00074726F6C20626173652063616C2E0043CB
:1018E0006F6E74726F6C2073656E736F72205A0026
:1018F000436F6E74726F6C2073656E736F722059D4
:1019000000436F6E74726F6C2073656E736F72201C
:101910005800436F6E74726F6C20656E6473746FE1
:101920007073005461726A657461207265746972C3
:10193000616461004174728A7300456E63656E6410
:1019400069646F004163616C6C6172004D6F646F1C
:101950000052656E642E706C656E6F004573747214
:101960006963746F00417669736F004E696E6775C5
:101970006E6F004675736F722061203238304321DC
:1019800020426F7175696C6C612063616D62696181
:10199000646F207920616A7573742E2061206C61F8
:1019A000206D65646964613F005061726120756EED
:1019B0002063616D62696F20646520626F71756973
:1019C0006C6C612C206C65650A70727573612E6990
:1019D0006F2F6E6F7A7A6C652D6D6B337300436178
:1019E0006C2E20504944207465726D696E6164618B
:1019F0000043616C2E2050494400496D707265733C
:101A000069AD6E20656E20706175736100496D70FF
:101A100072657369AD6E2063616E63656C6164614C
:101A200000436F70696172206964696F6D61207332
:101A3000656C656363696F6E61646F3F0044698ABA
:101A40006D6574726F20626F7175696C6C6120696D
:101A50006D707265736F7261206469666965726525
:101A600020646520636F642E472E0044698A6D658B
:101A700074726F20626F7175696C6C6120496D7052
:101A80007265736F7261206469666965726520644E
:101A90006520636F642E472E20436F6D70727565ED
:101AA0006261206C6F732076616C6F726573206564
:101AB0006E20616A75737465732E004E6F206861C5
:101AC00079206E696E67C06E2066696C616D656EA7
:101AD000746F206361726761646F2E00546F64617C
:101AE00076A261206573206E656365736172696FAC
:101AF00020686163657220756E612063616C696244
:101B000072616369AD6E205A2E205369676120654A
:101B10006C206D616E75616C2C20636170697475E9
:101B20006C6F205072696D65726F73207061736F96
:101B3000732E00496D707265736F7261206E6F2035
:101B40006573748A2063616C696272616461207478
:101B50006F646176A2612E2055736120656C206DE3
:101B6000616E75616C206361706974756C6F205073
:101B700072696D65726F73207061736F732043615A
:101B80006C696272616369AD6E20666C756A6F2EF6
:101B9000005365207265616C697A61728A20656C98
:101BA0002073656C66746573742070617261206364
:101BB000616C696272617220636F6E20707265631E
:101BC0006973696F6E206C61207675656C74612035
:101BD00061206C6120706F73696369AD6E20696EFE
:101BE000696369616C2073696E2073656E736F72CF
:101BF00065732E0053652068616E20656E636F6E9D
:101C0000747261646F20616A757374657320616EAC
:101C1000746572696F7265732E20536520616A75F1
:101C2000737461726120656C205049442C206C6F84
:101C300073207061736F732064656C2065787472B3
:101C400075736F722C206574632E00417669736F13
:101C50003A2074616E746F20656C207469706F2017
:101C6000646520696D707265736F726120636F6D5A
:101C70006F20656C207469706F206465206C612032
:101C8000706C6163612068616E2063616D6269617F
:101C9000646F2E00417669736F3A2068612063613A
:101CA0006D626961646F20656C207469706F206477
:101CB0006520696D707265736F72612E004176697F
:101CC000736F3A20656C207469706F2064652070B2
:101CD0006C6163612068612063616D626961646F3A
:101CE0002E004C8A6D696E61004F6375727269AD2A
:101CF00020756E206572726F7220696E65737065F3
:101D00007261646F2E0043616D62696F20646520AB
:101D100066696C616D656E746F204D3630302E20B3
:101D200043617267756520756E2066696C616D65CB
:101D30006E746F206E7565766F206F206578707594
:101D40006C736520656C20616E746572696F722EAC
:101D50000052657469726520656C2066696C616DFE
:101D6000656E746F20657870756C7361646F206444
:101D700065206C612070617274652066726F6E748C
:101D8000616C206465206C61204D4D552E004669C4
:101D90006C616D656E746F206465746563746164F5
:101DA0006F20696E65737065726164616D656E74D4
:101DB000652E2041736567C072617465206465207B
:101DC000717565206E6F2068617961206E696E673C
:101DD000C06E2066696C616D656E746F20636172A0
:101DE0006761646F2E20436F6D707275656261204C
:101DF0006C6F732073656E736F72657320792065E5
:101E00006C206361626C6561646F2E004572726F55
:101E10007220696E7465726E6F20646520656A65F4
:101E200063756369AD6E2E205265696E6963696181
:101E3000206C61204D4D55206F2061637475616C7D
:101E4000697A6120656C206669726D776172652EB2
:101E5000004C61207665727369AD6E206465206602
:101E600069726D77617265206465206C61204D4DEB
:101E70005520657320696E636F6D70617469626C63
:101E80006520636F6E20656C204657206465206C6A
:101E90006120696D707265736F72612E2041637489
:101EA00075616C697A61722061206C61207665725F
:101EB0007369AD6E20332E302E332E004572726F53
:101EC0007220696E7465726E6F2064656C2066693D
:101ED000726D77617265204D4D552C207265696E6B
:101EE0006963696120656C204D4D552E00456C205D
:101EF00066696C2E20736F6C6963697461646F200E
:101F00006E6F206573748A20646973706F6E696286
:101F10006C6520656E2065737465206861726477F6
:101F20006172652E2052657669736120656C20634D
:101F3000AD6469676F20472070617261207369200A
:101F4000656C20A26E6469636520646520686572B3
:101F500072616D69656E7461206573748A2066753F
:101F60006572612064652072616E676F202854304D
:101F70002D5434292E004E6F2073652070756564D2
:101F800065207265616C697A6172206C61206163A1
:101F90006369AD6E2C2066696C616D656E746F202F
:101FA0007961206361726761646F2E205072696D80
:101FB00065726F2064657363617267612E004D4DB9
:101FC00055206E6F20726573706F6E646520636F4D
:101FD0007272656374616D656E74652E20526576EC
:101FE000697361206C6F73206361626C6573207923
:101FF00020636F6E6563746F7265732E004C612091
:102000004D4D55206E6F20726573706F6E64652E36
:1020100020526576697361206C6F73206361626C16
:102020006573207920636F6E6563746F7265732EBC
:10203000004D8A7320646574616C6C6573206F6EEB
:102040006C696E652E00456C2074656E736F72202E
:102050006E6F20686163657220686F6D6520636FC5
:102060007272656374616D656E74652E20436F6D69
:102070007072756562612073692068617920616C96
:10208000676F2071756520626C6F71756561207373
:1020900075206D6F76696D69656E746F2E004E6F79
:1020A000207365207075656465206D6F766572209C
:1020B00053656C6563746F72206F2054656E736F27
:1020C000722E00456C2073656C6563746F72206EB0
:1020D0006F20686163657220686F6D6520636F7241
:1020E00072656374616D656E74652E20436F6D70EB
:1020F00072756562612073692068617920616C671F
:102100006F2071756520626C6F71756561207375E4
:10211000206D6F76696D69656E746F2E0045727201
:102120006F7220616C2063617267617220656E203E
:102130006C61206578747275736F722E20496E73AE
:1021400070656363696F6E61206C6120666F726D8C
:1021500061206465206C612070756E746120646517
:102160006C2066696C616D656E746F2E20526566B9
:10217000696E61206C612063616C69627261636980
:10218000AD6E2064656C2073656E736F722C207366
:1021900069206573206E656365736172696F2E00D7
:1021A000456C2073656C6563746F72206E6F20736D
:1021B00065207075656465206D6F76657220646555
:1021C0006269646F2061207175652046494E444103
:1021D000206465746563746120756E2066696C6146
:1021E0006D656E746F2E2041736567C07261746592
:1021F00020646520717565206E6F206861796120AB
:1022000066696C2E20656E20656C2073656C656355
:10221000746F722079207175652046494E444120C3
:1022200066756E63696F6E6520636F727265637445
:10223000616D656E74652E00456C2073656E736FFD
:10224000722064652066696C616D656E746F2073C1
:1022500065206163746976AD2064656D6173696141
:10226000646F2070726F6E746F20616C2063617296
:1022700067617220656C206578747275736F722E59
:1022800020436F6D70727565626120717565206E97
:102290006F2068612D7961206E61646120617461D5
:1022A000736361646F20656E20656C207475626F66
:1022B000206465207465666CAD6E2079207175654B
:1022C00020656C2073656E736F72207661206F6B72
:1022D0002E00456C206D6F746F72206465206C61F8
:1022E00020706F6C65612073652068612070617279
:1022F00061646F2E2041736567C0726174652064EC
:102300006520717565206C6120706F6C656120704F
:1023100075656465206D6F766572736520792063DD
:102320006F6D70727565626120656C206361626CAF
:102330006561646F2E00456C2073656E736F72204B
:1023400064652066696C616D656E746F206E6F20C8
:1023500073652061706167AD206D69656E7472612F
:1023600073207365206465736361726761626120C5
:10237000656C2066696C616D656E746F2E204173AB
:102380006567C0726174652064652071756520653C
:102390006C2066696C616D656E746F207075656424
:1023A00065206D6F7665727365207920656C20738A
:1023B000656E736F722066756E63696F6E612E0055
:1023C000456C2073656E736F722064652066696C5E
:1023D000616D656E746F206E6F207365206163742C
:1023E0006976AD20616C2063617267617220656CF3
:1023F0002066696C616D656E746F2E204173656730
:10240000C0726174652064652071756520656C20FB
:1024100066696C616D656E746F206C6C6567AD206C
:10242000616C2073656E736F722079207175652001
:102430009A7374652066756E63696F6E612E0046CF
:10244000494E4441206E6F2073652061706167AD15
:10245000206D69656E747261732064657363617267
:102460006761626120656C2066696C616D656E7480
:102470006F2E20496E74656E7461206465736361AC
:1024800072676172206D616E75616C6D656E7465E9
:102490002E20436F6D2D20707275656261207175FD
:1024A0006520656C2066696C2D20616D656E746FAA
:1024B000207075656465206D6F766572736520792F
:1024C0002046494E44412066756E63696F6E612EE9
:1024D0000046494E4441206E6F207365206163744D
:1024E0006976AD20616C2063617267617220656CF2
:1024F0002066696C616D656E746F2E20417365672F
:10250000C0726174652064652071756520656C20FA
:1025100066696C616D656E746F20707565646520A9
:102520006D6F766572736520792046494E4441206F
:1025300066756E63696F6E612E00446573616374C6
:102540002E005061726172004361726761720044D3
:102550006573632E005265696E742E0053656E7349
:102560006962696C6964616400436F6E74696E7559
:10257000616E2E20696D7072657369AD6E00436186
:102580006C656E74616E646F2050494E4441004327
:10259000616C696272616369AD6E204F4B0043618B
:1025A0006C696272616E646F205A004261736520CB
:1025B0007072657061726164610043616C656E7414
:1025C000616E646F20426173650043616C656E7477
:1025D000616E646F206163616261646F2E004361AC
:1025E0006C656E74616E646F2E2E2E00556C74696E
:1025F0006D6120696D7072657369AD6E0046616CC6
:102600006C6F73204D4D55004361726761204D4DD5
:10261000552066616C6C610046616C6C6F20726560
:1026200064204D4D550043616D62696F73206D618B
:1026300074657269616C657300C06C74696D6F73E9
:1026400020696D702E2066616C6C6F730046616C42
:102650006C6F7320746F74616C65730046696C2EC7
:10266000206163616261646F0054656D70657261C1
:10267000747572617300496E666F2073656E736F57
:102680007200496E666F2E2064656C2065787472E6
:1026900075736F7200446574616C6C65732063615F
:1026A0006C2E2058595A004469722E2049502069D6
:1026B0006D707265736F72613A00646573636F6EFB
:1026C0006F6369646F004D4D5520636F6E65637471
:1026D00061646F0046656368613A007061726120F1
:1026E0006465736361726761722066696C2E007045
:1026F0006172612063617267617220656C20666936
:102700006C2E0050756C736120656C206469616C7F
:102710000050726563616C656E742E20636F727415
:1027200061720050726563616C656E742E2065780D
:1027300070756C7361720050726563616C656E7464
:102740002E20646573636172676172005072656305
:10275000616C656E742E2063617267617200456EF4
:102760006672696172005365206578747275796567
:102770002066696C616D656E746F207920636F6E81
:1027800020656C20636F6C6F7220636F727265637B
:10279000746F3F00457870756C736172004C6120F6
:1027A0006361726761206175746F6D8A74696361BA
:1027B000206573748A2061637469766164612C207A
:1027C00070756C736520656C206469616C20652090
:1027D000696E736572746520656C2066696C616DE5
:1027E000656E746F2E2E2E0046696C616D656E7479
:1027F0006F20746F74616C005469656D706F207424
:102800006F74616C20696D702E0046696C616D6536
:102810006E746F20757361646F005469656D706FBD
:1028200020646520696D702E00456D70756A6120A9
:102830006861737461204653656E736F72004D6FEB
:102840007669656E646F2073656C6563746F720082
:10285000526574726165722064656C2046494E440D
:102860004100457870756C73616E646F2066696CA9
:10287000616D656E746F004170617263616E646F4B
:102880002073656C6563746F720053656C65637467
:102890006F7220766F6C7669656E646F0052656149
:1028A0006C697A616E646F20636F72746500456D48
:1028B00070756A616E646F2066696C616D656E74B7
:1028C0006F00507265706172616E646F2063756332
:1028D00068696C6C6100456C696769656E646F203E
:1028E000687565636F2066696C2E0044657363616B
:1028F0007267616E646F2066696C2E0045525220CB
:1029000046616C6C6F20544D430045525220417912
:102910007564612066696C616D656E746F00455207
:102920005220496E7465726E6F0045525220457395
:1029300070657261207573756172696F005465729C
:102940006D2E206D6F76696D69656E746F730045CD
:1029500076697461206D6F7264657200416C696D97
:10296000656E742E2061206C6120626F712E0041B3
:102970006C696D656E742E20616C2065787472755B
:10298000736F7200416C696D656E7461206861736C
:1029900074612046494E4441004465736361726727
:1029A0002E20686173746120706F6C6561004465EE
:1029B00073636172672E2068617374612046494EAB
:1029C000444100536F6C74616E646F2074656E7364
:1029D0006F7200456E67616E6368616E646F20742C
:1029E000656E736F72004552524F522044455343F7
:1029F0004F4E4F4349444F0043414D42494F2044BD
:102A0000452046494C414D454E544F0046494C41A6
:102A10004D454E544F20455850554C5341444F005E
:102A20004445534341524741204D414E55414C008E
:102A30004552524F5220454A4543554349AE4E20D8
:102A40004657004143542E204657204D4D552050A7
:102A500052454349534100434F4C41204C4C454E55
:102A60004100484552522E20494E56414C4944415E
:102A70000046494C2E205941204341524741444F82
:102A8000004552524F5220434F4D554E494341430A
:102A900049AE4E004D4D55204E4F20524553504F9C
:102AA0004E4445004D4D552053454C4654455354D6
:102AB0002046414C4C4F00434F52544F2044524902
:102AC00056455220544D43004552524F52205342D6
:102AD00052564F4C54414A4520544D4300524553A1
:102AE00045542044524956455220544D43004552C6
:102AF000524F522044524956455220544D430045AE
:102B000052524F5220534F42524543414C20544D54
:102B10004300415649534F20544D432044454D2EC8
:102B20002043414C4F520054454E534F523A20459A
:102B300052524F52204D4F562E0054454E534F5235
:102B40003A204552524F5220484F4D450053454C74
:102B50004543542E2053494E204D4F564552534520
:102B60000053454C4543542E2053494E20484F4D69
:102B7000450046414C4C2E20434152474152204192
:102B800020455854522E00494E5350454343494F17
:102B90004E41522046494E4441004653454E534F04
:102BA00052204D55592050524F4E544F00504F4CCB
:102BB00045413A204552524F52204D4F562E004625
:102BC00053454E534F522041544153434F204649A1
:102BD0004C2E004653454E534F52204E4F205345E6
:102BE0002041435449564F0046494E4441204154E8
:102BF0004153434F2046494C2E0046494E44412004
:102C00004E4F2053452041435449564F0056656E60
:102C100074696C61646F72206E6F20676972610005
:102C200056656E74696C61646F7220676972616E5B
:102C3000646F0056656E742E20697A7175696572CD
:102C4000646F3F0056656E742E2066726F6E7461FD
:102C50006C3F00546573742076656E74696C6164B2
:102C60006F7265730043616C696272616369AD6E16
:102C70002058595A20636F7272656374612E204C1C
:102C800061206465737669616369AD6E2073652048
:102C9000636F7272656769728A206175746F6D8A7D
:102CA000746963616D656E74652E0043616C696261
:102CB00072616369AD6E2058595A20636F727265F4
:102CC0006374612E204C6F7320656A657320582FE2
:102CD00059206573748A6E206C69676572616D65D1
:102CE0006E746520646573766961646F732E20422B
:102CF00075656E2074726162616A6F210043616C58
:102D0000696272616369AD6E2058595A206F6B2EEB
:102D100020456A657320582F592070657270656E62
:102D2000646963756C617265732E20456E686F729D
:102D3000616275656E61210043616C6962726163F5
:102D400069AD6E2058595A20636F6D70726F6D6552
:102D5000746964612E2050756E746F2066726F6E98
:102D600074616C206465726563686F206E6F2061AA
:102D70006C63616E7A61626C652E0043616C69629E
:102D800072616369AD6E2058595A20636F6D70721D
:102D90006F6D65746964612E2050756E746F732059
:102DA00066726F6E74616C6573206E6F20616C6308
:102DB000616E7A61626C65732E0043616C69627248
:102DC000616369AD6E2058595A2066616C6C61640C
:102DD0002E2050756E746F2066726F6E74616C2059
:102DE0006465726563686F206E6F20616C63616EED
:102DF0007A61626C652E0043616C6962726163691D
:102E0000AD6E2058595A2066616C6C6964612E2041
:102E100050756E746F732066726F6E74616C65733B
:102E2000206E6F20616C63616E7A61626C65732ED7
:102E30000043616C696272616369AD6E2058595AD2
:102E40002066616C6C6964612E20436F6E73756CD3
:102E5000746120656C206D616E75616C2E0043613C
:102E60006C696272616369AD6E2058595A2066615F
:102E70006C6C6964612E2050756E746F732064658C
:102E80002063616C696272616369AD6E20656E205A
:102E90006C612062617365206E6F20656E636F6E7A
:102EA000747261646F732E00436F6C6F6361206C8A
:102EB00061206C616D2E20646520616365726F20F6
:102EC000656E206C6120626173652E0044697374C5
:102ED000616E63696120656E747265206C6120703B
:102EE000756E74612064656C20626F7175696C6CBD
:102EF000612079206C612073757065726669636901
:102F000065206465206C6120626173652061756E67
:102F1000206E6F2066696A6164612E205369676163
:102F200020656C206D616E75616C2C206361706929
:102F300074756C6F205072696D65726F732050618B
:102F4000736F732E00436F6C6F71756520756E61C2
:102F500020686F6A6120646520706170656C206410
:102F60006562616A6F206465206C6120626F7175B3
:102F7000696C6C6120647572616E7465206C61208F
:102F800063616C696272616369AD6E206465206C17
:102F90006F73207072696D65726F73203420707565
:102FA0006E746F732E205369206C6120626F71758F
:102FB000696C6C6120636F676520656C207061705F
:102FC000656C2C2061706167756520696E6D656444
:102FD000696174616D656E74652E0042757363611D
:102FE0006E646F2070756E746F2064652063616C11
:102FF000696272616369AD6E2062617365004D69DB
:103000006469656E646F20616C74757261206465BB
:103010006C2070756E746F2064652063616C6962EA
:1030200072616369AD6E004C696D70696120626F99
:103030007175696C6C6120706172612063616C698B
:103040006272616369AD6E2E20436C6963206375A3
:10305000616E646F206163616265732E0049722046
:10306000616C206F726967656E00436F7274617284
:103070002066696C616D656E7400457870756C735F
:103080006172206465204D4D5500496E74726F6405
:10309000756369656E646F2066696C616D2E004DA5
:1030A0004D55205265696E74656E746F3A20526595
:1030B0007374617572616E646F2074656D70657292
:1030C00061747572612E2E2E004F7264656E616E92
:1030D000646F206172636869766F7300416C677515
:1030E0006E6F73206172636869766F73206E6F20F4
:1030F0007365206F7264656E61728A6E2E204D8AD0
:1031000078696D6F20313030206172636869766F45
:103110007320706F722063617270657461207061DA
:103120007261206F7264656E61722E00504152416F
:10313000444100496E6100416374000000000000DA
:10314000000000000000000000000000000000007F
:10315000000000000000000000000000000000006F
:10316000000000000000000000000000000000005F
:10317000000000000000000000000000000000004F
:103600000000536F6D652070726F626C656D206590
:103610006E636F756E74657265642C205A2D6C65CF
:1036200076656C696E6720656E666F72636564208F
:103630002E2E2E0001004D65736820626564206C9B
:103640006576656C696E67206661696C65642E20BD
:103650005072696E742063616E63656C65642E00E0
:10366000020048656174696E672064697361626C09
:103670006564206279207361666574792074696D70
:1036800065722E000300472D636F646520736C69BB
:1036900063656420666F7220612064696666657286
:1036A000656E74206C6576656C2E000400472D6392
:1036B0006F646520736C6963656420666F72206156
:1036C00020646966666572656E74206C6576656CEB
:1036D0002E20506C656173652072652D736C696373
:1036E0006520746865206D6F64656C206167616931
:1036F0006E2E000500472D636F646520736C69634F
:10370000656420666F722061206E65776572206641
:1037100069726D776172652E000600472D636F64D4
:103720006520736C6963656420666F722061206E2A
:1037300065776572206669726D776172652E2050BB
:103740006C6561736520757064617465207468656B
:10375000206669726D776172652E000700472D63E0
:103760006F646520736C6963656420666F722061A5
:1037700020646966666572656E74207072696E7425
:10378000657220747970652E000800472D636F64A0
:103790006520736C6963656420666F7220612064C4
:1037A0006966666572656E74207072696E746572A2
:1037B00020747970652E20506C6561736520726588
:1037C0002D736C69636520746865206D6F64656C2A
:1037D00020616761696E2E00090050726573732065
:1037E000746865206B6E6F6220746F2070726568FC
:1037F000656174206E6F7A7A6C6520616E642063F7
:103800006F6E74696E75652E000A00506C65617389
:103810006520707265737320746865206B6E6F62CB
:1038200020746F20756E6C6F61642066696C616DC9
:10383000656E74000B00616E642070726573732096
:10384000746865206B6E6F62000C00496E73657260
:10385000742066696C616D656E74000D00436F6C59
:103860006F72206E6F7420636F7272656374000EE6
:103870000046696C616D656E74206E6F74206C6FAC
:1038800061646564000F004368616E67656420636E
:103890006F72726563746C790010004C6F616469BB
:1038A0006E6720636F6C6F720011004368616E6712
:1038B00065207375636365737321001200506C6536
:1038C000617365206F70656E2069646C657220613C
:1038D0006E642072656D6F76652066696C616D65DA
:1038E0006E74206D616E75616C6C792E00130057DB
:1038F00061732066696C616D656E7420756E6C6FA6
:103900006164207375636365737366756C3F00143F
:1039100000506C6561736520757067726164652E17
:103920000015004E6577206669726D7761726520BB
:1039300076657273696F6E20617661696C61626C25
:10394000653A00160057616974696E6720666F7288
:103950002050494E44412070726F626520636F6F42
:103960006C696E67001700506C6561736520776144
:1039700069740018004E6F206D6F76652E00190077
:103980005761697420666F7220757365722E2E2ED2
:10399000001A00537461626C6520616D6269656E26
:1039A000742074656D706572617475726520323152
:1039B0002D323643206973206E656564656420612D
:1039C000207269676964207374616E642069732072
:1039D00072657175697265642E001B00506C6561BB
:1039E00073652072756E2058595A2063616C696244
:1039F000726174696F6E2066697273742E001C00A8
:103A0000426564206C6576656C696E6720666169E5
:103A10006C65642E2053656E736F72206469646EEA
:103A2000277420747269676765722E20446562721C
:103A30006973206F6E206E6F7A7A6C653F205761D4
:103A40006974696E6720666F722072657365742E83
:103A5000001D005072656865617420746865206E91
:103A60006F7A7A6C6521001E004552524F523A001F
:103A70001F00592064697374616E63652066726FFC
:103A80006D206D696E0020004C6566740021005247
:103A9000696768740022004D656173757265642002
:103AA000736B6577002300536C6967687420736BD0
:103AB000657700240053657665726520736B6577C2
:103AC0000025005B303B305D20706F696E74206FA5
:103AD000666673657400260041646A757374696E66
:103AE00067205A002700526561722073696465205F
:103AF0005BE46D5D00280046726F6E74207369642C
:103B0000655BE46D5D002900526967687420736924
:103B100064655BE46D5D002A004C65667420736922
:103B20006465205BE46D5D002B0053657420746553
:103B30006D70657261747572653A002C0041726532
:103B4000206C65667420616E6420726967687420F9
:103B50005A2D63617272696167657320616C6C20B4
:103B600075703F002D0043616C6962726174696E0B
:103B7000672058595A2E20526F74617465207468FA
:103B800065206B6E6F6220746F206D6F7665207498
:103B90006865205A2063617272696167652075707B
:103BA00020746F2074686520656E642073746F7074
:103BB000706572732E20436C69636B207768656E45
:103BC00020646F6E652E002E0043616C6962726125
:103BD00074696E67205A2E20526F74617465207468
:103BE0006865206B6E6F6220746F206D6F76652044
:103BF000746865205A206361727269616765207517
:103C00007020746F2074686520656E642073746F13
:103C100070706572732E20436C69636B20776865E2
:103C20006E20646F6E652E002F0050494E44412077
:103C300063616C6962726174696F6E206661696C40
:103C4000656400300050494E44412063616C6962F4
:103C5000726174696F6E2069732066696E6973683A
:103C6000656420616E64206163746976652E204905
:103C7000742063616E2062652064697361626C65A3
:103C80006420696E206D656E752053657474696E6D
:103C900067732D3E50494E44412063616C2E0031C4
:103CA0000045787472756465720032004D6F7665F8
:103CB000205A0033004D6F766520590034004D6F57
:103CC00076652058003500536865657420252E37C9
:103CD000730A5A206F66667365743A20252B312E5D
:103CE00033666D6D0A2563436F6E74696E75650A80
:103CF00025635265736574003600506C65617365A9
:103D0000206C6F61642066696C616D656E742066FD
:103D1000697273742E00370053656C656374206696
:103D2000696C616D656E743A00380043616E63655D
:103D30006C00390052756E6E696E672057697A6142
:103D400072642077696C6C2064656C6574652063AF
:103D5000757272656E742063616C696272617469F8
:103D60006F6E20726573756C747320616E6420735E
:103D7000746172742066726F6D207468652062656C
:103D800067696E6E696E672E003A005072656865ED
:103D90006174696E67206E6F7A7A6C652E20506C44
:103DA0006561736520776169742E003B00506C6516
:103DB00061736520696E736572742066696C616DEC
:103DC000656E7420696E746F207468652065787400
:103DD00072756465722C207468656E2070726573EC
:103DE0007320746865206B6E6F6220746F206C6F37
:103DF00061642069742E003C00506C65617365201D
:103E0000696E736572742066696C616D656E74208D
:103E1000696E746F207468652066697273742074AB
:103E2000756265206F6620746865204D4D552C20A5
:103E30007468656E20707265737320746865206B9A
:103E40006E6F6220746F206C6F61642069742E0045
:103E50003D00546865207072696E746572207769E0
:103E60006C6C207374617274207072696E74696E08
:103E7000672061207A69672D7A6167206C696E65B9
:103E80002E20526F7461746520746865206B6E6FAC
:103E90006220756E74696C20796F7520726561633C
:103EA0006820746865206F7074696D616C20686546
:103EB000696768742E20436865636B2074686520A9
:103EC000706963747572657320696E20746865200B
:103ED00068616E64626F6F6B202843616C69627207
:103EE0006174696F6E2063686170746572292E0059
:103EF0003E0053656C6563742074656D7065726116
:103F000074757265207768696368206D6174636891
:103F1000657320796F7572206D6174657269616C6B
:103F20002E003F0053656C65637420612066696CE8
:103F3000616D656E7420666F7220746865204669D5
:103F4000727374204C617965722043616C6962728E
:103F50006174696F6E20616E642073656C65637453
:103F600020697420696E20746865206F6E2D7363FC
:103F70007265656E206D656E752E0040004E6F7720
:103F800020492077696C6C2063616C69627261748E
:103F9000652064697374616E63652062657477651A
:103FA000656E20746970206F6620746865206E6F7E
:103FB0007A7A6C6520616E642068656174626564FC
:103FC00020737572666163652E0041005A2063613B
:103FD0006C6962726174696F6E207265636F6D6D7A
:103FE000656E6465642E2052756E206974206E6F54
:103FF000773F004200506C656173652072656D6F9C
:10400000766520737465656C2073686565742066D9
:10401000726F6D20686561746265642E00430049AB
:104020007320737465656C207368656574206F6EAA
:1040300020686561746265643F004400506C65618E
:10404000736520636865636B206F75722068616EAD
:1040500064626F6F6B20616E64206669782074689B
:10406000652070726F626C656D2E205468656E20DD
:10407000726573756D65207468652057697A617221
:1040800064206279207265626F6F74696E67207454
:104090006865207072696E7465722E004500416C0F
:1040A0006C20697320646F6E652E20486170707992
:1040B000207072696E74696E6721004600596F75D1
:1040C0002063616E20616C7761797320726573750E
:1040D0006D65207468652057697A61726420667224
:1040E0006F6D2043616C6962726174696F6E202D1F
:1040F0003E2057697A6172642E0047004966207934
:104100006F752068617665206164646974696F6E9B
:10411000616C20737465656C207368656574732CBD
:104120002063616C6962726174652074686569728C
:10413000207072657365747320696E2053657474A2
:10414000696E6773202D2048572053657475702061
:104150002D20537465656C207368656574732E003B
:104160004800506C6561736520636C65616E206802
:1041700065617462656420616E64207468656E2098
:10418000707265737320746865206B6E6F622E00A9
:104190004900446F20796F752077616E7420746FC9
:1041A00020726570656174206C617374207374652E
:1041B0007020746F20726561646A7573742064691D
:1041C0007374616E6365206265747765656E206ED9
:1041D0006F7A7A6C6520616E6420686561746265CF
:1041E000643F004A0053656C656374206E6F7A7A91
:1041F0006C6520707265686561742074656D7065AA
:10420000726174757265207768696368206D617486
:104210006368657320796F7572206D61746572696A
:10422000616C2E004B0049732066696C616D656E90
:1042300074206C6F616465643F004C004E6F7720A2
:10424000492077696C6C2070726568656174206EB6
:104250006F7A7A6C6520666F7220504C412E004D4B
:1042600000492077696C6C2072756E207A2063613A
:104270006C6962726174696F6E206E6F772E004E8A
:10428000004E6F772072656D6F76652074686520CB
:1042900074657374207072696E742066726F6D201D
:1042A000737465656C2073686565742E004F0050EB
:1042B0006C656173652072656D6F766520736869E2
:1042C0007070696E672068656C70657273206669CE
:1042D0007273742E005000492077696C6C207275DF
:1042E0006E2078797A2063616C6962726174696F9B
:1042F0006E206E6F772E2049742077696C6C207465
:10430000616B6520757020746F203234206D696E8A
:10431000732E00510046697273742C20492077690E
:104320006C6C2072756E207468652073656C6674A1
:1043300065737420746F20636865636B206D6F73A1
:104340007420636F6D6D6F6E20617373656D626C49
:10435000792070726F626C656D732E00520048692F
:104360002C204920616D20796F7572204F7269672A
:10437000696E616C205072757361206933207072B0
:10438000696E7465722E20576F756C6420796F7535
:10439000206C696B65206D6520746F20677569649A
:1043A0006520796F75207468726F7567682074680E
:1043B000652073657475702070726F636573733FE9
:1043C00000530048692C204920616D20796F757277
:1043D000204F726967696E616C205072757361203D
:1043E0006933207072696E7465722E204920776976
:1043F0006C6C20677569646520796F7520746872CC
:104400006F75676820612073686F727420736574BC
:1044100075702070726F636573732C20696E2077DE
:104420006869636820746865205A2D617869732013
:1044300077696C6C2062652063616C69627261747B
:1044400065642E205468656E2C20796F752077691D
:104450006C6C20626520726561647920746F2070D5
:1044600072696E742E0054005061757365005500BA
:10447000465320416374696F6E005600436F6E743B
:104480002E005700462E206A616D206465746563B6
:1044900074005800462E206175746F6C6F61640063
:1044A0005900462E2072756E6F7574005A00437560
:1044B00074746572005B0046616E2073706565649C
:1044C000005C00426564005D0046616E73206368B5
:1044D00065636B005E004D6F64656C005F004E6F3E
:1044E0007A7A6C65006000506C6561736520756E4A
:1044F0006C6F6164207468652066696C616D656EBF
:10450000742066697273742C207468656E207265FD
:1045100070656174207468697320616374696F6E7B
:104520002E006100436865636B730062004E6F7A12
:104530007A6C6520642E006300416C70686162656E
:1045400074006400536F727400650054696D6500F7
:1045500066004E6F726D616C0067005344206361AA
:10456000726400680053656C656374206C616E67EB
:10457000756167650069004E6F7A7A6C65206368C3
:10458000616E6765006A0048572053657475700056
:104590006B004C6F6164696E672054657374006CC6
:1045A0000044697361626C65207374657070657234
:1045B00073006D004D6F76652061786973006E0041
:1045C00054656D7065726174757265006F00504955
:1045D0004E44412063616C2E007000526573657417
:1045E0002058595A2063616C6962722E0071005321
:1045F000686F7720656E642073746F70730072004B
:104600005049442063616C6962726174696F6E0025
:104610007300426564206C6576656C20636F72720E
:104620006563740074004D65736820426564204CB6
:104630006576656C696E6700750043616C696272CE
:10464000617465205A00760043616C69627261741E
:10465000652058595A00770053656C667465737409
:1046600000780057697A6172640079005465737448
:10467000696E672066696C616D656E74007A004CC6
:104680006F616420416C6C007B00506C65617365E8
:104690002070756C6C206F75742066696C616D6537
:1046A0006E7420696D6D6564696174656C79007CF8
:1046B000005265736574007D0052656E616D650022
:1046C0007E004669727374206C6179657220636143
:1046D0006C2E007F0053656C65637400800053741A
:1046E00065656C207368656574730081005375702F
:1046F000706F72740082004661696C20737461741B
:1047000073204D4D550083004661696C20737461C0
:104710007473008400537461746973746963730003
:10472000850043616C6962726174696F6E00860016
:104730004175746F4C6F61642066696C616D656E64
:10474000740087004C6F61642066696C616D656EF2
:1047500074008800556E6C6F61642066696C616DD1
:10476000656E740089004C6F616420746F206E6FF9
:104770007A7A6C65008A005072656C6F616420748F
:104780006F204D4D55008B004E6F205344206361C8
:104790007264008C005072696E742066726F6D20B6
:1047A0005344008D00526573756D65207072696E9B
:1047B00074008E005061757365207072696E7400AC
:1047C0008F005365742052656164790090005365D1
:1047D00074206E6F7420526561647900910050728C
:1047E000656865617400920054756E650093004CB5
:1047F0006976652061646A757374205A009400526A
:10480000657072696E74009500496E666F207363FF
:104810007265656E0096004173736973740097004A
:104820004F6E6365009800536F756E640099004C7D
:104830006F7564009A0046696C2E2073656E736F05
:1048400072009B004368616E67652066696C616DEC
:10485000656E74009C00466C6F77009D0053706518
:104860006564009E004D61676E65747320636F6DB3
:10487000702E009F004E2F4100A0005A2D70726FC5
:104880006265206E722E00A1004D65736800A20063
:1048900053657474696E677300A30059657300A44F
:1048A000004E6F00A50053746F70207072696E74B3
:1048B00000A600436865636B696E672066696C6576
:1048C00000A70046696C6520696E636F6D706C654A
:1048D00074652E00A800845265667265736800A92D
:1048E000004D61696E00AA0057616974696E6720A6
:1048F000666F72206E6F7A7A6C6520616E642062DA
:10490000656420636F6F6C696E6700AB0053656C04
:104910006674657374204F4B00AC0053656C66740D
:1049200065737420737461727400AD0053776170A5
:1049300070656400AE0046726F6E742F6C656674AD
:104940002066616E7300AF004178697300B000416A
:10495000786973206C656E67746800B1004C6F6F86
:1049600073652070756C6C657900B200456E647378
:10497000746F70206E6F742068697400B300456EA8
:104980006473746F7000B4004D6F746F7200B50083
:10499000456E6473746F707300B600576972696E08
:1049A00067206572726F7200B7004265642F4865B8
:1049B0006174657200B8004E6F7420636F6E6E652F
:1049C0006374656400B9004865617465722F54684A
:1049D00065726D6973746F7200BA00506C656173B3
:1049E0006520636865636B3A00BB0053656C667451
:1049F000657374206572726F722100BC0046696C29
:104A0000616D656E742073656E736F7200BD0050CA
:104A100072696E742066616E3A00BE00486F7465FC
:104A20006E642066616E3A00BF0043616C69627219
:104A30006174696E6720686F6D6500C00053656CB6
:104A40006674657374206661696C656400C10041B9
:104A50006C6C20636F727265637400C2004368659A
:104A6000636B696E672073656E736F727300C3004A
:104A7000436865636B696E6720686F74656E640078
:104A8000C400436865636B696E672062656400C536
:104A900000436865636B696E67205A2061786973AB
:104AA00000C600436865636B696E672059206178B2
:104AB000697300C700436865636B696E672058209F
:104AC0006178697300C800436865636B696E67202D
:104AD000656E6473746F707300C900436172642003
:104AE00072656D6F76656400CA004261636B00CBCE
:104AF000004175746F20706F77657200CC00536948
:104B00006C656E7400CD004D6F646500CE00486921
:104B1000676820706F77657200CF005374726963A5
:104B20007400D0005761726E00D1004E6F6E650048
:104B3000D200486F74656E6420617420323830434F
:104B400021204E6F7A7A6C65206368616E676564B8
:104B500020616E64207469676874656E6564207492
:104B60006F2073706563733F00D300466F722061DE
:104B7000204E6F7A7A6C65206368616E676520707D
:104B80006C6561736520726561640A70727573612A
:104B90002E696F2F6E6F7A7A6C652D6D6B33730093
:104BA000D4005049442063616C2E2066696E69739D
:104BB00068656400D5005049442063616C2E00D6BE
:104BC000005072696E742070617573656400D7005F
:104BD0005072696E742061626F7274656400D800EF
:104BE000436F70792073656C6563746564206C61D4
:104BF0006E67756167653F00D9004E6F7A7A6C65A4
:104C0000206469616D6574657220646966666572A9
:104C1000732066726F6D2074686520472D636F6422
:104C2000652E00DA004E6F7A7A6C65206469616DDA
:104C30006574657220646966666572732066726F5A
:104C40006D2074686520472D636F64652E20506C5D
:104C50006561736520636865636B207468652076A1
:104C6000616C756520696E2073657474696E677315
:104C70002E00DB005468657265206973206E6F201A
:104C800066696C616D656E74206C6F616465642E1D
:104C900000DC005468657265206973207374696C68
:104CA0006C2061206E65656420746F206D616B659A
:104CB000205A2063616C6962726174696F6E2E2084
:104CC000506C6561736520666F6C6C6F77207468DB
:104CD00065206D616E75616C2C2063686170746510
:104CE000722046697273742073746570732C20731C
:104CF000656374696F6E2043616C69627261746987
:104D00006F6E20666C6F772E00DD005072696E74D6
:104D1000657220686173206E6F74206265656E2015
:104D200063616C69627261746564207965742E20B8
:104D3000506C6561736520666F6C6C6F772074686A
:104D400065206D616E75616C2C206368617074659F
:104D5000722046697273742073746570732C2073AB
:104D6000656374696F6E2043616C69627261746916
:104D70006F6E20666C6F772E00DE0053656C667474
:104D80006573742077696C6C2062652072756E2083
:104D9000746F2063616C6962726174652061636322
:104DA00075726174652073656E736F726C65737371
:104DB000207265686F6D696E672E00DF004F6C644E
:104DC0002073657474696E677320666F756E642EE8
:104DD0002044656661756C74205049442C204573ED
:104DE00074657073206574632E2077696C6C206223
:104DF00065207365742E00E0005761726E696E67FE
:104E00003A20626F7468207072696E7465722074E3
:104E100079706520616E64206D6F74686572626F71
:104E20006172642074797065206368616E6765647F
:104E30002E00E1005761726E696E673A20707269E8
:104E40006E7465722074797065206368616E676541
:104E5000642E00E2005761726E696E673A206D6FD2
:104E600074686572626F6172642074797065206322
:104E700068616E6765642E00E300536865657400C1
:104E8000E400556E657870656374656420657272C0
:104E90006F72206F636375727265642E00E5004D5A
:104EA0003630302046696C616D656E7420436861F0
:104EB0006E67652E204C6F61642061206E657720DF
:104EC00066696C616D656E74206F7220656A6563DA
:104ED0007420746865206F6C64206F6E652E00E628
:104EE0000052656D6F76652074686520656A65633C
:104EF0007465642066696C616D656E742066726F9E
:104F00006D207468652066726F6E74206F66207401
:104F10006865204D4D552E00E70046696C616D6552
:104F20006E7420646574656374656420756E65785D
:104F30007065637465646C792E20456E7375726557
:104F4000206E6F2066696C616D656E7420697320D8
:104F50006C6F616465642E20436865636B207468C0
:104F6000652073656E736F727320616E642077695C
:104F700072696E672E00E800496E7465726E616C2E
:104F80002072756E74696D65206572726F722E2065
:104F900054727920726573657474696E67207468E1
:104FA00065204D4D55206F72207570646174696E77
:104FB0006720746865206669726D776172652E007E
:104FC000E9004D4D552046572076657273696F6E26
:104FD00020697320696E636F6D70617469626C65BE
:104FE0002077697468207072696E74657220465704
:104FF0002E55706461746520746F207665727369D4
:105000006F6E20332E302E332E00EA004D4D55208A
:105010004669726D7761726520696E7465726E6142
:105020006C206572726F722C20706C6561736520E4
:10503000726573657420746865204D4D552E00EBC4
:10504000005265717565737465642066696C616D85
:10505000656E7420746F6F6C206973206E6F74209E
:10506000617661696C61626C65206F6E207468693D
:10507000732068617264776172652E20436865638E
:105080006B2074686520472D636F646520666F72BE
:1050900020746F6F6C20696E646578206F75742062
:1050A0006F662072616E6765202854302D54342954
:1050B0002E00EC0043616E6E6F7420706572666F37
:1050C000726D2074686520616374696F6E2C206650
:1050D000696C616D656E7420697320616C726561C5
:1050E0006479206C6F616465642E20556E6C6F610D
:1050F000642069742066697273742E00ED004D4D52
:1051000055206E6F7420726573706F6E64696E6780
:1051100020636F72726563746C792E2043686563D7
:105120006B2074686520776972696E6720616E64B0
:1051300020636F6E6E6563746F72732E00EE004DA8
:105140004D55206E6F7420726573706F6E64696E5A
:10515000672E20436865636B2074686520776972E9
:10516000696E6720616E6420636F6E6E6563746F35
:1051700072732E00EF004D6F726520646574616973
:105180006C73206F6E6C696E652E00F0005468655C
:105190002049646C65722063616E6E6F7420686F65
:1051A0006D652070726F7065726C792E2043686532
:1051B000636B20666F7220616E797468696E672018
:1051C000626C6F636B696E6720697473206D6F76B4
:1051D000656D656E742E00F10043616E2774206D5D
:1051E0006F76652053656C6563746F72206F7220F3
:1051F00049646C65722E00F2005468652053656C3A
:105200006563746F722063616E6E6F7420686F6D7A
:10521000652070726F7065726C792E2043686563CB
:105220006B20666F7220616E797468696E672062A8
:105230006C6F636B696E6720697473206D6F766540
:105240006D656E742E00F3004C6F6164696E6720AB
:10525000746F206578747275646572206661696C1C
:1052600065642E20496E73706563742074686520D0
:1052700066696C616D656E74207469702073686115
:1052800070652E20526566696E65207468652073AE
:10529000656E736F722063616C6962726174696FAD
:1052A0006E2C206966206E65656465642E00F400CE
:1052B00053656C6563746F722063616E2774206D33
:1052C0006F76652064756520746F2046494E4441B1
:1052D00020646574656374696E6720612066696C1B
:1052E000616D656E742E204D616B652073757265FE
:1052F000206E6F2066696C616D656E742069732025
:10530000696E2053656C6563746F7220616E6420F2
:1053100046494E444120776F726B732070726F70F4
:1053200065726C792E00F50046696C616D656E746E
:105330002073656E736F722074726967676572653A
:105340006420746F6F206561726C79207768696C76
:1053500065206C6F6164696E6720746F2065787476
:1053600072756465722E20436865636B207468658E
:1053700072652069736E277420616E797468696E36
:105380006720737475636B20696E20505446452006
:10539000747562652E20436865636B207468617460
:1053A0002073656E736F7220726561647320707212
:1053B0006F7065726C792E00F60050756C6C6579B3
:1053C000206D6F746F72207374616C6C65642E2035
:1053D000456E73757265207468652070756C6C65B8
:1053E000792063616E206D6F766520616E64206345
:1053F0006865636B2074686520776972696E672ED3
:1054000000F70046696C616D656E742073656E739C
:105410006F72206469646E2774207377697463689F
:10542000206F6666207768696C6520756E6C6F61A9
:1054300064696E672066696C616D656E742E2045C7
:105440006E737572652066696C616D656E7420633C
:10545000616E206D6F766520616E642074686520D2
:1054600073656E736F7220776F726B732E00F80026
:1054700046696C616D656E742073656E736F722022
:105480006469646E27742074726967676572207737
:1054900068696C65206C6F6164696E67207468650B
:1054A0002066696C616D656E742E20456E73757231
:1054B00065207468652073656E736F722069732050
:1054C00063616C6962726174656420616E642074EA
:1054D00068652066696C616D656E742072656163D4
:1054E0006865642069742E00F90046494E444120E5
:1054F0006469646E277420737769746368206F66CB
:1055000066207768696C6520756E6C6F6164696E82
:10551000672066696C616D656E742E205472792007
:10552000756E6C6F6164696E67206D616E75616C1C
:105530006C792E20456E737572652066696C616D9D
:10554000656E742063616E206D6F766520616E6498
:105550002046494E444120776F726B732E00FA004B
:1055600046494E4441206469646E27742074726910
:1055700067676572207768696C65206C6F61646924
:105580006E67207468652066696C616D656E742E47
:1055900020456E73757265207468652066696C615C
:1055A0006D656E742063616E206D6F766520616E2F
:1055B000642046494E444120776F726B732E00FB86
:1055C0000044697361626C6500FC0053746F700085
:1055D000FD004C6F616400FE00556E6C6F616400ED
:1055E000FF0052657365744D4D550000015265749E
:1055F000727900010153656E736974697669747913
:10560000000201446F6E65000301526573756D6998
:105610006E67207072696E7400040150494E4441F7
:105620002048656174696E6700050143616C6962B9
:10563000726174696F6E20646F6E6500060143616C
:105640006C6962726174696E67205A000701426575
:105650006420646F6E6500080142656420486561DE
:1056600074696E6700090148656174696E6720643A
:105670006F6E652E000A0148656174696E67000BE4
:1056800001546F74616C000C014C61737420707272
:10569000696E74000D014D4D55206661696C730093
:1056A0000E014D4D55206C6F6164206661696C730D
:1056B000000F014D4D5520706F776572206661694E
:1056C0006C730010014D6174657269616C206368D0
:1056D000616E6765730011014C61737420707269AB
:1056E0006E74206661696C75726573001201546F87
:1056F00074616C206661696C757265730013014694
:10570000696C2E2072756E6F757473001401546588
:105710006D70657261747572657300150153656E05
:10572000736F7220696E666F00160145787472752A
:1057300064657220696E666F00170158595A2063BC
:10574000616C2E2064657461696C7300180150727D
:10575000696E74657220495020416464723A001980
:1057600001756E6B6E6F776E001A014D4D5520639B
:105770006F6E6E6563746564001B01446174653A05
:10578000001C01746F20756E6C6F61642066696C1B
:10579000616D656E74001D01746F206C6F61642013
:1057A00066696C616D656E74001E0150726573737D
:1057B00020746865206B6E6F62001F01507265680F
:1057C000656174696E6720746F20637574002001D1
:1057D00050726568656174696E6720746F20656AD0
:1057E00065637400210150726568656174696E6754
:1057F00020746F20756E6C6F6164002201507265B9
:1058000068656174696E6720746F206C6F616400F5
:105810002301436F6F6C646F776E00240146696CDF
:10582000616D656E7420657874727564696E672049
:1058300026207769746820636F72726563742063D1
:105840006F6C6F723F002501456A65637400260125
:105850004175746F6C6F6164696E672066696C6115
:105860006D656E74206973206163746976652C20A0
:105870006A75737420707265737320746865206B29
:105880006E6F6220616E6420696E7365727420664B
:10589000696C616D656E742E2E2E002701546F7435
:1058A000616C2066696C616D656E74002801546FCF
:1058B00074616C207072696E742074696D65002962
:1058C0000146696C616D656E742075736564002AAC
:1058D000015072696E742074696D65002B01466514
:1058E0006564696E6720746F204653656E736F72CE
:1058F000002C014D6F76696E672073656C6563746B
:105900006F72002D01486F6D696E67002E01526540
:1059100074726163742066726F6D2046494E444113
:10592000002F01456A656374696E672066696C6162
:105930006D656E740030015061726B696E67207323
:10594000656C6563746F7200310152657475726EB7
:10595000696E672073656C6563746F720032015005
:105960006572666F726D696E6720637574003301CE
:1059700050757368696E672066696C616D656E74D9
:10598000003401507265706172696E6720626C61EB
:10599000646500350153656C656374696E672066E4
:1059A000696C2E20736C6F74003601556E6C6F61DC
:1059B00064696E672066696C616D656E740037019D
:1059C00045525220544D43206661696C656400382D
:1059D000014552522048656C702066696C616D65A6
:1059E0006E7400390145525220496E7465726E61C1
:1059F0006C003A01455252205761697420666F72FB
:105A00002055736572003B0146696E697368696E63
:105A100067206D6F76656D656E7473003C0141762D
:105A20006F6964696E67206772696E64003D014644
:105A3000656564696E6720746F206E6F7A7A6C6535
:105A4000003E0146656564696E6720746F20657865
:105A5000747275646572003F0146656564696E67BE
:105A600020746F2046494E4441004001556E6C6FD2
:105A70006164696E6720746F2070756C6C65790065
:105A80004101556E6C6F6164696E6720746F2046CA
:105A9000494E4441004201446973656E676167691C
:105AA0006E672069646C6572004301456E676167CB
:105AB000696E672069646C65720044014F4B004554
:105AC00001554E4B4E4F574E204552524F520046B5
:105AD0000146494C414D454E54204348414E4745AF
:105AE00000470146494C414D454E5420454A4543E7
:105AF000544544004801554E4C4F4144204D414EC1
:105B000055414C4C5900490146572052554E544975
:105B10004D45204552524F52004A014D4D552046A9
:105B20005720555044415445204E45454445440076
:105B30004B0151554555452046554C4C004C0149AB
:105B40004E56414C494420544F4F4C004D0146495C
:105B50004C2E20414C5245414459204C4F41444524
:105B600044004E01434F4D4D554E49434154494F1A
:105B70004E204552524F52004F014D4D55204E4F31
:105B80005420524553504F4E44494E470050014D0A
:105B90004D55204D4355204552524F520051014D15
:105BA0004D552053454C4654455354204641494C8D
:105BB0004544005201544D43204452495645522019
:105BC00053484F52544544005301544D4320554EC1
:105BD000444552564F4C544147452045525200547B
:105BE00001544D4320445249564552205245534595
:105BF00054005501544D43204452495645522045C6
:105C000052524F52005601544D43204F5645524870
:105C1000454154204552524F520057015741524E70
:105C2000494E4720544D4320544F4F20484F540075
:105C3000580149444C45522043414E4E4F54204D4B
:105C40004F564500590149444C45522043414E4E60
:105C50004F5420484F4D45005A0153454C4543543D
:105C60004F522043414E4E4F54204D4F5645005BFE
:105C70000153454C4543544F522043414E4E4F54DF
:105C800020484F4D45005C014C4F414420544F206B
:105C9000455854522E204641494C4544005D014927
:105CA0004E53504543542046494E4441005E014600
:105CB00053454E534F5220544F4F204541524C595B
:105CC000005F0150554C4C45592043414E4E4F54B6
:105CD000204D4F56450060014653454E534F5220CC
:105CE00046494C2E20535455434B006101465345C1
:105CF0004E534F52204449444E5420545249474732
:105D00002E00620146494E44412046494C414D2EE9
:105D100020535455434B00630146494E44412044AF
:105D200049444E5420545249474745520064014E5D
:105D30006F74207370696E6E696E670065015370D1
:105D4000696E6E696E670066014C65667420686FE7
:105D500074656E642066616E3F00670146726F6E07
:105D600074207072696E742066616E3F006801462F
:105D7000616E207465737400690158595A2063611B
:105D80006C6962726174696F6E20616C6C207269FB
:105D90006768742E20536B65772077696C6C20627E
:105DA0006520636F72726563746564206175746FDA
:105DB0006D61746963616C6C792E006A0158595A7F
:105DC0002063616C6962726174696F6E20616C6CD2
:105DD0002072696768742E20582F59206178657386
:105DE0002061726520736C696768746C7920736BCD
:105DF000657765642E20476F6F64206A6F622100AB
:105E00006B0158595A2063616C6962726174696FE1
:105E10006E206F6B2E20582F59206178657320619A
:105E200072652070657270656E646963756C61720D
:105E30002E20436F6E67726174756C6174696F6E4A
:105E40007321006C0158595A2063616C6962726158
:105E500074696F6E20636F6D70726F6D69736564C6
:105E60002E2052696768742066726F6E74206361B9
:105E70006C6962726174696F6E20706F696E7420F4
:105E80006E6F7420726561636861626C652E006D6F
:105E90000158595A2063616C6962726174696F6E4E
:105EA00020636F6D70726F6D697365642E2046722A
:105EB0006F6E742063616C6962726174696F6E20C9
:105EC000706F696E7473206E6F74207265616368A1
:105ED00061626C652E006E0158595A2063616C69CD
:105EE00062726174696F6E206661696C65642E20F0
:105EF00052696768742066726F6E742063616C69A2
:105F000062726174696F6E20706F696E74206E6F5B
:105F10007420726561636861626C652E006F015860
:105F2000595A2063616C6962726174696F6E206690
:105F300061696C65642E2046726F6E742063616CBB
:105F40006962726174696F6E20706F696E7473201C
:105F50006E6F7420726561636861626C652E00709B
:105F60000158595A2063616C6962726174696F6E7D
:105F7000206661696C65642E20506C6561736520D4
:105F8000636F6E73756C7420746865206D616E75D7
:105F9000616C2E00710158595A2063616C696272FC
:105FA0006174696F6E206661696C65642E2042655C
:105FB000642063616C6962726174696F6E20706FD6
:105FC000696E7420776173206E6F7420666F756ED2
:105FD000642E007201506C6561736520706C6163A2
:105FE0006520737465656C207368656574206F6ED9
:105FF00020686561746265642E007301446973747E
:10600000616E6365206265747765656E2074697082
:10601000206F6620746865206E6F7A7A6C652061E7
:106020006E642074686520626564207375726661B1
:10603000636520686173206E6F74206265656E20F1
:10604000736574207965742E20506C6561736520CA
:10605000666F6C6C6F7720746865206D616E75611A
:106060006C2C206368617074657220466972737469
:106070002073746570732C2073656374696F6E2070
:106080004669727374206C617965722063616C6912
:1060900062726174696F6E2E007401506C61636589
:1060A0002061207368656574206F6620706170657B
:1060B0007220756E64657220746865206E6F7A7ADE
:1060C0006C6520647572696E672074686520636111
:1060D0006C6962726174696F6E206F6620666972A6
:1060E0007374203420706F696E74732E204966209B
:1060F000746865206E6F7A7A6C652063617463687A
:106100006573207468652070617065722C20706FF3
:10611000776572206F666620746865207072696E9C
:1061200074657220696D6D6564696174656C792E42
:10613000007501536561726368696E67206265640A
:106140002063616C6962726174696F6E20706F693F
:106150006E740076014D6561737572696E672072A9
:1061600065666572656E6365206865696768742039
:106170006F662063616C6962726174696F6E207012
:106180006F696E74007701506C6561736520636C94
:1061900065616E20746865206E6F7A7A6C65206622
:1061A0006F722063616C6962726174696F6E2E2018
:1061B000436C69636B207768656E20646F6E652E33
:1061C0000078014175746F20686F6D650079014337
:1061D00075742066696C616D656E74007A01456A3C
:1061E0006563742066726F6D204D4D55007B014CC8
:1061F0006F6164696E672066696C616D656E7400BD
:106200007C014D4D552052657472793A2052657368
:10621000746F72696E672074656D706572617475F4
:1062200072652E2E2E007D01536F7274696E672089
:1062300066696C6573007E01536F6D652066696CDD
:1062400065732077696C6C206E6F742062652073B3
:106250006F727465642E204D61782E204E6F2E2053
:106260006F662066696C657320696E203120666FE9
:106270006C64657220666F7220736F7274696E67EA
:10628000206973203130302E007F0153544F50501D
:1062900045442E0080014F66660081014F6E006507
:1062A0006E717565696E67202200446F6E6520709F
:1062B00072696E74696E672066696C65004E6F2046
:1062C0004C696E65204E756D6265722077697468E1
:1062D00020636865636B73756D2C204C617374204B
:1062E0004C696E653A20004E6F20436865636B739E
:1062F000756D2077697468206C696E65206E756DA8
:106300006265722C204C617374204C696E653A2072
:1063100000636865636B73756D206D69736D61747F
:1063200063682C204C617374204C696E653A2000C0
:106330004C696E65204E756D626572206973206EC2
:106340006F74204C617374204C696E65204E756DBE
:106350006265722B312C204C617374204C696E6520
:106360003A2000257520627974657320777269740C
:1063700074656E20746F20255320617420616464FD
:1063800072657373203078253038780A00442564AC
:10639000202D20526561642F577269746520255342
:1063A0000A003F3F00526F6D616E61004872766176
:1063B00074736B69004D616779617200536C6F761D
:1063C000656E63696E61004E6F72736B0053766524
:1063D0006E736B61004E656465726C616E64730010
:1063E000506F6C736B69004974616C69616E6F000A
:1063F0004672616E6361697300457370616E6F6CA4
:1064000000446575747363680043657374696E61F5
:1064100000456E676C6973680020436F756E742069
:10642000583A200045303A25642052504D205052B1
:106430004E313A25642052504D204530403A257562
:106440002050524E31403A25750A00526573656EF0
:10645000640025533A20256C640A25530A002F2F27
:10646000616374696F6E3A6E6F74696669636174B3
:10647000696F6E2025530A0046696C616D656E7404
:106480002072756E6F7574206465746563746564DD
:10649000210064697361626C656400656E61626CA1
:1064A000656400454550524F4D005352414D0044E4
:1064B0002D31202D20456E646C657373206C6F6FD9
:1064C000700A00416374697665204578747275645A
:1064D00065723A203000496E76616C696420657897
:1064E000747275646572004D323230205325640039
:1064F0005344207072696E74696E672062797465A6
:106500002000257500556E6B6E6F776E20636F6D82
:106510006D616E643A2022004D32303020496E7633
:10652000616C696420657874727564657220007AA4
:106530005F6D61783A20007A5F6D696E3A2000796C
:106540005F6D696E3A2000545249474745524544B1
:10655000006F70656E00785F6D696E3A200052655D
:10656000706F7274696E6720656E6473746F7020EB
:10657000737461747573004D3131322063616C6CDA
:1065800065642E20456D657267656E63792053746E
:106590006F702E002F2F616374696F6E3A75766C81
:1065A0006F5F7265636F766572795F72656164793A
:1065B0000025533A256C7520636D0A25533A256CE6
:1065C00075206D696E0A0053494C454E54004E4F7C
:1065D000524D414C002553204D4F44453A205065C3
:1065E0007263656E7420646F6E653A202568686416
:1065F0003B207072696E742074696D652072656DE0
:1066000061696E696E6720696E206D696E733A20EC
:1066100025643B204368616E676520696E206D6963
:106620006E733A2025640A005072696E7465725365
:10663000746174653A2025640A00456E64206669B9
:106640006C65206C69737400426567696E206669C9
:106650006C65206C69737400556E6B6E6F776E207D
:10666000256320636F64653A2025730A000A504948
:106670004E44412074656D70657261747572653A3F
:1066800020252E3166205A20736869667420286D93
:106690006D293A20252E3366000A537465703A201E
:1066A00025642F360A000A537465703A2025642F3A
:1066B000362028736B6970706564290A50494E440E
:1066C000412074656D70657261747572653A20253C
:1066D00064205A20736869667420286D6D293A30E9
:1066E0000A000A5A45524F3A20252E33660A007393
:1066F000746172742074656D706572617475726511
:106700003A20252E31660A0025642020252E326687
:1067100000255320583A20252E356620593A202549
:106720002E3566205A3A20252E35660A00536C65B0
:1067300065702E2E2E0045303A25642052504D0AA9
:1067400050524E303A25642052504D0A00312F39B4
:1067500000473930004D3130370025362E32666D16
:106760006D0025530A25530A25533A0A25533A004A
:1067700025332E32668100252D31342E3134533AA3
:106780000A25530A252D31342E3134533A25332E20
:106790003266810A252D31342E3134533A25332E79
:1067A000326681002020300020203100423A20252E
:1067B0003364202020202058643A2536640A533A56
:1067C00020253364202020202059643A2536640097
:1067D00046494E44410050494E44410057697A6150
:1067E000726420656E642073746174653A20256458
:1067F0000A0053706F6F6C4A6F696E004669726D64
:106800007761726500537570657250494E4441005E
:1068100048426564206F6E206C6F616400466C6155
:106820007368416972004572723A484F54454E444C
:106830002046414E204552524F52002F2F61637423
:10684000696F6E3A726573756D6564002F2F6163B1
:1068500074696F6E3A726573756D65002F2F616391
:1068600074696F6E3A7265616479002F2F61637489
:10687000696F6E3A6E6F745F7265616479002F2F75
:10688000616374696F6E3A63616E63656C004D3865
:1068900034004F4B004C4344207374617475732073
:1068A0006368616E676564005344206361726420AD
:1068B00072656C6561736564002F2F616374696F25
:1068C0006E3A737461727400473931004D3730325B
:1068D000004732382057004D353030004261642087
:1068E000696E746572727570740057617463686460
:1068F0006F672074696D656F757400537461746996
:1069000063206D656D6F7279206861730A626565D9
:106910006E206F7665727772697474656E00464991
:10692000524D57415245204352415348210A437228
:1069300061736820726561736F6E3A0A002020509F
:106940006C616E6E657242756666657242797465D9
:10695000733A20002046726565204D656D6F72792F
:106960003A2000207C20417574686F723A20002024
:106970004C61737420557064617465643A20002022
:10698000536F667477617265205265736574002079
:106990005761746368646F67205265736574002083
:1069A00042726F776E206F75742052657365740044
:1069B0002045787465726E616C2052657365740051
:1069C000506F7765725570006572726F72207772C2
:1069D0006974696E6720746F2066696C6500446F26
:1069E0006E6520736176696E672066696C652E003E
:1069F0006F6B0046696C616D656E74008800207471
:106A00006F6F206C6F6E6720657874727573696F35
:106A10006E2070726576656E7465640020636F6CBD
:106A20006420657874727573696F6E207072657614
:106A3000656E746564004D6F76652061626F727477
:106A40006564004572723A5052494E542046414E98
:106A5000204552524F520025632533642F2564810F
:106A6000005A25362E32662563005A2020202D2D0F
:106A70002D2000862533642525002D2D2D2525006C
:106A80002533642525002053440020202000204881
:106A90004F002046524D2000872D2D3A2D2D2020CD
:106AA00000872533756820256325630087253032EC
:106AB000753A2530327525632563002F2F61637485
:106AC000696F6E3A706175736564002F2F6163742E
:106AD000696F6E3A70617573650044756D702074EE
:106AE0006F2073657269616C0068656C702E7072DE
:106AF00075736133642E636F6D00666F72756D2EF2
:106B0000707275736133642E636F6D00707275738C
:106B10006133642E636F6D004D3730310025533A79
:106B20000A2531382E32666D200A25533A0A25315E
:106B3000306C646420253032646820253032646D06
:106B40000025533A0A2531382E32666D200A255326
:106B50003A0A2531306C646820253032646D202576
:106B600030326473004D6561737572656420736BB8
:106B70006577733A2025662025660A004669747495
:106B8000696E67206661696C6564203D3E206361C3
:106B90006C6962726174696F6E206661696C6564AC
:106BA0002E0A0043616C6962726174696F6E2073B2
:106BB0007563636573732E0A00416C6C2034206327
:106BC000616C6962726174696F6E20706F696E7456
:106BD0007320666F756E642E0A00312F3400312FDA
:106BE0003400312F39005072757361206933204DA4
:106BF0004B322E35204F4B2E00534420636172647C
:106C0000206F6B006F70656E526F6F7420666169E4
:106C10006C656400766F6C756D652E696E697420A5
:106C20006661696C656400534420696E697420660E
:106C300061696C006F70656E206661696C65642CBB
:106C40002046696C653A200043616E6E6F74206562
:106C50006E746572207375626469723A20004D36F5
:106C60003030004D3234004D3233202573005072E5
:106C7000696E7465722073746F70706564206475DA
:106C80006520746F206572726F72732E2053757059
:106C90006572766973696F6E207265717569726568
:106CA000642E0047312045252D2E3366204632378D
:106CB0003030004D383300084AD73B3BCE016E845C
:106CC000BCBFFDC12F3D6C74319ABD56833DDA3D8A
:106CD00000C77F11BED9E4BB4C3E916BAAAABE008F
:106CE0000000803F05A84CCDB2D44EB93836A90279
:106CF0000C50B9918688083CA6AAAA2ABE000000BA
:106D0000803F07634236B79BD8A71A39685618AE3A
:106D1000BAAB558C1D3CB7CC5763BD6DEDFD753ED0
:106D2000F6177231BF000000803F08000000BE92DD
:106D30002449123EABAAAA2ABECDCCCC4C3E0000C0
:106D40000080BEABAAAAAA3E00000000BF0000005F
:106D5000803F0000000000084178D3BB4387D11377
:106D60003D190E3CC3BD4282AD2B3E68EC8276BE1F
:106D7000D98FE1A93E4C80EFFFBE01C4FF7F3F00E9
:106D8000000000000D941A050C94CFCF0C9499D8F4
:106D90000C946CFE0C94A6D30C949DC30C94D1D38C
:106DA0000C944B770C9450EC0D94DB040C9456D956
:106DB0000C9437C80C9441BF0C94EBFE0C945FBF4D
:106DC0000C941FBD0D9446050C9494BF0D94EE0CCD
:106DD0000C9418D40C945FD00D94B9260C9432C046
:106DE0000C946AFA0D949B0F0C94DAEC0D944B07FB
:106DF0000C9433BD0C9489BF0C941C770C9457BD34
:106E00000C944CEB0C94EBD30C94E1CF0D94AB961B
:106E10000C9454770C9425DB0C944ABD0C9425C239
:106E20000C94EBEC0C946FD00C94FCF90C9440D4C3
:106E30000C9499C30D946E270C9442DF0C947BD074
:106E40000D9477330D94059D0C9459C80C9495D0EE
:106E50000C9469F70C9403ED0C9427770C94B3D33E
:106E60000D949F170D94E40F0C9425BD0C9420BF36
:106E70000D948C040C94EED00C9419DB0C9462C825
:106E80000C940ED40D9476270C9480C30D94880F27
:106E90000D94219D0C942CD40C9433D10C94C3BE2E
:106EA0000C942EDB0C948AC30C9492CF0C946B73CD
:106EB0000D949E270C9407C20D94B2260D94F526CE
:106EC0000C9473C40D9472260C9494C30C947AC4DD
:106ED0000D94A6270C94F5EC0D94AE270C94D9D301
:106EE0000C945CBD0C94C8CE0D94D90B0D94960CEB
:106EF0000C94F5D30C940ABD0D9424270C9450C81F
:106F00000C942FBD0C94D5CF0C944BBD0D942697AB
:106F10000C9437BF0D9486270C94D8CF0C9455BF92
:106F20000C94D4C70D942A970C94DBC30C9488C49A
:106F30000C9428DB0C9420ED0C9410F90C9403EACB
:106F40000C9486EC0C9489770D94EF030D94260530
:106F50000C9487C00C9468D70C94FFD30C94C1FB9D
:106F60000C947BC30C947CE30C9405BF0D94239785
:106F70000C94C0EC0C9470EC0C948FC40D947E2790
:106F80000C94E1D30C943DBD0D94289D0C9497D0A6
:106F90000C9429BD0C9481C40D9496270D9443053F
:106FA0000D94BC260D9444100C94E5CC0C943577CC
:106FB0000C94D2CF0C94D3DA0C949AD00C94A5DE16
:106FC0000C942CBF0D94D5070C9475BF0D945E27BF
:106FD0000D9435040D948A260C945DCF0D94AF2644
:106FE0000C9445BD0C94AED30D94B2070C94BF7AAB
:106FF0000C94C7D30C94FAC80D94C4960C9476C321
:107000000D945B270C94AFDA0C94A3F80C9418BD84
:107010000D9427270D9475040C943ADB0C9464C0EE
:107020000C9446DB0C945BC10C94CEBE0C94777729
:107030000C9441BD0D94319D0C9462C20D94369D0B
:107040000D9406970C9467CF0C9416E90C94CCCF52
:107050000C940CC60C94C9CF0D94380B0C94B9DE6B
:107060000D9455270D9458270C947CEC0C946ECB02
:107070000C943BFF0C9480E90C947FBF0C948FC35D
:107080000C946DDF0C94AA780C940CED0C9486D0C3
:107090000C94D6FE0C9441CE0C94A0E50C941CBD2F
:1070A0000C9463F70C944ECB0D9421270C9411BFD4
:1070B0000C9414F90D9417100C9449C40C9485C3C6
:1070C0000C94A5F90C9457D00C944BBF0C9422D47B
:1070D0000C9496E90C9453FF0C94BBDA0C9427CCD7
:1070E0000C946BBF0D94BF9C0C942BDB0C9437BDA0
:1070F0000C9402770C9492C60C9466FA0C9410BD12
:107100000D94B6270C944FBD0C94BDD30D942964F7
:107110000C94BDBE0C944EC00C9453BD0D9428101D
:107120000C948BDE0C9436D40C94C8FA0C94BEBF2D
:107130000D941A110C9467D00C946BC80D946627AB
:107140000C94E9D00D94249D0C9407D70D948E27B0
:107150000D9437050C9482730D94FC0D0C94F1EC96
:107160000C94CF630D94D1070D94F7060C9414BDC5
:107170000C94ABBF0C946BC06E616E00696E6600C0
:1071800000407A10F35A00A0724E18090010A5D4DE
:10719000E80000E87648170000E40B54020000CA3B
:1071A0009A3B000000E1F505000080969800000081
:1071B00040420F000000A0860100000010270000E0
:1071C0000000E803000000006400000000000A0066
:1071D000000000000100000000002C76D888DC6769
:1071E0004F0823DFC1DFAE59E1B1B796E5E3E453C1
:1071F000C63AE651997696E8E6C28426EB898C9BDE
:1072000062ED407C6FFCEFBC9C9F40F2BAA56FA57D
:10721000F490055A2AF75C936B6CF9676DC11BFCFF
:10722000E0E40D47FEF520E6B500D0ED902E03001A
:10723000943577050080841E080000204E0A000067
:1072400000C80C333333330F986E12831141EF8D26
:107250002114893BE65516CFFEE6DB18D1844B3866
:107260001BF77C1D901DA4BBE424203284725E2297
:107270008100C9F124ECA1E53D27220000204553FF
:107280005000204E535000204F464600204F4E00E5
:107290005056303100205B4D505D2000256920683C
:1072A0006F757273202569206D696E757465730042
:1072B00052582074696D656F7574004D333130001C
:1072C0004D313132004D3131300046756C6C2052F9
:1072D00058204275666665720053657474696E67FE
:1072E000732053746F7265640053746F7265642009
:1072F00073657474696E67732072657472696576FC
:1073000065640048617264636F6465642044656607
:1073100061756C742053657474696E6773204C6F6B
:107320006164656400563200000000C8420000C875
:10733000420000C8430000054300004843000048E5
:1073400043000040410000F042E8030000E8030071
:1073500000C80000008813000000409C4400409CCE
:10736000440000000000000000204E00000000204B
:107370004100002041CDCCCC3E00009040000000F8
:10738000000000000000000000CDCCCC3E3D0A8192
:1073900041FF08433EB099AB438F42FC42E65A346A
:1073A0003F4C62B045000000000040400000344205
:1073B000000000000000000000000041000000E0AC
:1073C0003F00002C4300002C43000040410000F02F
:1073D00042C0030000C0030000C800000088130082
:1073E000001010101000409C440000803F0000007E
:1073F0003F191400000020307800203078006572BA
:10740000726F723A2000443233202D20656D657210
:1074100067656E63792073657269616C2064756D50
:107420007000437573746F6D004E796C6F6E5041D0
:1074300000536174696E2020005465787475720081
:10744000536D6F6F746800312E3000312E3500554A
:107450004E4B4E4F574E004C413130433A204C6911
:107460006E65617220416476616E6365206D6F6444
:10747000653A20004C413130433A2041646A7573CB
:1074800074656420452D4A65726B3A2000D5E91574
:10749000683E0FA8AF00480069960000DF602555E0
:1074A0005887680427F2E0005E3403CC1960F33C8F
:1074B0000EF88F00DB08029492003E1C079A8700AA
:1074C000E524008528527E06001BE4007E781270B9
:1074D000787061F812788F8841784270787061789E
:1074E0002570787061F850788F88D1F0252707874C
:1074F00061F025278F88412C0D27AA50D1BC0707A2
:10750000871161BE788F881141785270787061F868
:1075100052788F8841201278887063205278887062
:10752000634852788887430311179970641812785A
:10753000F870654412F8F8F045184278F87065184C
:107540002578F87065185278F87065185078F870DA
:10755000650C078F872365A20F8F8F1145001206D8
:10756000227069001207222749002506227069004F
:10757000250722274900120622276C026236A270D4
:107580006C40456C44704C03622222706C438888C6
:1075900088F04C7812BC88806E7852BC88806E3837
:1075A000127888706F78127888874F3842788870A0
:1075B0006F38257888706F3A0079AC786F3D079AFC
:1075C000AC786F7850788887EF39497888706F0881
:1075D00052BC8880729852F88F985220127870F0BE
:1075E0007348127863875320527870F0734852784A
:1075F0006387531007870F247312786387245360BF
:10760000699A988BE22304E4443074104E44432476
:10761000747C12888960753C50888870557825285C
:107620008960757949088960753C12887070790C99
:1076300012885222594412F124F07A4452F124F073
:107640007A8C52F0368F5A4420F124F07A0040149C
:1076500054CDCCCC3D0AD7233C17B7D13877CC2BAF
:10766000329595E6241FB14F0A000020410000C862
:107670004200401C4620BCBE4CCA1B0E5AAEC59DE3
:10768000744E414E494E4600007A4300005243007A
:1076900000524300000000000080C09A99193E008B
:1076A000000000000080C09A99193E20503A002046
:1076B00042403A0020403A00202F002054303A0047
:1076C000202F0020423A00202F00543A0025534535
:1076D000786365737369766520626564206C65768E
:1076E000656C696E6720636F7272656374696F6E33
:1076F0003A202569206D6963726F6E730A004265D6
:1077000064206C6576656C696E67206661696C657E
:10771000642E20546F6F206D7563682076617269E6
:107720006174696F6E2066726F6D20656570726F2F
:107730006D206D65736800426564206C6576656CCC
:10774000696E67206661696C65642E2053656E738F
:107750006F722074726967676572656420746F6FF9
:1077600020736F6F6E002020004D65617375726528
:107770006420706F696E74733A005A207365617289
:107780006368206865696768743A20352E30660042
:107790004E756D20582C593A20372C37004D6573A3
:1077A0006820626564206C6576656C696E67206E22
:1077B0006F74206163746976652E0020453A00205D
:1077C0005A3A0020593A0020453A00205A3A0020FF
:1077D000593A00583A00202D3E200053706F6F6CCC
:1077E0004A6F696E3A20002C2000496E616374690B
:1077F000766974792053687574646F776E004B49AD
:107800004C4C45442E005072696E7465722068615C
:107810006C7465642E206B696C6C28292063616C24
:107820006C656421005A206C6976652061646A7514
:107830007374206F7574206F662072616E67652E99
:107840002053657474696E6720746F20302E204356
:107850006C69636B20746F20636F6E74696E7565FD
:107860002E005A206C6976652061646A75737420F5
:107870006F7574206F662072616E67652E20536588
:107880007474696E6720746F20300020453A302090
:10789000423A00543A00627573793A207061757308
:1078A000656420666F7220696E707574006275730E
:1078B000793A2070617573656420666F7220757304
:1078C000657200627573793A2070726F63657373C5
:1078D000696E670073657269616C2064756D7020F4
:1078E00000496E76616C6964205420636F64652E74
:1078F000004475706C696361746520542D636F6416
:10790000652069676E6F7265642E00416476616EF2
:107910006365204B3D004B206F7574206F662061BE
:107920006C6C6F7765642072616E676521004D4BEA
:10793000322E35004D4B322E354D4D5532001A4FFB
:10794000FA002533642F2533640025336400200AB0
:10795000200A200A200025535374617469737469E6
:1079600063733A0A255320204D37382053256C7510
:107970002054256C750A00255341726320536574A9
:1079800074696E67733A20503A4D6178206C656E69
:10799000677468286D6D2920533A4D696E206C65B7
:1079A0006E67746820286D6D29204E3A436F72729D
:1079B000656374696F6E7320523A4D696E2073650A
:1079C000676D656E747320463A5365676D656E74B6
:1079D000732F7365632E0A255320204D32313420D6
:1079E00050252E32662053252E3266204E256420E7
:1079F000522564204625640A00255346696C616D52
:107A0000656E742073657474696E67733A20446997
:107A10007361626C65640A00255346696C616D652B
:107A20006E742073657474696E67733A0A25532007
:107A300020204D3230302044252E32660A00255356
:107A4000526574726163743A20533D4C656E67747D
:107A50006820286D6D2920463A537065656420289A
:107A60006D6D2F6D29205A3A205A4C696674202872
:107A70006D6D290A25532020204D323037205325A3
:107A80002E32662046252E3266205A252E32660A70
:107A900025535265636F7665723A20533D4578747D
:107AA0007261206C656E67746820286D6D292046B0
:107AB0003A537065656420286D6D2F6D290A255332
:107AC0002020204D3230382053252E326620462586
:107AD0002E32660A25534175746F2D52657472619A
:107AE00063743A20533D3020746F2064697361627F
:107AF0006C652C203120746F20696E746572707211
:107B0000657420657874727564652D6F6E6C79206C
:107B10006D6F766573206173207265747261637432
:107B200073206F72207265636F7665726965730A80
:107B300025532020204D323039205325640A00255A
:107B400053504944206865617462656420736574AC
:107B500074696E67733A0A25532020204D33303400
:107B60002050252E32662049252E32662044252EAF
:107B700032660A0025535049442073657474696E57
:107B800067733A0A25532020204D33303120502589
:107B90002E32662049252E32662044252E32660A72
:107BA00000255353746570732070657220756E697B
:107BB000743A0A255320204D39322058252E32663A
:107BC0002059252E3266205A252E32662045252E34
:107BD00032660A25534D6178696D756D206665655D
:107BE00064726174657320286D6D2F73293A0A25BC
:107BF0005320204D3230332058252E32662059250F
:107C00002E3266205A252E32662045252E32660AEF
:107C100025534D6178696D756D20616363656C6591
:107C2000726174696F6E20286D6D2F7332293A0A64
:107C3000255320204D3230312058256C7520592590
:107C40006C75205A256C752045256C750A255341A5
:107C50006363656C65726174696F6E3A20503D7044
:107C600072696E742C20523D726574726163742C5B
:107C700020543D74726176656C0A255320204D3284
:107C800030342050252E32662052252E3266205464
:107C9000252E32660A2553416476616E6365642041
:107CA0007661726961626C65733A20533D4D696E0D
:107CB00020666565647261746520286D6D2F732977
:107CC0002C20543D4D696E2074726176656C20667F
:107CD0006565647261746520286D6D2F73292C2091
:107CE000423D6D696E696D756D207365676D656E7A
:107CF000742074696D6520287573292C20583D6D9A
:107D00006178696D756D205859206A65726B2028FD
:107D10006D6D2F73292C20205A3D6D6178696D752A
:107D20006D205A206A65726B20286D6D2F73292C87
:107D30002020453D6D6178696D756D2045206A652F
:107D4000726B20286D6D2F73290A255320204D3228
:107D500030352053252E32662054252E326620429F
:107D6000256C752058252E32662059252E32662026
:107D70005A252E32662045252E32660A2553486F35
:107D80006D65206F666673657420286D6D293A0AEB
:107D9000255320204D3230362058252E326620596A
:107DA000252E3266205A252E32660A004361703A2B
:107DB00025533A25630A0050525553415F4D4D55A6
:107DC0003200455854454E4445445F4D32300041E1
:107DD00055544F5245504F52545F504F5349544998
:107DE0004F4E004155544F5245504F52545F4641FB
:107DF0004E53004155544F5245504F52545F5445D5
:107E00004D50000044656C6574696F6E2066616951
:107E10006C65642C2046696C653A200046696C6587
:107E20002064656C657465643A004E6F7420534439
:107E3000207072696E74696E67005072696E74208A
:107E40007361766564005344207072696E742070AB
:107E50006175736564002533642F2533640066768D
:107E6000007468780050524E0022283229006E6F4C
:107E70002076616C696420636F6D6D616E64007A59
:107E800065726F72697A656400666163746F727996
:107E900020726573746F72656400696E6465782C16
:107EA0002074656D702C2075737465702C20756D51
:107EB0000050494E44412063616C207374617475B5
:107EC000733A2000503A005761697420666F72203F
:107ED00050494E4441207461726765742074656D29
:107EE00070657261747572653A002041002050001F
:107EF000204200204C00205200205A00204E4F54B7
:107F000020494E495449414C495A454400536865FB
:107F100065742000205A2056414C5545204F555439
:107F2000204F462052414E474500496E76616C69AC
:107F3000642073686565742049442E20416C6C6F21
:107F40007765643A20302E2E004155544F004C4145
:107F50004E472053454C20464F5243454400206431
:107F60003A0020693A0020703A0020643A00206903
:107F70003A0020703A00256925250A002569252543
:107F80000A0022283129002F2F0000204558545282
:107F9000554445525F434F554E543A3100204D41B0
:107FA0004348494E455F545950453A00312E300000
:107FB000206261736564206F6E204D61726C696E22
:107FC000204649524D574152455F55524C3A6874CC
:107FD0007470733A2F2F6769746875622E636F6DC2
:107FE0002F707275736133642F50727573612D46F3
:107FF00069726D776172652050524F544F434F4CF8
:108000005F56455253494F4E3A003737333130327D
:10801000346564005F0038323739002B004649521E
:108020004D574152455F4E414D453A50727573610F
:108030002D4669726D7761726520004D31313320B4
:1080400053006F6B20006E2F61003F546F7368699F
:10805000626120466C6173684169722047657449AA
:1080600050206661696C65640A00000125301D0CB2
:10807000FF24311C0BFF232F1B0A17FF0406222BA2
:108080001A03363535382569206D696E2C2025692F
:108090002073656300496E76616C6964204D2063CE
:1080A0006F64653A2025730A0050494E44412070A0
:1080B000726F62652063616C6962726174696F6E70
:1080C000207374617274004E6F2050494E444120F9
:1080D000746865726D6973746F7200736574006E95
:1080E0006F7A7A6C65004D424C004652004C7A0023
:1080F0004C616E6700315F37356D6D5F4D4B3235CA
:108100002D52414D426F3133612D453344763666F1
:10811000756C6C0052657600332E31342E312D385B
:108120003237390046697200534E20696E76616CB1
:10813000696400534E005245534554004D4D55520D
:1081400045530075766C6F0046414E0046414E50D7
:10815000494E54535400505255534100252E31304E
:1081600053200025346400457872656D6520737076
:10817000616E206F6620746865205A2076616C7588
:108180006573210025642F39004D313034533000A0
:10819000473158313059313830463430303000476B
:1081A000315A31304631333030004D313430533074
:1081B000004731452D302E303735463231303000D2
:1081C0004D32303453313030300047315A35463734
:1081D000323030004731452D312E35463231303086
:1081E0000047315A302E32004731583230322E3566
:1081F00045384631343030004731592D3246313020
:108200003030004731583234304532354632323022
:10821000300047315A302E3346313030300047314C
:1082200058353545384632303030004731583545BD
:1082300032394631383030004731583535453239DA
:108240004631303733004739324530004732380045
:108250004D313039004D31393000252D31322E313C
:108260003253252B382E316600457874727564655B
:10827000723A0025632531372E32666D6D00583A0B
:1082800000593A005A3A002563252D31332E3133F7
:1082900053252B352E3366002533750050494E4447
:1082A000412063616C6962726174696F6E206661FE
:1082B000696C65642E20436F6E74696E75652077F6
:1082C000697468207072657373696E67207468657D
:1082D000206B6E6F622E0050494E44412063616CEA
:1082E0006962726174696F6E20646F6E652E2043DF
:1082F0006F6E74696E756520776974682070726539
:108300007373696E6720746865206B6E6F622E00F0
:108310005A30005A31005930005931005830005855
:108320003100456E642073746F70732064696167F7
:1083300000473830004D3435004D3435205A004761
:108340003736004D3730312050300057697A61722E
:10835000642073746174653A2025640A004578705E
:108360006572696D656E74616C00302E3830003056
:108370002E363000302E343000302E323500446935
:108380007361626C65206661726D206D6F6465005B
:108390005265736574204D4D55004D4D55004D345B
:1083A00034004739390044697361626C6520666145
:1083B000726D206D6F64653F004732382058590058
:1083C0004D20383400852E2E002533642F300025B3
:1083D00033642F30006C63645F73656C666368653B
:1083E000636B5F617869732025642C2025640A0023
:1083F000486F74656E6400426564005A0059005805
:10840000002D2D2D2D2D2D2D2D2D2D2D2D2D2D2DC9
:108410002D2D2D2D2D00537570657250494E444100
:108420003A0051675567B181AA819F819081CC68DC
:1084300089818E68473159252E346645252E34664C
:108440000047315A252E32660047315835305931B0
:1084500035350046825167B36CD481CA81C08147EB
:108460003158252E346645252E3466004731463175
:108470003038300038822B821E821282468203827C
:10848000F881E881E1815425640047315A302E3467
:10849000004731592D334631303030005567558211
:1084A00050824C8246824D3834205859004D31302C
:1084B0003920533238300047312058313235205A74
:1084C00032303020463130303000496E76616C6990
:1084D00064205049442063616C2E20726573756C72
:1084E00074732E204E6F742073746F7265642074E1
:1084F0006F20454550524F4D2E004D3330312050A6
:10850000252E32662049252E32662044252E3266DD
:10851000004D33303320453020532533750052430E
:1085200000444556004245544100414C50484100EA
:1085300000002100240027002A002D003000330015
:1085400001010000040107010A01000022002500CA
:1085500028002B002E00310034000201000005012C
:1085600008010B01000020002300260029002C0038
:108570002F0032000001000003010601090105057A
:108580000505070508080808020202020A0A080889
:1085900004040404010101010101010103030303B7
:1085A00003030303040707070C0C0C0C0C0C0C0C46
:1085B0000202020206060606060606060B0B0B0B57
:1085C0000B0B0B0B07070A0A0A0A0A0A0505050422
:1085D0000404080801021020200808102040102080
:1085E0004080020102010804020101020408102077
:1085F0004080804020100804020180040201804075
:1086000020100804020108040201010204081020DD
:1086100040800102040810204080100804088010E7
:108620002040044080102040048000000A0B020912
:108630000C0D0E08070304010000000000000000FC
:10864000000000000000000000000000000000002A
:1086500000000000000012111000000000000000E7
:10866000000000000000000000000000000000000A
:1086700000000000000000000000000000000000FA
:10868000332E31342E31000A204F726967696E61D2
:108690006C2050727573612069330A20202050725B
:1086A0007573612052657365617263680A253230A3
:1086B0002E3230530053706F6F6C4A6F696E2069B1
:1086C0007320006164635F696E697400200A200A88
:1086D000200A2000416C6C20446174610053657273
:1086E000766963652070726570005368697070699F
:1086F0006E67207072657000537461746973746979
:108700006373004C616E6775616765004552415344
:10871000494E4720616C6C2064617461004661635E
:10872000746F72792052455345540050525553414D
:10873000334446570003000E0001004000030002CE
:1087400000000004007072757361336400323032CF
:10875000352D30342D32322032323A30333A3533FF
:108760000020332E31342E312D383237395F3737F0
:1087700033313032346564007374617274004D3289
:108780003900252D392E39535B00200A200A20009C
:1087900000004842000058419A998D4133335340BC
:1087A0004D4D55323A004D494E54454D50204245AD
:1087B00044206669786564004D494E54454D50200B
:1087C000484F54454E44206669786564004D4D55C8
:1087D000323A002533640018010419020A5E55E894
:1087E000546E540154B8532653AE524652F751D7E3
:1087F000518B51D7517451745174517451745174D7
:108800005174517451745174517451745174517440
:108810005174517451745174517451745174517430
:10882000513D51FC50B2503F500A50C04F764F1846
:108830004FDF4E9D4E804E01010101010101027189
:108840000171013232320303030303030303030301
:1088500003030303030303030393932438039303E2
:1088600001025603650066006700680069006A003F
:108870006B006C00730074007D007E00C900D300A3
:10888000DD00CA00D400DE002D01370141012E01B8
:10889000380142012F013901430130013A014401FD
:1088A00031013B014501320191019201F501F601CF
:1088B000F701F801F901FA01FB01FC018403EB5512
:1088C0000156E055D755D0554658E647C955BF55CE
:1088D000252E3230530A70727573612E696F2F30F6
:1088E00034256875007B5B4552523A00332E313493
:1088F0002E31005D5B4657523A005D5B54494D3A5C
:10890000005D5B464E4D3A005D5B46454D3A005D6D
:108910005B5043443A005B5446553A005B50524E1C
:108920003A005B50464E3A305D005B4449413A00A4
:108930005D5B4154423A005D5B4154303A005D5BFF
:108940005354423A005B5354303A007B5B50524ED2
:108950003A355D007B5B50524E3A305D007B5B5098
:10896000524E3A395D007B5B50524E3A385D007B87
:108970005B5245533A305D5B46494C3A007B5B5253
:1089800045533A315D5B46494C3A000000211042A4
:108990002063308440A550C660E770088129914A61
:1089A000A16BB18CC1ADD1CEE1EFF13112100273E8
:1089B000325222B5529442F772D662399318837BB1
:1089C000B35AA3BDD39CC3FFF3DEE3622443342038
:1089D000040114E664C774A44485546AA54BB52801
:1089E000850995EEE5CFF5ACC58DD55336722611C8
:1089F000163006D776F6669556B4465BB77AA71951
:108A0000973887DFF7FEE79DD7BCC7C448E558868F
:108A100068A7784008611802282338CCC9EDD98EA0
:108A2000E9AFF9488969990AA92BB9F55AD44AB727
:108A30007A966A711A500A333A122AFDDBDCCBBFF0
:108A4000FB9EEB799B588B3BBB1AABA66C877CE4F7
:108A50004CC55C222C033C600C411CAEED8FFDEC40
:108A6000CDCDDD2AAD0BBD688D499D977EB66ED507
:108A70005EF44E133E322E511E700E9FFFBEEFDD90
:108A8000DFFCCF1BBF3AAF599F788F8891A981CA6D
:108A9000B1EBA10CD12DC14EF16FE18010A100C24C
:108AA00030E3200450254046706760B9839893FBFB
:108AB000A3DAB33DC31CD37FE35EF3B1029012F39C
:108AC00022D2323542145277625672EAB5CBA5A84B
:108AD0009589856EF54FE52CD50DC5E234C324A0EC
:108AE0001481046674476424540544DBA7FAB799DB
:108AF00087B8975FE77EF71DC73CD7D326F236913C
:108B000006B01657667676154634564CD96DC90EA2
:108B1000F92FE9C899E9898AB9ABA944586548068B
:108B2000782768C018E1088238A3287DCB5CDB3F3A
:108B3000EB1EFBF98BD89BBBAB9ABB754A545A37DB
:108B40006A167AF10AD01AB32A923A2EFD0FED6C0A
:108B5000DD4DCDAABD8BADE89DC98D267C076C642B
:108B60005C454CA23C832CE01CC10C1FEF3EFF5D1A
:108B7000CF7CDF9BAFBABFD98FF89F176E367E557B
:108B80004E745E932EB23ED10EF01E7C3C3E3F2FC3
:108B90002A225C0024F4D43050C38E20C2A2401795
:108BA000828B7011127A910D816CD90AA861E1084B
:108BB000C7586607615143061E4B5D05C145A704B2
:108BC0001A411104093D9803713931034036DB0223
:108BD00065339102D4305402802E1D02632CEE01C5
:108BE000752AC501B028A001102781018F256401D5
:108BF0002B244B01E0223401AC211F018D200D01FB
:108C0000801FFC00841EED00971DDF00B81CD20001
:108C1000E61BC600201BBC00641AB200B219A800F3
:108C20000A19A0006A189900D117910040178B000B
:108C3000B516840031167E00B31579003A1573001D
:108C4000C7146F0058146A00EE136600881363009F
:108C500025135E00C7125B006C12570015125400FA
:108C6000C111510070114F0021114B00D610490065
:108C70008D1047004610440002104200C00F400013
:108C8000800F3E00420F3C00060F3B00CB0E380029
:108C9000930E37005C0E3500270E3400F30D3200C2
:108CA000C10D3100900D3000600D2E00320D2D00F1
:108CB000050D2C00D90C2B00AE0C2900850C2900C9
:108CC0005C0C2700350C27000E0C2600E80B240056
:108CD000C40B2400A00B23007D0B23005A0B2100A2
:108CE000390B2100180B2000F80A1F00D90A1E00BA
:108CF000BB0A1E009D0A1D00800A1D00630A1C009D
:108D0000470A1B002C0A1B00110A1A00F7091A0057
:108D1000DD091900C4091900AB09190092091700EF
:108D20007B091800630917004C0916003609160064
:108D3000200916000A091500F5081500E0081400BE
:108D4000CC081400B8081400A408140090081300FC
:108D50007D0812006B081300580812004608120024
:108D60003408110023081100120811000108110035
:108D7000F0071000E0071000D0071000C007100037
:108D8000B0070F00A107100091070E0083070F0026
:108D900074070F0065070E0057070E0049070E0005
:108DA0003B070D002E070E0020070D0013070D00D6
:108DB00006070D00F9060C00ED060D00E0060C009C
:108DC000D4060C00C8060C00BC060C00B0060C0053
:108DD000A4060B0099060C008D060B0082060B0002
:108DE00077060B006C060B0061060A0057060B00A5
:108DF0004C060A0042060A0038060A002E060A003F
:108E000024060A001A060A001006090007060A00CE
:108E1000FD050900F4050900EB050900E20509005C
:108E2000D9050900D0050900C7050900BE050900DC
:108E3000B5050800AD050800A50509009C0508005A
:108E4000940508008C050800840508007C050800CE
:108E5000740508006C050700650508005D0507003E
:108E6000560508004E0507004705070040050800A5
:108E700038050700310507002A050700230507000C
:108E80001C050600160507000F050700080506006B
:108E900002050700FB040600F5040700EE040600C7
:108EA000E8040600E2040700DB040600D50406001F
:108EB000CF040600C9040600C3040600BD04060072
:108EC000B7040600B1040500AC040600A6040600C1
:108ED000A00405009B04060095040500900406000C
:108EE0008A04050085040500800406007A04050054
:108EF00075040500700405006B0405006604050098
:108F0000610405005C0405005704050052040500D7
:108F10004D04050048040500430405003E04040018
:108F20003A04050035040500300404002C04050053
:108F300027040400230405001E0404001A0404008E
:108F400016040500110404000D04040009040500C2
:108F50000404040000040400FC030400F8030400FB
:108F6000F4030400F0030400EC030400E80304002D
:108F7000E4030400E0030400DC030400D80304005D
:108F8000D4030400D0030400CC030400C80303008E
:108F9000C503030024F404D9201BC40C5C0E980400
:108FA000C4095F0265077101F405F900FB04B30011
:108FB00048048700C10369005803550003034500B6
:108FC000BE023A008402310053022A002902250021
:108FD00004022000E4011C00C8011900AF011700C1
:108FE0009801140084011300710110006101100048
:108FF00051010E0043010D0036010B002B010B0047
:1090000020010B00150109000C01090003010800F3
:10901000FB000800F3000800EB000700E400060076
:10902000DE000600D8000600D2000600CC000500D5
:10903000C7000500C2000500BD000400B90004001F
:10904000B5000400B1000400AD000400A900040054
:10905000A5000300A20003009F0004009B00030082
:1090600098000300950002009300030090000300A5
:109070008D0002008B0003008800020086000200C1
:1090800084000300810002007F0002007D000200D6
:109090007B000200790002007700010076000200E8
:1090A0007400020072000100710002006F000200F3
:1090B0006D0001006C0002006A00010069000200FE
:1090C0006700010066000100650001006400020005
:1090D0006200010061000100600001005F00020009
:1090E0005D0001005C0001005B0001005A0001000E
:1090F000590001005800010057000100560001000E
:10910000550001005400010053000000530001000D
:109110005200010051000100500001004F00010009
:109120004E0000004E0001004D0001004C00010007
:109130004B0000004B0001004A0001004900010003
:109140004800000048000100470001004600000000
:1091500046000100450000004500010044000100F8
:1091600043000000430001004200000042000100F3
:109170004100000041000100400001003F000000EC
:109180003F0001003E0000003E0001003D000000E5
:109190003D0001003C0000003C0000003C000100DC
:1091A0003B0000003B0001003A0000003A000100D3
:1091B00039000000390001003800000038000000CC
:1091C00038000100370000003700010036000000C1
:1091D00036000000360001003500000035000000B8
:1091E00035000100340000003400000034000100AC
:1091F00033000000330000003300010032000000A3
:109200003200000032000100310000003100000097
:10921000310001003000000030000000300001008B
:109220002F0000002F0000002F0000002F00010081
:109230002E0000002E0000002E0001002D00000076
:109240002D0000002D0000002D0001002C0000006A
:109250002C0000002C0000002C0001002B0000005E
:109260002B0000002B0000002B0001002A00000052
:109270002A0000002A0000002A0001002900000046
:109280002900000029000000290000002900010039
:10929000280000002800000028000000280000002E
:1092A0002800010027000000270000002700000020
:1092B0002700000027000100260000002600000013
:1092C0002600000026000000260001002500000006
:1092D00025000000250000002500000025000000FA
:1092E00025000100240000002400000024000000EC
:1092F00024000000240001002300000023000000DF
:1093000023000000230000002300000023000000D1
:1093100023000100220000002200000022000000C3
:1093200022000000220000002200010021000000B5
:1093300021000000210000002100000021000000A9
:10934000210000002100010020000000200000009A
:10935000200000002000000020000000200000008D
:1093600020000000200001001F0000001F0000007E
:109370001F0000001F0000001F0000001F00000071
:109380001F0001001E0000001E0000001E00000063
:109390001E00000045303A20005A3A2000593A2079
:1093A00000583A20004D53312C4D53322050696EF5
:1093B0007300504944204175746F74756E65206662
:1093C000696E6973686564212050757420746865DE
:1093D000206C617374204B702C204B6920616E648B
:1093E000204B6420636F6E7374616E7473206672B9
:1093F0006F6D2061626F766520696E746F20436FB8
:109400006E66696775726174696F6E2E6800504987
:1094100044204175746F74756E65206661696C6572
:1094200064212074696D656F75740020403A0054A2
:109430003A00423A00504944204175746F74756E89
:1094400065206661696C6564212054656D70657284
:10945000617475726520746F6F2068696768002099
:109460004B643A2000204B693A2000204B703A2090
:109470000020436C617373696320504944200020CD
:1094800054753A2000204B753A2000206D61783ADF
:109490002000206D696E3A200020643A200020628E
:1094A0006961733A2000504944204175746F7475A6
:1094B0006E65207374617274005049442041757464
:1094C0006F74756E65206661696C65642E204261FB
:1094D00064206578747275646572206E756D62655E
:1094E000722E00486F74656E642066616E20737022
:1094F000656564206973206C6F776572207468619C
:109500006E206578706563746564005072696E746E
:109510002066616E207370656564206973206C6FCE
:10952000776572207468616E206578706563746514
:1095300064004D494E54454D5020424544004D492C
:109540004E54454D50004D415854454D50004D41ED
:109550005854454D50204245440070012C01900163
:109560002701B0012201C0011D01F0011801100204
:10957000130130020E016002090190020401C002D1
:10958000FF000003FA004003F5008003F000D00361
:10959000EB002004E6007004E100E004DC0040057C
:1095A000D700C005D2004006CD00D006C800800715
:1095B000C3003008BE00F008B900C009B400B00A0A
:1095C000AF00B00BAA00D00CA500000EA000500FF9
:1095D0009B00C01096005012910000148C00C01522
:1095E0008700B0178200B0197D00D01B7800001EE4
:1095F000730040206E0090226900F0246400402730
:109600005F0090295A00E02B5500102E50002030AA
:109610004B0010324600E033410090353C001037DB
:10962000370070383200A0392D00B03A2800A03B36
:109630002300603C1E00103D1900903D1400103EB8
:109640000F00703E0A00C03E0500003F00002048A9
:109650004F54454E4420544845524D414C2052559C
:109660004E415741590020484541544245442054F9
:109670004845524D414C2052554E41574159005496
:109680004845524D414C2052554E41574159004298
:10969000454420544845524D414C2052554E415767
:1096A00041590020544845524D414C2052554E419D
:1096B00057415920285052454845415420484F545D
:1096C000454E44290020544845524D414C205255A6
:1096D0004E41574159202850524548454154204851
:1096E0004541544245442900505245484541542083
:1096F0004552524F52004245442050524548454140
:1097000054204552524F5200207472696767657247
:1097100065642100486561746572732073776974AC
:1097200063686564206F66662E20003A20004572EB
:10973000723A200000FF0102010002FFFFFE00015B
:10974000FE01FF00506C6561736520726573746182
:109750007274005553415254322072782046756C11
:109760006C212121003A2000252D31322E31325337
:10977000252D642F36002533642F252D33640020DA
:109780003A200025335300252D377300252D313520
:109790002E313553252D35640A252D31352E3135A1
:1097A00053252D35640A0025530A20252D31362EE8
:1097B000313653252D33640A20252D31362E31368E
:1097C00053252D33640025530A20252D31362E31A3
:1097D0003653252D33640A20252D31362E3136534C
:1097E000252D33640A20252D31362E313653252D73
:1097F00033640025530A20252D31362E313653256A
:109800002D33640A25530A20252D31362E31365347
:10981000252D33640A0020257325336481200A0036
:1098200025752E25752E25752E2575002000200006
:10983000466C6173684169722049502041646472CA
:109840003A004D4D5520202020202020204E2F4131
:109850000025642E25642E2564002046573A0032E8
:109860003032352D30342D32320045334476366671
:10987000756C6C0052414D426F31336100315F377E
:10988000356D6D5F4D4B32350020486173683A3756
:10989000373331303234656400205265706F3A706E
:1098A0007275736133640020332E31342E312D38BC
:1098B000323739004669726D776172653A003E0051
:1098C000464C4558202D20203234302F353000466C
:1098D0004C4558202D20203234300050502020207C
:1098E0002D20203235342F313030005050202020B0
:1098F0002D20203235340048495053202D2020326D
:1099000032302F3130300048495053202D20203242
:1099100032300041425320202D20203235352F3166
:1099200030300041425320202D2020323535005068
:10993000412020202D20203237352F393000504152
:109940002020202D20203237350050564220202D57
:1099500020203231352F37350050564220202D201F
:10996000203231350050432020202D202032373541
:109970002F3130350050432020202D202032373524
:109980000041534120202D20203236302F313035F8
:109990000041534120202D202032363000504554C4
:1099A00020202D20203233302F38350050455420D0
:1099B000202D202032333000504C4120202D2020FB
:1099C0003231352F363000504C4120202D202032AE
:1099D0003135006E6F7A7A6C65202D20203235305B
:1099E0002F30006661726D2020202D20203235300E
:1099F0002F3830001000C90210012C014001220153
:109A000070011801B0010E01F00104015002FA00CA
:109A1000B002F0003003E600D003DC009004D20076
:109A20007005C800A006BE000008B400B009AA0076
:109A3000D00BA000600E960060118C000015820013
:109A400020197800C01D6E00A0226400B0275A00C3
:109A5000902C500000314600E0343C0010383200B9
:109A6000903A2800603C1E00A03D1400803E0A0091
:109A7000203F00004D6561737572652063656E74EB
:109A8000657220200078797A63616C5F6D6561731F
:109A90007572655F656E7465720A0078797A6361C4
:109AA0006C5F73706972616C382063783D25642047
:109AB00063793D2564207A303D256420647A3D2514
:109AC00064207261646975733D25642061643D257D
:109AD000640A0078797A63616C5F736561726368A8
:109AE0005A206E6F207369676E616C0A20783D257D
:109AF0006C6420793D256C64207A3D256C640A00F5
:109B0000204F4E2D5349474E414C20617420783DE3
:109B1000256420793D2564207A3D25642061643DDB
:109B200025640A0078797A63616C5F73656172639A
:109B3000685A20783D256C6420793D256C64207A34
:109B40003D256C640A002530327800205B256620B4
:109B500025665D206D6D207061747465726E206382
:109B6000656E7465720A00205B25662025665D5B64
:109B700025665D206D6D20646976657267656E632C
:109B8000650A000000F000F801FC03FE07FE07FE76
:109B900007FE07FC03F801F000000000000000F0E1
:109BA00000F801FC03FC03FC03FC03F801F00000D7
:109BB00000000078797A63616C5F6D65617375721E
:109BC000655F6C656176650A00203C200057415254
:109BD0004E494E473A2046726F6E7420706F696E20
:109BE00074206E6F7420726561636861626C652EAB
:109BF000205920636F6F7264696E6174653A00006A
:109C0000000040410000804000005C4300008040B4
:109C100000005C4300004443000040410000444316
:109C200025642F3400497465726174696F6E3A203F
:109C30000043616C6962726174696F6E206661696C
:109C40006C65642120436865636B207468652061DE
:109C500078657320616E642072756E20616761693A
:109C60006E2E0078797A63616C5F73706972616CD3
:109C7000322063783D25642063793D2564207A3065
:109C80003D256420647A3D256420726164697573A2
:109C90003D25642061643D25640A000A00436F7518
:109CA0006E74646F776E3A202564200025640A0084
:109CB0005363616E20636F756E74646F776E3A20C4
:109CC000005061747465726E2063656E74657220F5
:109CD0005B25662025665D2C206D617463682025F8
:109CE0006625250A00205B25662C2025665D5B2500
:109CF000665D2066696E616C20636972636C650ADB
:109D0000000000A0400000A0400000004000007AD9
:109D100043000056439AD95143FFFFFFE02D903E88
:109D20008988B24111369C3E7777C14129CBB03E3C
:109D3000EFEEDA41BA49CC3EEFEEFC4161C3F33EAF
:109D4000EFEE16429CA2133FCDCC36428AB0113FB3
:109D5000ABAA56428863DD3DABAA5642B8AF433F3B
:109D6000555572421826533F33B38242302A593F29
:109D7000EF6E8642000070C10000C8420000C4C1FE
:109D80000000A0410000E0C000002041000060C0D1
:109D90000000C0400000A0412222F2400000A0C10B
:109DA0009A99A14000000CC255550542436F6F6C53
:109DB000696E672074696D65722073746F70706569
:109DC000640048656174657220636F6F6C646F77BF
:109DD0006E00436F6F6C696E672054696D656F75B7
:109DE00074207374617274656400536176696E6780
:109DF00020616E64207061726B696E6700486561F6
:109E000074657220636F6F6C646F776E2070656E1F
:109E100064696E6700526573756D696E6720585985
:109E20005A0057726974696E6720746F2066696C96
:109E3000653A200046696C6520616C7265616479E1
:109E4000206F70656E656400BA5AA95A955A805A97
:109E50006A5A575A415A2D5A1C5A065A955AA95AA3
:109E6000F259E359CF59BE59A959ED619359815916
:109E70006E595D594859355921590C590359F158B2
:109E8000DC584D363030204155544F0046494E4441
:109E9000412066696C616D656E742072756E6F75B8
:109EA000742100436F6D6D756E69636174696F6EC7
:109EB0002074696D656F75740050726F746F636F95
:109EC0006C204572726F72000300035665727369ED
:109ED0006F6E206D69736D6174636800436F6D6DA3
:109EE000616E64204572726F7200436F6D6D616EBA
:109EF000642072656A6563746564004D4D55204247
:109F00007574746F6E207075736865640052657443
:109F10007279427574746F6E507265737365640004
:109F2000175D025DEB5CD65CC15CAD5C9D5C865CE4
:109F30006F5C585C445C305C1A5C1A5C1A5C055CB3
:109F4000055C055CF25BF25BF25BDF5BDF5BDF5BBA
:109F5000C85BC85BC85BB35BB35BB35B9D5B9D5B7E
:109F60009D5B8D5B785B625B4C5B3D5B305B195B43
:109F7000065BF45AE15ACF5ABF5A427574746F6E39
:109F800000436865636B55736572496E7075742D17
:109F900062746E4C4D522000526573657452657444
:109FA0007279417474656D7074730046493A20206B
:109FB00046533A202020203E20208220202081006D
:109FC000486F74656E642074656D70657261747538
:109FD0007265207265616368656400526573756DB2
:109FE000696E672054656D7000436F6F6C646F77A6
:109FF0006E20666C616720636C6561726564002029
:10A00000573A0020453A00543A004E6F20307846C7
:10A01000462072656365697665640053656E6469A0
:10A020006E6720307846460046696C652073656C23
:10A030006563746564002053697A653A2000466957
:10A040006C65206F70656E65643A20004E6F7720F6
:10A0500066726573682066696C653A20004E6F779A
:10A0600020646F696E672066696C653A2000222063
:10A07000706F73002220706172656E743A22005313
:10A080005542524F5554494E452043414C4C207443
:10A0900061726765743A2200747279696E67207420
:10A0A0006F2063616C6C207375622D67636F6465EC
:10A0B0002066696C6573207769746820746F6F20FF
:10A0C0006D616E79206C6576656C732E00062833A1
:10A0D000D036C23E013F154132423B43F2443B453C
:10A0E000F24622473B48F2493B4AF05898590C5AED
:10A0F000085B0C5C086110679B6E2271077208FF99
:10A10000095A0D000EF019145E0820642B6D322FD1
:10A11000FF2022257322002025236C780044495219
:10A120005F45584954004449525F454E5445523AA0
:10A1300020257320222573220A006175746F25691A
:10A140002E6700041A44656372656D656E7452650E
:10A15000747279417474656D70747300081B1C0B04
:10A1600014525354436F6D6D54696D656F7574006F
:10A170002C206C6173742062797465733A2000221C
:10A18000206661696C65643A204275666665722076
:10A1900066756C6C21002200456E717565696E678D
:10A1A00020746F207468652066726F6E743A202286
:10A1B000004572726F723A004D4D5532746F6F6C7C
:10A1C0003D004D4D55323A004D4D55323A006563D4
:10A1D000686F3A003E53302A63362E004D4D5520AD
:10A1E000697320008638CF6311241FBECFEFD1E200
:10A1F000DEBFCDBF00E00CBF13E0A0E0B2E0E8E5B9
:10A20000F5E503E00BBF02C007900D92A230B10745
:10A21000D9F727E1A2E0B3E001C01D92A731B20750
:10A22000E1F710E5C3EFD0E500E006C02197010992
:10A23000802FFE010F94F0A4C23FD10780E00807F1
:10A24000A9F70E9441ED0D949AAA0C94DE862F92F4
:10A250003F924F925F926F927F928F929F92AF92B6
:10A26000BF92CF92DF92EF92FF920F931F93CF9303
:10A27000DF93CDB7DEB72F970FB6F894DEBF0FBED2
:10A28000CDBF6C011B015A01FC011782168283812C
:10A290009E012F5F3F4F490181FDD2C08FEF9FEF9D
:10A2A000EEC2F12C512C00E0003238F48B3209F16F
:10A2B00090F48032F9F0833209F107FD34C020EDCB
:10A2C000280F2A3020F506FF1BC0FAE0FF9E200D64
:10A2D0001124F22E05C08D3279F0803371F70160C0
:10A2E000F10193FD859193FF81911F018111DCCFD5
:10A2F0001AC002600460F4CF0860F2CF0061F0CFB2
:10A300003AE0539E200D1124522E0062E9CF8E3286
:10A3100021F406FDB1C20064E3CF8C3611F400686D
:10A32000DFCF8836E9F29BEB980F933008F05FC0DF
:10A330000061805E06FD02C046E0F42E102F1F7300
:10A34000853609F05BC0106417FF61C08F2D9BE359
:10A350009F1508F48BE344244394480E27E035010D
:10A36000F4E06F0E711CF50160817181828193812F
:10A37000042DA4010F9499A05C01F981FC87F0FFE2
:10A3800003C00DE2F3FF07C00BE211FD04C0012F73
:10A39000047012FD00E22C852C70E22E09F46BC0D3
:10A3A0000111D8C2F3E0E12CF515A0F483E0E52C0F
:10A3B000E81A13FD08C0B60180E290E00F9448A2AD
:10A3C000EA94E110F8CF002329F0B601802F90E045
:10A3D0000F9448A23C8528E7A22E21E7B22E33FD38
:10A3E00004C09CE7A92E91E7B92E107122C09BE909
:10A3F000980F933008F047C10F7E9CCF863611F43A
:10A400001068A2CFFF2009F49FCFFA949DCFE7E018
:10A410002F2DEF1518F427E037E0F32E412C9FCFB6
:10A4200011118052B60190E00F9448A28FEFA81A44
:10A43000B80AF50184918111F3CFE11084C2530170
:10A44000F6019381F10193FD859193FF81911F01A5
:10A45000882309F411C2853241F493FD859193FF5D
:10A4600081911F01853209F01CCFB60190E00F9455
:10A4700048A23501E4CF17FF6FC04A0CFC85F4FFFA
:10A4800004C08A81813309F44A9414140CF086C004
:10A4900028E0241510F488E0482E85E090E017FFAE
:10A4A00006C0C501B7FE02C090E080E00196011130
:10A4B0000196FF2031F02F2D30E02F5F3F4F820FAC
:10A4C000931F5816190619F014F0E52CE81A812F7D
:10A4D000897011F4E11067C0002329F0B601802FC4
:10A4E00090E00F9448A213FD02C0E11063C017FF73
:10A4F0007CC08501B7FE02C010E000E0C5018419F0
:10A5000091092C016F2D70E0EE27FF27E61BF70B5A
:10A51000FF87EE870F3F100729F4B6018EE290E027
:10A520000F9448A2A016B1060CF44BC04016510679
:10A530000CF047C0F501E01BF10BE80DF91D81811E
:10A54000015011092E853F8502171307E4F1B6016A
:10A5500090E00F9448A2DECF16FD9FCFEF2DF0E0E4
:10A56000EA15FB0534F03CEFA3163FEFB3060CF001
:10A5700010683296E80DF91D01C0FA94FF2019F019
:10A5800082918033D1F317FF88CF442443944F0C3A
:10A59000FA141B0431F02CF0FA187FCF44244394B2
:10A5A0007CCFF12C7ACFB60180E290E00F9448A2E4
:10A5B000EA9490CFB60180E390E00F9448A2EA9429
:10A5C00094CF80E3BDCFA016B10641F49A819633B3
:10A5D00050F4953319F43C8534FF05C0B60190E082
:10A5E0000F9448A22ACF81E3F9CF8A81813319F0F1
:10A5F0009C859F7E9C87B60190E00F9448A2FF2027
:10A60000A9F0B6018EE290E00F9448A2F394F3947F
:10A61000E2E001E00E0FE80DF92DF11D8081B60199
:10A6200090E00F9448A2E02F0F11F3CF85E690E061
:10A6300014FF02C085E490E0B6010F9448A2B7FC75
:10A6400006C0A114B104C1F4EC85E4FF15C0B194B7
:10A65000A194B1088DE2B60190E00F9448A280E386
:10A660002AE0A216B10454F4B60190E00F9448A277
:10A67000B601C501C096B4CF8BE2EDCF8F5FFAE093
:10A68000AF1AB108EDCF8336C9F0833771F1833546
:10A6900009F05BC03501F2E06F0E711CF501A0807E
:10A6A000B1806F2D70E006FD02C06FEF7FEFC50136
:10A6B0000F94DCA19D878C8700680DC0350132E0C6
:10A6C000630E711CF5018081898321E030E03D87B4
:10A6D0002C8754010F7703FD06C02C853D8552164B
:10A6E000130609F0A8F4E52C2BC0350132E0630E07
:10A6F000711CF501A080B1806F2D70E006FD02C0D5
:10A700006FEF7FEFC5010F9401A29D878C87E2CF89
:10A71000B60180E290E00F9448A25A94DECFF50192
:10A7200007FD859107FF81915F01B60190E00F94CD
:10A7300048A2E110EA948C859D8501979D878C87BE
:10A74000EC85FD85EF2B59F778CE843619F08936E4
:10A7500009F074C0350107FF66C0F4E06F0E711C8C
:10A76000F5016081718182819381102F1F7697FF9F
:10A7700008C090958095709561957F4F8F4F9F4F42
:10A7800010682AE030E0A4010F946FA3A82EA81847
:10A79000BA2C012F16FF0AC00E7FAF1438F414FF35
:10A7A00004C012FD02C0012F0E7EBF2C04FFA3C007
:10A7B000FE01EA0DF11D8081803309F095C0097E0C
:10A7C000F02FF870EF2E03FDA5C000FF9FC0FA2CFC
:10A7D000B51410F4F50CFB1804FFA2C0B60180E319
:10A7E00090E00F9448A202FF09C088E790E001FFC3
:10A7F00002C088E590E0B6010F9448A2AF1408F4B7
:10A800009BC0AA940A2D10E00F5F1F4F080D191D61
:10A81000F80182918F01B60190E00F9448A2801652
:10A820009106B1F70ACEF2E06F0E711CF50160815E
:10A830007181072E000C880B990B97CF102F85374D
:10A84000A9F41F7E2AE030E0350117FF44C0F4E090
:10A850006F0E711CF5016081718182819381A40169
:10A860000F946FA3A82EA8181F7792CF197F8F3649
:10A8700079F1F0F4883539F1F601868197812F96C8
:10A880000FB6F894DEBF0FBECDBFDF91CF911F9101
:10A890000F91FF90EF90DF90CF90BF90AF909F907F
:10A8A0008F907F906F905F904F903F902F90089582
:10A8B000803739F0883701F714FD146020E130E06B
:10A8C000C3CF1061F9CF04FD166020E132E0BCCFA8
:10A8D00028E030E0B9CFF2E06F0E711CF501608125
:10A8E000718190E080E0BBCF02FD02C0B39468CFDD
:10A8F000B394B39465CF802F867809F461CFF6CFF7
:10A90000B60180E290E00F9448A2B394B514C0F36E
:10A91000E12C62CFE52CEB18B51408F45DCFF8CF2D
:10A92000802F867809F46ACF8BE201FF80E207FD71
:10A930008DE2B60190E060CFB60180E390E00F9425
:10A9400048A2FA945BCFB60180E290E00F9448A24F
:10A95000EA9473CD24E0E12C251508F036CD84E08F
:10A9600026CD20E030E040E85FEB60917E02709100
:10A970007F0280918002909181020F94FDA588232F
:10A9800021F1E0913812F0913912E55BFF4E8081A0
:10A990008B7F8230D1F480E1EEE7F2E0A1E6B2E114
:10A9A00001900D928A95E1F780E090E0A0E8BFEB7E
:10A9B00080937E0290937F02A0938002B0938102E5
:10A9C00080914D1290914E12089581E090E008958B
:10A9D00080E1E9E2F6E0A1E6B2E101900D928A950C
:10A9E000E1F70895E0E5F6E7833021F0E82FF0E0A5
:10A9F000E35BF94884910895809142059091430565
:10AA00002091440530914505821B930B8F77992740
:10AA10000895982F9F7083FF0DC080917B00886000
:10AA200080937B0080917C00887F9770892B809336
:10AA30007C00089580917B00877FF2CF4FEF5FEF1E
:10AA4000BA0185EE9FE00F9416A44FEF5FEFBA01B5
:10AA500089EE9FE00F9416A44FEF5FEFBA018DEDE2
:10AA60009FE00F9416A44FEF5FEFBA0181EE9FE0D5
:10AA70000F9416A44FEF5FEFBA0185ED9FE00F949E
:10AA800016A44FEF5FEFBA0189ED9FE00F9416A473
:10AA90004FEF5FEFBA0185EC9FE00F9416A44FEFE4
:10AAA0005FEFBA0189EC9FE00F9416A44FEF5FEFC0
:10AAB000BA018DEC9FE00F9416A44FEF5FEFBA013F
:10AAC00081ED9FE00D9416A480369105F8F4409135
:10AAD0003812509139122091491030914A10421782
:10AAE000530739F460913C1270913D121616170607
:10AAF0006CF0B901680F791FFB01E359FF4F241770
:10AB0000350730F481E04E175F0708F480E00895C0
:10AB1000EE3EF140F8F06C5F7F4F6E3E714018F4EE
:10AB200049365105B8F483599F4F4817590770F3B8
:10AB30004DEE51E0421B530B70E060E0C901855BB4
:10AB40009F4E0F9412AA8FB7F89410924A10109249
:10AB500049108FBF81E0089580914405909145058B
:10AB6000909343058093420580EF99E69F938F93DE
:10AB700080913E1290913F12A0914012B0914112EB
:10AB80000196A11DB11DBF93AF939F938F938BE44B
:10AB900094E69F938F9382E594E69F938F930F940F
:10ABA000A2A28DB79EB70A960FB6F8949EBF0FBEAD
:10ABB0008DBF08950F931F93CF93DF93EC01C60FC2
:10ABC000D71F8C179D0779F08C010F5F1F4F0F94D3
:10ABD000E0A38F3F31F081E0DF91CF911F910F9182
:10ABE0000895C801EECF80E0F7CF682F880F770B6C
:10ABF0008091381290913912825B9F4E0F9437AA40
:10AC00009C019093BC048093BB0481E0232B09F446
:10AC100080E008958091BB049091BC044AE050E02C
:10AC200070E060E001960F946B9F862F08958091ED
:10AC3000BB049091BC044AE050E070E060E00196F3
:10AC40000F946B9FCB0108950F931F93CF93DF93C6
:10AC50008C01862FEA010E94F555882319F10E9484
:10AC600017569C0197FF03C0319521953109253670
:10AC700031059CF09F938F9381EB91EA9F938F9383
:10AC80008DEC96E79F938F930F94A2A20F900F9055
:10AC90000F900F900F900F9080E0DF91CF911F9158
:10ACA0000F910895F80180818823B1F3CE01DF91DF
:10ACB000CF911F910F910D94E0A38091BB049091CF
:10ACC000BC044AE050E070E060E001960D946B9F98
:10ACD00060E086E69FE00F9404A460E088E69FE0D1
:10ACE0000F9404A460E085E69FE00F9404A460E064
:10ACF00084E69FE00F9404A460E082ED9EE00F9450
:10AD000004A460E08FEC9EE00D9404A42F923F9287
:10AD10004F925F926F927F928F929F92AF92BF926B
:10AD2000CF92DF92EF92FF920F931F93CF93DF9317
:10AD3000CDB7DEB7CC58D2400FB6F894DEBF0FBE09
:10AD4000CDBFCB58DD4F688379838A839B83C557FA
:10AD5000D240FE01E754FE4F88E2DF011D928A9542
:10AD6000E9F7E85BF1401F0180E991E0DF01FC01B8
:10AD70001D923197E9F7C75ADD4F19821882C955DC
:10AD8000D2409E012F513E4FC159DD4F3983288358
:10AD9000CF56D2408E01075A1D4FCE018F5C9D4F7A
:10ADA000C359DD4F99838883CD56D2403C01490178
:10ADB00040EBA42E4FE0B42E53E2C52ED12CF12C43
:10ADC000E12CB6010D2C000C880B990B0F946E9E94
:10ADD000D4016D937D938D939D934D01F801619105
:10ADE00071918F01072E000C880B990B0F946E9EAA
:10ADF000D3016D937D938D939D933D01BFEFEB1A2E
:10AE0000FB0AE6E0EE16F10409F038C3CB58DD4F3B
:10AE1000288139814A815B81C557D240C159DD4FB4
:10AE2000A881B981CF56D2406D917D918D919C9131
:10AE30000F9491A7412C512C320118160CF402C327
:10AE4000C359DD4F08811981CD56D2400C5E1F4F8A
:10AE5000C159DD4FE880F980CF56D240B4E1EB0E06
:10AE6000F11C6E01EFEDCE1AEDEFDE0A9E012B55BF
:10AE70003E4FCF58DD4F39832883C157D240D80188
:10AE80004D905D906D907C90F70160817181828121
:10AE90009381D7015E914E913E912E917D010F9449
:10AEA00007A54B015C01F801529142913291229128
:10AEB0008F01C301B2010F9407A5A50194010F945E
:10AEC00007A6D6019E938E937E936E936D01CF5805
:10AED000DD4FE881F981C157D240B292A29292929D
:10AEE0008292CF58DD4FF983E883C157D240C359CE
:10AEF000DD4F28813981CD56D2400217130709F062
:10AF0000BECF4E013FE6831A3EEF930A5E0183EF08
:10AF1000A81A8DEFB80A61018101EE24E394F12CA7
:10AF2000D4014D905D906D907D904D012D913D919E
:10AF30004D915C91C301B2010F9408A59B01AC0136
:10AF40000F9408A5F80164A775A786A797A7F1E055
:10AF5000EF16F10461F0D80198964D925D926D92D2
:10AF60007C929B97F8014482558266827782FFEF3C
:10AF7000EF1AFF0AF501208131814281538184E07B
:10AF8000A80EB11C64817581868197810F9407A5F5
:10AF900020E030E040EC50E40F94AD9ED601DC960A
:10AFA0006D937D938D939C93DF97045D1F4FB8E263
:10AFB000CB0ED11CE5E0EE16F10409F0B1CF7E0115
:10AFC000FDE2EF0EF11C28E2A22EB12C00EB1FEFE8
:10AFD00024E0220E311CD7012D913D914D915C91C1
:10AFE000139798966D917D918D919C919B970F945D
:10AFF00007A62B013C016101C01AD10A8824839461
:10B00000912CF601E00FF11FEA0DFB1D208131812B
:10B0100042815381C301B2010F94AD9E9B01AC01EB
:10B02000F60160817181828193810F9407A5D60119
:10B030006D937D938D939D936D01BFEF8B1A9B0A4A
:10B04000E6E08E169104E9F63CE2E30EF11C0852AC
:10B05000110988E2A80EB11C08339FEF190709F007
:10B06000BACF1E01F5EB2F0E311C6E0121EBC20E83
:10B07000D11C7E0137E3E31A3EEFF30A04E010E04F
:10B080004801B12CA12C412C512C3201F601EA0DC2
:10B09000FB1DD701AA0DBB1D2D913D914D915C91DA
:10B0A00060817181828193810F94AD9E9B01AC017F
:10B0B000C301B2010F9408A52B013C018FEF881A40
:10B0C000980A94E0A90EB11CA5E08A169104F1F645
:10B0D000A3019201F10160817181828193810F94BA
:10B0E00007A5D6012D913D914D915C910F9407A636
:10B0F000F701608371838283938301501109F8E221
:10B100002F1A31082CE2C21AD10834E0E31AF108F0
:10B110000115110509F0B4CFCB50DE4F888199811C
:10B12000AA81BB81C55FD140CF57DD4F888399830A
:10B13000AA83BB83C158D2401E0197E4291A9EEF0F
:10B14000390A10E000E0C159DD4FA881B981CF561E
:10B15000D240CD90DD90ED90FD90C159DD4FB98387
:10B16000A883CF56D240CB58DD4F288139814A8100
:10B170005B81C557D240C701B6010F94FDA51816D3
:10B18000B4F0CB58DD4F288139814A815B81C557A6
:10B19000D240C159DD4FE881F981CF56D24060815C
:10B1A0007181828193810F9491A787FF18C0043029
:10B1B000110509F030C1CB58DD4F288139814A8112
:10B1C0005B81C557D240CF57DD4F688179818A8135
:10B1D0009B81C158D2400F94FDA587FF1CC1D101AE
:10B1E00014968D909D90AD90BC9017978D919D91E8
:10B1F0000D90BC91A02DCF58DD4F88839983AA83F1
:10B20000BB83C157D240F801EE0FFF1FEE0FFF1FA7
:10B2100021E931E02C0F3D1FE20FF31F40805180E8
:10B2200062807380C359DD4FA881B981CD56D24069
:10B230008D919D910D90BC91A02DC358DD4F8883B9
:10B240009983AA83BB83CD57D240A7019601CB58DF
:10B25000DD4F688179818A819B81C557D2400F94E7
:10B2600007A56B017C0120E030E040E450E40F943E
:10B2700078A8CB57DD4F688379838A839B83C55831
:10B28000D240C358DD4F288139814A815B81CD5737
:10B29000D240C359DD4FE881F981CD56D240648157
:10B2A0007581868197810F9407A5A30192010F9460
:10B2B00007A6C758DD4F688379838A839B83C95764
:10B2C000D240A3019201C301B2010F9408A5CF5847
:10B2D000DD4F288139814A815B81C157D2400F946B
:10B2E000AD9EC757DD4F688379838A839B83C95896
:10B2F000D240A3019201C501B4010F94AD9E9B0100
:10B30000AC01C757DD4F688179818A819B81C9581B
:10B31000D2400F9408A520E030E040EC50E40F94B8
:10B3200007A69B01AC01C758DD4F688179818A81EE
:10B330009B81C957D2400F9407A5A70196010F948E
:10B34000AD9EC758DD4F688379838A839B83C95735
:10B35000D240CF58DD4F288139814A815B81C15766
:10B36000D240C501B4010F9407A54B015C0120E058
:10B3700030E040EC50E4C301B2010F94AD9E9B015C
:10B38000AC01C501B4010F9407A6CB57DD4F28814E
:10B3900039814A815B81C558D2400F94AD9E4B01E3
:10B3A0005C0120E030E040E05FE3CF58DD4F688192
:10B3B00079818A819B81C157D2400F94AD9E2B0128
:10B3C0003C01A7019601C701B6010F94AD9E9B01F8
:10B3D000AC01C301B2010F94AD9E9B01AC01C5014C
:10B3E000B4010F9408A59B01AC01C758DD4F6881DB
:10B3F00079818A819B81C957D2400F9408A5C3588F
:10B40000DD4F288139814A815B81CD57D2400F942D
:10B4100008A52B013C010F5F1F4FF4E02F0E311CDC
:10B42000C359DD4F28813981CD56D2402C5F3F4F23
:10B43000C359DD4F39832883CD56D24005301105DD
:10B4400009F081CEC301B201C457DD4F0FB6F894A5
:10B45000DEBF0FBECDBFDF91CF911F910F91FF9047
:10B46000EF90DF90CF90BF90AF909F908F907F90A4
:10B470006F905F904F903F902F900895C5010F946B
:10B48000EEA3D8018D939C93B5E0CB0ED11CE2E0E6
:10B49000AE0EB11C96CC0F931F93CF932091011346
:10B4A000213079F58C0180E50E94F555882349F11A
:10B4B0000E940A56C82F853020F5013C82E018070B
:10B4C00049F0023C124069F08C2FCF911F910F91EF
:10B4D0000D94899D60E08C2FCF911F910F910D9459
:10B4E000CC9D8EEC9EE00F94E0A3882351F00F9446
:10B4F000A679882331F08C2FCF911F910F910D9455
:10B50000499ECF911F910F9108958F929F92AF9274
:10B51000BF92CF92DF92EF92FF920F931F93CF9340
:10B52000DF930091BB041091BC040F5F1F4F6801B3
:10B530008FEFC81AD80AD801DC918D2F90E00F94B4
:10B5400071A17C01892B01F5DD3201F56801B2E0C2
:10B55000CB0ED11CF801D181C1E086010150110947
:10B5600043E050E064E876E7C8010F94A7A1892B77
:10B57000C1F460E070E080E89FEFC111DBC060E0E3
:10B5800070E080E89FE7D6C08601D1CFDB3239F486
:10B590006801F2E0CF0ED11CD8011196DC91C0E019
:10B5A000DCCF43E050E061E876E7C8010F94A7A143
:10B5B000892B09F4CCC0F60110E000E020E030E077
:10B5C000A9016F01D053DA3060F5BC2E6894B1F850
:10B5D0008C2F8870C2FF09C0811102C00F5F1F4FFE
:10B5E0003196D601DC91CB2DECCF882311F00150A0
:10B5F0001109A5E0B0E00F9475A49B01AC01220FE6
:10B60000331F441F551F2D0F311D411D511D28395A
:10B61000B9E93B074B07B9E15B0710F3C660BC2EE5
:10B62000DFCFDE3F31F4C3FD33C0BC2E6894B3F8E6
:10B63000D7CFD53369F580818D3231F4C061BF0138
:10B640006E5F7F4F818105C0BF018B32C9F36F5F91
:10B650007F4F80538A30E0F4FB01B0E8EB16BCE08A
:10B66000FB065CF4B701660F771F660F771FE60EC7
:10B67000F71EEE0CFF1CE80EF11C819180538A30FE
:10B6800060F3C4FF03C0F194E194F1080E0D1F1D97
:10B69000CA01B9010F946C9EC370C33009F490586D
:10B6A0004B015C0120E030E0A9010F94FDA5882347
:10B6B00009F43EC0CDE7D6E717FF05C01195019507
:10B6C0001109C5E6D6E76E01E8E1CE1AD10880E29D
:10B6D000E82EF12C0DC0FE01259135914591549134
:10B6E0000E191F09C501B4010F94AD9E4B015C01F9
:10B6F000D501C4010E151F0574F72497F594E7943E
:10B70000CC16DD06A9F78A2F880F8B2F881F8F3F55
:10B7100049F020E030E0A901C501B4010F94FDA576
:10B72000811106C082E290E090930C1780930B1772
:10B73000C501B401DF91CF911F910F91FF90EF9060
:10B74000DF90CF90BF90AF909F908F90089560E072
:10B7500070E080EC9FE7EECF2F923F924F925F9286
:10B760006F927F928F929F92AF92BF92CF92DF9211
:10B77000EF92FF920F931F93CF93DF93CDB7DEB776
:10B78000A1970FB6F894DEBF0FBECDBF84EC92E058
:10B790009D8F8C8F81E6282E82E1382E09E216E0FB
:10B7A00091E09A8F198EEC8DFD8D8191FD8FEC8F3C
:10B7B0000E94F555E82E882309F454C1F0905712E1
:10B7C000FA8DFF220E94855A2B013C01F80140822C
:10B7D000518262827382F98DF33009F045C0DD2415
:10B7E000D394F11001C0D12C8090100290901102DE
:10B7F000A0901202B090130220E030E040E85FE336
:10B80000C501B4010F94FDA5882359F1F11015C0AD
:10B8100020916D1230916E1240916F125091701202
:10B82000C301B2010F9407A56093350670933606E5
:10B830008093370690933806DE2CA5019401609121
:10B8400035067091360680913706909138060F9430
:10B85000AD9E6093350670933606809337069093BD
:10B860003806D11003C05FC0FF2089F0F1012081AC
:10B87000318142815381F80160817181828193819C
:10B880000F9408A5F8016083718382839383F98DF7
:10B89000F230D9F58091BB03823009F0EEC08CE024
:10B8A000E0EAF2E0DE011D9601900D928A95E1F743
:10B8B0008CE0ECEAF2E0DE01119601900D928A959F
:10B8C000E1F7C0903106D0903206E0903306F09058
:10B8D000340620E030E0A901C701B6010F94FDA5B0
:10B8E00087FF52C0CE0101967C01D12CF7016191F6
:10B8F0007191819191917F010F9479A68D2D0F9473
:10B900005E1AD394F3E0DF12F1CFF98DFF5FF98F68
:10B910008A8D880F8A8F94E0290E311C0C5F1F4F8F
:10B92000F43009F040CF86E40E94F555882399F061
:10B930000E94855A6B017C0120E030E0A9010F9440
:10B9400091A7181644F4C0927A02D0927B02E0923A
:10B950007C02F0927D02A1960FB6F894DEBF0FBE76
:10B96000CDBFDF91CF911F910F91FF90EF90DF90AE
:10B97000CF90BF90AF909F908F907F906F905F908F
:10B980004F903F902F90089520E030E048E453E43A
:10B99000C701B6010F9491A71816A4F4CE010D9615
:10B9A0007C01D12CF70161917191819191917F017D
:10B9B0000F9479A68D2D0F945E1AD394F3E0DF12C5
:10B9C000F1CFA3CFCE01019699A388A3FE013D96A6
:10B9D000FF8FEE8F1B8EE8A1F9A1C190D190E1906D
:10B9E000F190F9A3E8A3EE8DFF8D619171918191A2
:10B9F0009191FF8FEE8FA70196010F9407A520E08C
:10BA000030E048E453E40F9407A64B015C01209119
:10BA100031063091320640913306509134060F942E
:10BA2000AD9E2B013C0120E030E0A901C501B4012D
:10BA30000F94AD9E9B01AC01C701B6010F9407A501
:10BA40009B01AC01C301B2010F9408A50F9479A624
:10BA50008B8D0F945E1AFB8DFF5FFB8FF33009F027
:10BA6000BACF53CFF10180819181A281B381F801D6
:10BA700080839183A283B38348CFEA8DEE0FEA8F50
:10BA8000F4E02F0E311C0C5F1F4F83E0898F8BCEAB
:10BA9000609113177091141790E08A3020F0895A42
:10BAA0009F4F0D9448A2C096FCCF84FF18C05A9AAD
:10BAB00085FF17C0A49A2FB786FF15C0F894909100
:10BAC00002019068909302012FBF87FF11C0A39AD3
:10BAD0005B9A85E08A95F1F700005B9808955A9883
:10BAE000E7CFA498E8CFF894909102019F77EACF2E
:10BAF000A398EECF0F931F93CF93DF93C82FD62F2A
:10BB00008A0160FF15C05D9A8AE18A95F1F700C04D
:10BB10008C2F0E94555DD1FD04C08C2F82950E9410
:10BB2000555DC801DF91CF911F910F910C94DBD22D
:10BB30005D98EACFCF92DF92EF92FF92CF93DF939F
:10BB4000EC016A017B010F94E8A36F3F7F4F8F4F99
:10BB50009F4F59F4B701A601CE01DF91CF91FF901D
:10BB6000EF90DF90CF900D9436A4DF91CF91FF90AE
:10BB7000EF90DF90CF9008957F928F929F92AF9237
:10BB8000BF92CF92DF92EF92FF920F931F93CF93CA
:10BB9000DF93CDB7DEB760970FB6F894DEBF0FBE68
:10BBA000CDBF5C016B01742E81E0809378021F93FE
:10BBB0000F931F922F938DE893E69F938F930F948B
:10BBC000A2A281E40E94F5550F900F900F900F9064
:10BBD0000F900F90882389F08091BB049091BC0452
:10BBE000FC012181283709F056C040E150E070E0A7
:10BBF00060E002960F946B9F5B0183E40E94F55511
:10BC0000882309F44DC00E945D564B017501CA148A
:10BC1000DB0408F47601C4018E0D9F1DC816D906F9
:10BC200018F08E159F0518F446018E189F0888E5B8
:10BC30000E94F555882309F471C02091BB0430910E
:10BC4000BC042F5F3F4FCE0101965C01DC01D12C7B
:10BC5000C12CF90180812F5F3F4F8823B9F190E11A
:10BC6000C916D10499F18032A1F38A3079F190EDAF
:10BC7000980F9A30C8F48295807F9F012E5F3F4FC6
:10BC8000918140ED490F4A30B8F4842B8D93EFEF4A
:10BC9000CE1ADE0ADECF0E94855A0F9479A6ACCF69
:10BCA00088248A94982CB2CF9FE9980F963058F444
:10BCB0008295807F8057E1CF4FE9490F463018F4D5
:10BCC0009755892BE3CFD194C194D108912C812C25
:10BCD000C814D90491F0F50161915F01C4018E0D82
:10BCE0009F1DF1E07F1631F0FC016083FFEF8F1A9A
:10BCF0009F0AEECF0F9428A4F9CFFF92EF921F93E3
:10BD00000F939F928F9283E693E69F938F930F9466
:10BD1000A2A20FB6F894DEBF0FBECDBF472DB4016F
:10BD2000C70160960FB6F894DEBF0FBECDBFDF919E
:10BD3000CF911F910F91FF90EF90DF90CF90BF9028
:10BD4000AF909F908F907F900D94D2780F931F9318
:10BD5000CF93DF9300D01F92CDB7DEB79B01AC012C
:10BD600001E612E1F801608571858285938569831A
:10BD70007A838B839C830F9407A5F8016087718772
:10BD80008287938765E575E585E591E40F94814C9D
:10BD90000F94FB1A89819A81AB81BC81F80180875D
:10BDA0009187A287B387CE0101960F940C3D0F9027
:10BDB0000F900F900F90DF91CF911F910F910895E9
:10BDC000682F70E090E080E00F946C9E20E030E0FF
:10BDD00048E052E40F94AD9E20E030E040E85FE39D
:10BDE0000F9408A5089582E00F94E71A60936912F2
:10BDF00070936A1280936B1290936C1289E692E1B1
:10BE00000D940C3D4F925F926F927F928F929F9212
:10BE1000AF92BF92CF92DF92EF92FF920F931F9358
:10BE2000CF93DF9301E612E1CAE9D4E0288139819A
:10BE30004A815B81F80160817181828193810F94D5
:10BE400007A54B015C012C813D814E815F81F8018A
:10BE500064817581868197810F9407A56B017C01B0
:10BE6000CAE8D4E0288139814A815B81C501B401E7
:10BE70000F94AD9E2B013C012C813D814E815F8151
:10BE8000C701B6010F94AD9E9B01AC01C301B20185
:10BE90000F9408A5F80160837183828393832885BA
:10BEA00039854A855B85C501B4010F94AD9E4B0170
:10BEB0005C012C853D854E855F85C701B6010F94D9
:10BEC000AD9E9B01AC01C501B4010F9408A5F8011A
:10BED0006483758386839783DF91CF911F910F9140
:10BEE000FF90EF90DF90CF90BF90AF909F908F909A
:10BEF0007F906F905F904F9008954F925F926F92F6
:10BF00007F928F929F92AF92BF92CF92DF92EF92E9
:10BF1000FF920F931F93CF93DF9300D000D01F9217
:10BF20001F92CDB7DEB7DC01CD90DD90ED90FC9097
:10BF30001397C0926F03D0927003E0927103F09256
:10BF4000720314960D911D912D913C9117970983C1
:10BF50001A832B833C8300937703109378032093F9
:10BF6000790330937A03DB010D911D912D913C9162
:10BF700013970D831E832F833887009373031093C9
:10BF80007403209375033093760314964D905D905F
:10BF90006D907C90179740927B0350927C03609247
:10BFA0007D0370927E03FA016081718182819381A9
:10BFB00060939A0470939B0480939C0490939D04D7
:10BFC00084809580A680B78080929E0490929F0482
:10BFD000A092A004B092A10420E030E0A9010F9447
:10BFE000FDA58111AAC020E030E0A901C501B4017E
:10BFF0000F94FDA58111A1C01092A20420E030E0B1
:10C0000040E85FE3C701B6010F94FDA5811121C08F
:10C0100020E030E0A9016D817E818F8198850F94A9
:10C02000FDA5811116C020E030E0A90169817A8167
:10C030008B819C810F94FDA581110BC020E030E025
:10C0400040E85FE3C301B2010F94FDA5882309F422
:10C0500078C08091A20482608093A204A30192011F
:10C06000C701B6010F94AD9E4B015C012D813E814D
:10C070004F81588569817A818B819C810F94AD9E17
:10C080009B01AC01C501B4010F9407A54B015C01F4
:10C09000AC019B01C301B2010F9407A660938A040F
:10C0A00070938B0480938C0490938D046D817E81BA
:10C0B0008F8198859058A50194010F9407A66093ED
:10C0C0008E0470938F0480939004909391046981FF
:10C0D0007A818B819C819058A50194010F9407A6C9
:10C0E00060939204709393048093940490939504C6
:10C0F000A5019401C701B6010F9407A660939604A9
:10C1000070939704809398049093990428960FB69F
:10C11000F894DEBF0FBECDBFDF91CF911F910F917D
:10C12000FF90EF90DF90CF90BF90AF909F908F9057
:10C130007F906F905F904F90089581E08093A2046C
:10C140005DCF80E090E0A0E8BFE380938A04909305
:10C150008B04A0938C04B0938D0410928E041092E3
:10C160008F041092900410929104109292041092F5
:10C1700093041092940410929504809396049093E3
:10C180009704A0939804B0939904C0CF4F925F9204
:10C190006F927F928F929F92AF92BF92CF92DF92D7
:10C1A000EF92FF921F93CF93DF93CDB7DEB7A8979F
:10C1B0000FB6F894DEBF0FBECDBF48E050E06DED86
:10C1C0007FE0CE0101960F94D0A348E050E065EDEA
:10C1D0007FE0CE0109960F94D0A348E050E065EED1
:10C1E0007FE0CE0141960F94D0A389899A89AB89CB
:10C1F000BC8989A39AA3ABA3BCA38F3F9F4FAF4F2A
:10C20000BF4F09F4B1C08D899E89AF89B88D8DA3C8
:10C210009EA3AFA3B8A78F3F9F4FAF4FBF4F09F467
:10C22000A3C089809A80AB80BC808FEF8816980667
:10C23000A806B80609F498C08D819E81AF81B885A3
:10C24000898F9A8FAB8FBC8F8F3F9F4FAF4FBF4F60
:10C2500009F48AC0C984DA84EB84FC848FEFC816A1
:10C26000D806E806F80609F47FC08D859E85AF855F
:10C27000B8898D8F9E8FAF8FB8A38F3F9F4FAF4FE1
:10C28000BF4F09F471C0298D3A8D4B8D5C8DC5016E
:10C29000B4010F94A4A72B013C0126E636E646E63E
:10C2A0005FE30F94FDA511E087FD0BC02DEC3CEC86
:10C2B0004CE85FE3C301B2010F9491A718160CF08C
:10C2C00010E02D8D3E8D4F8D58A1C701B6010F9402
:10C2D000A4A72B013C0126E636E646E65FE30F9471
:10C2E000FDA587FD7FC02DEC3CEC4CE85FE3C3016E
:10C2F000B2010F9491A718160CF474C02DA13EA1A1
:10C300004FA158A569A17AA18BA19CA10F94A4A7C4
:10C3100020E030E040E751E40F9491A718160CF4A8
:10C3200011E0A5019401C701B6010F94AD9E6B0108
:10C330007C012D8D3E8D4F8D58A1698D7A8D8B8D11
:10C340009C8D0F94AD9E9B01AC01C701B6010F946B
:10C3500008A59F772DEC3CEC4CEC5DE30F9491A786
:10C36000181614F01123F1F00E941E5580E090E0A1
:10C37000A0E8BFE389839A83AB83BC831D821E82BE
:10C380001F82188619861A861B861C868D879E87B3
:10C39000AF87B88B198A1A8A1B8A1C8A1D8A1E8A43
:10C3A0001F8A188EAE014F5E5F4FBE01675F7F4FE1
:10C3B000CE0101960E947D5FA8960FB6F894DEBF6D
:10C3C0000FBECDBFDF91CF911F91FF90EF90DF9017
:10C3D000CF90BF90AF909F908F907F906F905F9025
:10C3E0004F90089511E08ACFCF93DF93CDB7DEB79A
:10C3F00068970FB6F894DEBF0FBECDBF80E090E027
:10C40000A0E8BFE389839A83AB83BC831D821E822D
:10C410001F82188619861A861B861C868D879E8722
:10C42000AF87B88B198A1A8A1B8A1C8A1D8A1E8AB2
:10C430001F8A188EAE014F5E5F4FBE01675F7F4F50
:10C44000CE0101960E947D5F68960FB6F894DEBF1C
:10C450000FBECDBFDF91CF9108958091A2048823B4
:10C46000D1F00E94F4610F94FB1A80E00F94E71A58
:10C4700060936112709362128093631290936412BE
:10C4800081E00F94E71A60936512709366128093AF
:10C4900067129093681208958091630490916204EA
:10C4A00089130BC090916104992339F020911E06E5
:10C4B00030911F068217130639F081E09091C40372
:10C4C000911103C080E0089581E0089520916304F4
:10C4D00080911E0690911F062817190611F080E220
:10C4E00008958EE3089582E0809359028091630459
:10C4F0008F5F8093630484E08093600410926204F1
:10C5000010926104089580916004843038F5809120
:10C51000630490E020911E0630911F06281739070A
:10C5200044F0019790931F0680931E0687E00F94B6
:10C53000AD2580911E062091920330E02D5F3F4F84
:10C540008217130659F054F09DEF980F90939203C1
:10C550008450809362048FEF809360040895E6E92D
:10C56000F3E080E2DF011D928A95E9F70895CF9309
:10C570003FB7F894E0910204F0910304E817F9073B
:10C58000C9F0C42F909303048093020470931F0694
:10C5900060931E061092920382E0809359023FBF7F
:10C5A000222319F080E00F94AD25CC2321F0CF9108
:10C5B0000C94AF623FBFCF910895DC01262F90917C
:10C5C000DF039730D8F4492F50E0FA01EE0FFF1F38
:10C5D000E40FF51FE95AFC4F409102045091030407
:10C5E0005183408380911E069F5F9093DF03828377
:10C5F00041E070E060E0CD010C94B7620895982F9F
:10C600008091DF039817A8F4891B8093DF0390E0E3
:10C61000FC01EE0FFF1FE80FF91FE95AFC4F628182
:10C62000062E000C770B20E041E0808191810C9474
:10C63000B76280E0EACF81E00C94FF621F920F9214
:10C640000FB60F9211240BB60F922F933F934F9377
:10C650006F937F938F939F93EF93FF938091C80085
:10C6600084FF12C08091CE00FF91EF919F918F9136
:10C670007F916F914F913F912F910F900BBE0F9033
:10C680000FBE0F901F9018954091CE0080911C0610
:10C69000813051F72091420530914305C90101963F
:10C6A0008F77992760914405709145058617970704
:10C6B000D9F22E533B4FF901408390934305809369
:10C6C0004205D2CF1F920F920FB60F9211240BB6D4
:10C6D0000F922F933F934F936F937F938F939F93DB
:10C6E000EF93FF938091C00084FF12C08091C60039
:10C6F000FF91EF919F918F917F916F914F913F911A
:10C700002F910F900BBE0F900FBE0F901F9018959A
:10C710004091C60080911C068111EACF209142050C
:10C7200030914305C90101968F779927609144059F
:10C730007091450586179707D9F22E533B4FF901A3
:10C7400040839093430580934205D2CF80E1E1E698
:10C75000F2E1A0E9B2E001900D928A95E1F78091B3
:10C760008E0290918F029093601280935F1280915D
:10C770005D1290915E1290935C1280935B12809197
:10C780005912809358128091571283FB882780F9A1
:10C790008093561280915512809354120895CF932E
:10C7A000DF9387E696E10E94AB7985EA94E1892BD5
:10C7B00051F0C7E7D5E1A397CE010E94AB7984E1A0
:10C7C000C53AD807C1F782E894E10E94AB798DE5BC
:10C7D00094E1DF91CF910C94AB79CF93DF93C1E6D5
:10C7E000D2E120E030E048EC51E46C857D858E8517
:10C7F0009F850F9408A56C877D878E879F8763E34D
:10C8000073E383E590E4DF91CF910D94814C60E078
:10C8100085EA9FE00F9404A460E08FE79CE00F940A
:10C8200004A480E090E0A0E8BFEB80937E029093A8
:10C830007F02A0938002B093810282E0809379020C
:10C8400010927312089580915B1290915C12209166
:10C850005D1230915E122817390771F090935E12C5
:10C8600080935D1281E08093CB030F94F00D0F94C1
:10C87000857482E08093CB0308958091731288239E
:10C8800041F080918E0290918F029093601280937C
:10C890005F120895CF92DF92EF92FF92C090FF0D4A
:10C8A000D090000EE090010EF090020E8091FE0DEF
:10C8B000882309F44EC020E030E0A901C701B60189
:10C8C0000F9491A718160CF044C02BED3FE049E4FB
:10C8D00050E4C701B6010F94AD9EA70196010F94D5
:10C8E000AD9E20E030E040E85EE30F94AD9E9B01FA
:10C8F000AC0160E070E080E89FE30F9407A66B0155
:10C900007C01609175027091760264367105A1F028
:10C91000072E000C880B990B0F946E9E2AE037EDC2
:10C9200043E25CE30F94AD9E9B01AC01C701B601ED
:10C930000F94AD9E6B017C01C0921002D092110247
:10C94000E0921202F0921302FF90EF90DF90CF90EE
:10C950000895C12CD12C80E8E82E8FE3F82ED1CF9A
:10C960008F929F92AF92BF92CF92DF92EF92FF92FF
:10C9700081EF9FE00F94D86C6B017C018DEE9FE0FE
:10C980000F94D86C4B015C010F946D172CE330E0D1
:10C9900040E050E00F9453A4BA01A901480D591D7D
:10C9A0006A1D7B1D8DEE9FE00F9416A46091170603
:10C9B000709118068091190690911A0628EE33E0BE
:10C9C00040E050E00F9453A4BA01A9014C0D5D1D45
:10C9D0006E1D7F1D81EF9FE00F9416A40F940A191E
:10C9E00010921706109218061092190610921A0645
:10C9F00080910113813081F46091051370910613C9
:10CA000090E080E00F94C06C109206131092051312
:10CA10001092081310920713FF90EF90DF90CF90C1
:10CA2000BF90AF909F908F900895809155121F9264
:10CA30008F9380913E031F928F93E7EBF3E0428147
:10CA400053812CE3249FC001259F900D11249F93B7
:10CA50008F9340815181249FC001259F900D112407
:10CA60009F938F9384E294E69F938F930F94A2A257
:10CA70008DB79EB70A960FB6F8949EBF0FBE8DBFB6
:10CA8000089588E493E00D94471020E030E040E7FB
:10CA900052E40F9407A6089510927702409139034B
:10CAA00050913A0360913B0370913C0340937A02AA
:10CAB00050937B0260937C0270937D0290938F026F
:10CAC00080938E0288E493E00D9447101F93CF93D8
:10CAD000DF93182F80917A0290917B02A0917C02C3
:10CAE000B0917D028093390390933A03A0933B0366
:10CAF000B0933C03C0918E02D0918F0284E690E007
:10CB000090938F0280938E0288E493E00F944710F5
:10CB100010937702CE01DF91CF911F910895CF92AC
:10CB2000DF92EF92FF920F931F93CF93DF9390E0EA
:10CB3000EC01CC0FDD1FCC0FDD1FFE01E156F948E3
:10CB40002591359145915491FE01E154F24FC080F9
:10CB5000D180E280F3808E010F591D4EC701B601CE
:10CB60000F9408A5F8016083718382839383FE018B
:10CB7000ED56F94825913591459154918E010C5D02
:10CB80001D4FC701B6010F9408A5F801608371839A
:10CB900082839383FE01E957F948259135914591A8
:10CBA0005491C85EDD4FC701B6010F9408A5688394
:10CBB00079838A839B83DF91CF911F910F91FF909F
:10CBC000EF90DF90CF90089540E050E0BA018DEEF5
:10CBD0009FE00F9416A440E050E0BA0181EF9FE07F
:10CBE0000F9416A40E94685670E060E085E09FE014
:10CBF0000F9422A470E060E083E09FE00F9422A4F1
:10CC000070E060E081E09FE00F9422A470E060E0BB
:10CC10008FEF9EE00F9422A470E060E083ED9EE031
:10CC20000F9422A470E060E080ED9EE00F9422A4B7
:10CC300040E050E0BA0188EA9CE00D9416A4F89414
:10CC400088E19FE00FB6F894A895809360000FBE2E
:10CC500090936000FFCF85EA9FE00F94E0A391E0FE
:10CC6000811101C090E0892F08958091CD03811139
:10CC700006C081E090918B03923009F080E0089526
:10CC80008091D71381110AC080914212811106C090
:10CC900081E090918B03913009F080E00895CF936B
:10CCA000DF93C0917112C1111FC080917212811166
:10CCB0001CC00E943566811118C0D0915E0DD43021
:10CCC00061F480915D1290915E12892B91F48091B4
:10CCD000591290915A12892B61F40E944066C82F14
:10CCE000811103C0C1E0D111C0E08C2FDF91CF9141
:10CCF0000895C1E0FACF0E944F66882389F020E0B2
:10CD000030E040E050E46091691270916A128091C5
:10CD10006B1290916C120F94FDA5881F8827881FB5
:10CD200008950E944066811118C00E9435668111E5
:10CD300014C080917312811110C080915E0D811119
:10CD40000BC080910213811107C080917112811173
:10CD500004C080917212089581E0089580E1E1E6B7
:10CD6000F2E1A9E2B6E001900D928A95E1F708950B
:10CD70004F925F926F927F928F929F92AF92BF92EB
:10CD8000CF92DF92EF92FF920F931F93CF93DF9397
:10CD900000D000D01F921F92CDB7DEB72091731242
:10CDA000222309F473C12091CE03223009F46EC10D
:10CDB0002091CE03213011F41092CE032B013C01BF
:10CDC00010925512109158126091BC037091BD03DE
:10CDD0008091BE039091BF030F9480A6611731F03C
:10CDE000812F90E090935A12809359120E942364ED
:10CDF000809154128093551290915712809156123F
:10CE0000819589278870892780935712A301920101
:10CE100060919C0270919D0280919E0290919F0270
:10CE20000F9407A56D837E838F839887CE01059627
:10CE30000F94D93C1092400220E030E040E85FEBD4
:10CE40006091900270919102809192029091930270
:10CE50000F94FDA5811120C0809161129091621202
:10CE6000A0916312B091641280939002909391020A
:10CE7000A0939202B09393028091651290916612F2
:10CE8000A0916712B09168128093940290939502DA
:10CE9000A0939602B0939702A301920160919C0225
:10CEA00070919D0280919E0290919F020F9407A520
:10CEB00069837A838B839C83E0906912F0906A1275
:10CEC00000916B1210916C12209194023091950296
:10CED0004091960250919702609190027091910258
:10CEE00080919202909193021F921F921F921F9223
:10CEF000E2E68E2EE7E29E2EE6E7AE2EE2E4BE2EBE
:10CF0000FE0131966F010F94333DA30192016091B0
:10CF10009C0270919D0280919E0290919F020F94BD
:10CF200007A569837A838B839C83E0909802F090B5
:10CF3000990200919A0210919B02209194023091E3
:10CF400095024091960250919702609190027091E3
:10CF5000910280919202909193021F921F921F92D0
:10CF60001F920F94333DE0909802F0909902009147
:10CF70009A0210919B022091940230919502409167
:10CF80009602509197026091900270919102809167
:10CF90009202909193021F921F921F921F92812CD6
:10CFA000912CF8EEAF2EF2E4BF2EACE9CA2EA2E02F
:10CFB000DA2E0F94333D0F94FB1A11E010934002C8
:10CFC00060914F127091501290E080E00F946C9E2F
:10CFD00060937A0270937B0280937C0290937D022F
:10CFE00080915F129091601290938F0280938E02D5
:10CFF00080E1E0E9F2E0A1E6B2E101900D928A95CC
:10D00000E1F70E94AE66809179020FB6F894DEBF18
:10D010000FBECDBF811151C0609145127091461273
:10D0200080914712909148126093EB167093EC1622
:10D030008093ED169093EE160F9417688091451229
:10D0400090914612A0914712B091481280934912D4
:10D0500090934A12A0934B12B0934C121093D71393
:10D0600060E085EA9FE00F9404A460E08FE79CE015
:10D070000F9404A486EE9BE60E9494DE82E08093E7
:10D0800079021092731281E08093420D28960FB6B8
:10D09000F894DEBF0FBECDBFDF91CF911F910F91EE
:10D0A000FF90EF90DF90CF90BF90AF909F908F90C8
:10D0B0007F906F905F904F900895813089F68091B6
:10D0C000451290914612A0914712B0914812809358
:10D0D0003E1290933F12A0934012B09341121092CF
:10D0E0004810109247100E94AC55BACF3F924F9211
:10D0F0005F926F927F928F929F92AF92BF92CF92E8
:10D10000DF92EF92FF920F931F93CF93DF933090B4
:10D11000A204332009F480C08B01EC0131FE54C01D
:10D1200088809980AA80BB80FB01C080D180E2808A
:10D13000F3802091770330917803409179035091E7
:10D140007A03C501B4010F94AD9E2B013C012091DF
:10D150007B0330917C0340917D0350917E03C70196
:10D16000B6010F94AD9E9B01AC01C301B2010F94B7
:10D1700008A52B013C0120916F0330917003409171
:10D18000710350917203C501B4010F94AD9E4B0120
:10D190005C012091730330917403409175035091A9
:10D1A0007603C701B6010F94AD9E9B01AC01C5018A
:10D1B000B4010F9408A5688379838A839B83F8015F
:10D1C000408251826282738230FE26C020919A048E
:10D1D00030919B0440919C0450919D046881798119
:10D1E0008A819B810F9408A5688379838A839B83B6
:10D1F00020919E0430919F044091A0045091A1047D
:10D20000F80160817181828193810F9408A5F801F2
:10D210006083718382839383DF91CF911F910F91FC
:10D22000FF90EF90DF90CF90BF90AF909F908F9046
:10D230007F906F905F904F903F9008952F923F9214
:10D240004F925F926F927F928F929F92AF92BF9216
:10D25000CF92DF92EF92FF920F931F93CF93DF93C2
:10D2600000D000D01F921F92CDB7DEB78C011B01FA
:10D27000FC0180819181A281B38189839A83AB83F0
:10D28000BC83FB0180819181A281B3818D839E83C8
:10D29000AF83B887BE016B5F7F4FCE0101960E94BE
:10D2A0007668C980DA80EB80FC8020E030E0A9015C
:10D2B000C701B6010F94FDA587FF35C019821A82F8
:10D2C0001B821C82FF24F3948D809E80AF80B884E3
:10D2D00020E030E040E850ECC501B4010F94FDA51A
:10D2E00087FF35C080E090E0A0E8B0EC8D839E839E
:10D2F000AF83B887CD80DE80EF80F88489809A8004
:10D30000AB80BC807090A20471104CC0F801808288
:10D310009182A282B382F101C082D182E282F38241
:10D32000FF24F39425C020E030E04AE753E4C7012E
:10D33000B6010F9491A7F12C181634F680E090E016
:10D34000AAE7B3E489839A83AB83BC83BBCF20E095
:10D3500030E042E553E4C501B4010F9491A71816DB
:10D360002CF480E090E0A2E5B3E4C0CFF110C2CF8E
:10D370008F2D28960FB6F894DEBF0FBECDBFDF917C
:10D38000CF911F910F91FF90EF90DF90CF90BF90C2
:10D39000AF909F908F907F906F905F904F903F9055
:10D3A0002F90089570FE1CC020919A0430919B0428
:10D3B00040919C0450919D04C501B4010F9407A5B0
:10D3C0004B015C0120919E0430919F044091A00488
:10D3D0005091A104C701B6010F9407A56B017C0110
:10D3E00071FE9ECF20918A0430918B0440918C0471
:10D3F00050918D04C501B4010F94AD9E2B013C01E9
:10D4000020918E0430918F044091900450919104AA
:10D41000C701B6010F94AD9E9B01AC01C301B201DF
:10D420000F9408A5F8016083718382839383209110
:10D430009204309193044091940450919504C50155
:10D44000B4010F94AD9E4B015C0120919604309184
:10D4500097044091980450919904C701B6010F9424
:10D46000AD9E9B01AC01C501B4010F9408A5F1016B
:10D47000608371838283938353CFCF93DF930E9422
:10D480004165C1E6D2E180E090E0A0EAB0E488879F
:10D490009987AA87BB8765E575E585E591E40F94D3
:10D4A000F6508DEC9CECACE4BEE388839983AA83B0
:10D4B000BB8383E393E3A3E7B0EC8C839D83AE83CC
:10D4C000BF8365E672E1CE010E941E6960E070E0F4
:10D4D00086E193E40F94F6508AE999E9A9E1BEE365
:10D4E00088879987AA87BB8765E575E585E591E417
:10D4F000DF91CF910D94F650CF92DF92EF92FF9291
:10D50000CF93DF93EC01BC016C5F7F4F0E941E69DB
:10D51000C0902C02D0902D02E0902E02F0902F02AD
:10D52000A7019601688579858A859B850F94FDA55D
:10D5300087FF04C0C886D986EA86FB86C090200291
:10D54000D0902102E0902202F0902302A7019601E0
:10D55000688579858A859B850F9491A7181624F490
:10D56000C886D986EA86FB86DF91CF91FF90EF903F
:10D57000DF90CF9008952F923F924F925F926F92DB
:10D580007F928F929F92AF92BF92CF92DF92EF9253
:10D59000FF920F931F93CF93DF93CDB7DEB7A29780
:10D5A0000FB6F894DEBF0FBECDBF1C0189E296E036
:10D5B0000E947C6A88E493E00F94471040906112C7
:10D5C000509062126090631270906412C0902906AD
:10D5D000D0902A06E0902B06F0902C06A701960129
:10D5E000C301B2010F94FDA581113FC020912D060A
:10D5F00030912E0640912F065091300660916512B1
:10D600007091661280916712909168120F94FDA537
:10D6100081112BC020E030E040E752E460917A02B3
:10D6200070917B0280917C0290917D020F9407A6FD
:10D630000F944E4C0E94E854A2960FB6F894DEBFA9
:10D640000FBECDBFDF91CF911F910F91FF90EF9053
:10D65000DF90CF90BF90AF909F908F907F906F9012
:10D660005F904F903F902F90089560918E0270913F
:10D670008F02072E000C880B990B0F946E9E209141
:10D680007A0230917B0240917C0250917D020F948E
:10D69000AD9E2EE333EC4EE259E30F94AD9E6F83C3
:10D6A000788789879A8780910913882309F40FC1A5
:10D6B000A3019201C701B6010F9407A52B013C01FC
:10D6C0002091651230916612409167125091681254
:10D6D00060912D0670912E0680912F069091300654
:10D6E0000F9407A56B877C878D879E87C301B20146
:10D6F0009F772B853C854D855E855F770F9408A5C8
:10D700006B017C0120E030E0A9010F9491A718166D
:10D710000CF0DDC020E030E040EF51E4C701B6017D
:10D720000F9407A60F94E6A50F9480A67E836D83C1
:10D730006230710508F4CBC02114310409F4C7C06C
:10D740002091691230916A1240916B1250916C12C3
:10D7500060913106709132068091330690913406C3
:10D760000F9407A56F87788B898B9A8B20916D1208
:10D7700030916E1240916F12509170126091350687
:10D780007091360680913706909138060F9407A560
:10D790006B8B7C8B8D8B9E8BAD81BE81CD01B0E080
:10D7A000A0E08F8F98A3A9A3BAA32D813E81221652
:10D7B000330608F08CC0B10190E080E00F946C9EBD
:10D7C0006B017C016F8D78A189A19AA10F946C9E49
:10D7D0009B01AC01C701B6010F9407A66B017C0148
:10D7E000AC019B016B897C898D899E890F94AD9ECC
:10D7F0009B01AC0160916D1270916E1280916F125D
:10D80000909170120F9408A569837A838B839C830F
:10D81000A70196016F85788989899A890F94AD9EB1
:10D820002091691230916A1240916B1250916C12E2
:10D830000F9408A56F8B788F898F9A8FA701960117
:10D840006B857C858D859E850F94AD9E209165129C
:10D850003091661240916712509168120F9408A59A
:10D860006B8F7C8F8D8F9E8FA7019601C301B201B4
:10D870000F94AD9E2091611230916212409163121B
:10D88000509164120F9408A53F922F92A1E6B2E145
:10D89000BF93AF938F809884A984BA84DE011196D8
:10D8A0006D01EF88F88C098D1A8D2B8D3C8D4D8D77
:10D8B0005E8D0F94333D0F900F900F900F908091DD
:10D8C000420D8111B7CEBFEF2B1A3B0A6ECFE0900D
:10D8D0003106F09032060091330610913406209103
:10D8E0002D0630912E0640912F0650913006609102
:10D8F000290670912A0680912B0690912C061F9282
:10D900001F92E1E6F2E1FF93EF938F809884A98460
:10D91000BA84E5E3CE2EE6E0DE2E0F94333D0F9081
:10D920000F900F900F9086CECF92DF92EF92FF92E2
:10D93000CF93C0906912D0906A12E0906B12F09071
:10D940006C12A70196010F9408A560936912709359
:10D950006A1280936B1290936C1283B190913B0684
:10D96000911102C084FF26C081E692E10E947C6A88
:10D970006091830D7091840D8091850D9091860D3D
:10D980000F94814C0F94FB1AA701960160916912C4
:10D9900070916A1280916B1290916C120F9407A58E
:10D9A0006B017C01C701B601CF91FF90EF90DF9032
:10D9B000CF90089515980F94FB1A81E00F94882555
:10D9C000C82F65E575E585E591E40F94814C0F94CA
:10D9D000FB1A82E00F94E71AA70196010F9407A59E
:10D9E0006B017C018C2F0F948825DCCF8F929F9246
:10D9F000AF92BF92CF92DF92EF92FF924B015C0108
:10DA0000C0906912D0906A12E0906B12F0906C1284
:10DA1000AC019B01C701B6010F9491A787FF11C00C
:10DA2000A5019401C701B6010F9407A59F77FF9048
:10DA3000EF90DF90CF90BF90AF909F908F900C941D
:10DA4000946CFF90EF90DF90CF90BF90AF909F903D
:10DA50008F9008952F923F924F925F926F927F9294
:10DA60008F929F92AF92BF92CF92DF92EF92FF92EE
:10DA70000F931F93CF93DF9300D01F921F92CDB7C8
:10DA8000DEB7D82E2A013B01322EE982FA820B83BF
:10DA90001C830F94FB1A81E080937112FC2CE32C01
:10DAA000D31010C0ED2CDC100DC060E070E080EAF7
:10DAB00090E40E94F66CFF24F394EE24E394222475
:10DAC000239401C02D2C0E942D62809109138D8317
:10DAD0001092091382E00F94E71A60936912709311
:10DAE0006A1280936B1290936C12F1100F94AA54E7
:10DAF00081E00E9466658C010E94AE6610927A02F7
:10DB000010927B0210927C0210927D02222019F06A
:10DB100080E00F94AE79EE2019F081E00F94AE7999
:10DB2000DD20E9F04114510461047104C1F0C30126
:10DB3000B2010F946E9E9B01AC016091BF0D70917C
:10DB4000C00D8091C10D9091C20D0F9408A56093F6
:10DB50006112709362128093631290936412332067
:10DB600001F189819A81AB81BC810097A105B10542
:10DB7000C1F0BC01CD010F946E9E9B01AC01609180
:10DB8000C30D7091C40D8091C50D9091C60D0F9479
:10DB900008A5609365127093661280936712909344
:10DBA0006812FF2009F499C060E070E080EA90E418
:10DBB0000E94F66C80913906811102C00F94AE79F3
:10DBC00080913A06811103C081E00F94AE790E94E2
:10DBD000C660E4E0FCE985919591A591B491E0E0FF
:10DBE000FCE94591559165917491409329065093B4
:10DBF0002A0660932B0670932C0680932D06909333
:10DC00002E06A0932F06B09330066DE276E089E2EF
:10DC100096E00E9476680E94F46120E030E040E8DF
:10DC200050EC60912D0670912E0680912F069091F8
:10DC300030060F94FDA587FF0CC080E090E0A0E8BF
:10DC4000B0EC80932D0690932E06A0932F06B093F0
:10DC5000300680E090E0A6E1B3E480937A029093EE
:10DC60007B02A0937C02B0937D02109277020F9406
:10DC7000414B60917A0270917B0280917C0290917D
:10DC80007D020F944E4C0F94FB1A809129069091BF
:10DC90002A06A0912B06B0912C06809361129093D6
:10DCA0006212A0936312B093641280912D0690913A
:10DCB0002E06A0912F06B0913006809365129093A6
:10DCC0006612A0936712B093681281E08093770286
:10DCD0000F94A42582E00F94AE79CC20E9F0811452
:10DCE0009104A104B104C1F0C501B4010F946E9E6A
:10DCF0009B01AC016091C70D7091C80D8091C90D59
:10DD00009091CA0D0F9408A56093691270936A12DE
:10DD100080936B1290936C120F94414BC8010E9438
:10DD20004C650F94A4250E94C6600E94025FD1102A
:10DD300007C0311005C08B8D811102C0CC2039F194
:10DD4000F11025C09D81992311F181E08093091381
:10DD50000F94E71A6B017C0180E00F94E71AA7018A
:10DD600096010F9478919B01AC01609169127091BA
:10DD70006A1280916B1290916C120F9407A56093B8
:10DD8000691270936A1280936B1290936C1284E103
:10DD90000F9479320F94FB1A109271120F900F901A
:10DDA0000F900F900F90DF91CF911F910F91FF90E7
:10DDB000EF90DF90CF90BF90AF909F908F907F902B
:10DDC0006F905F904F903F902F900895E1E3F3E0C4
:10DDD0009FE781918F3731F0DF01119787FF07C0EF
:10DDE0008F778C9383E0E933F80799F708959C9334
:10DDF000F9CF90915902981710F4809359028091AD
:10DE00005A02882339F0E0910404F0910504309718
:10DE100009F019940895CF93DF93CDB7DEB7AE0123
:10DE20004A5F5F4FFA0161917191AF0182EF93E018
:10DE30000F9427A3DF91CF91089562EF73E00D94C3
:10DE400078A262EF73E0082E000C990B0D9448A2A3
:10DE5000CF93C82FC15020F080E20E94216FFACFEB
:10DE6000CF9108950F931F93CF93DF93EB01142F5E
:10DE7000052F0E94216FCE010E941D6F8AE30E9430
:10DE8000216FCE010F949EA19EE0981B892F0E94C6
:10DE9000286F0F931F9383E691E89F938F930E94BF
:10DEA0000B6F0F900F900F900F90DF91CF911F91FC
:10DEB0000F910895CF93C82F862F643008F083E028
:10DEC000809330030E94F2548C0F80932F0344E61A
:10DED00050E060E08068CF910C947A5D7F928F92E1
:10DEE0009F92AF92BF92CF92DF92EF92FF920F93E9
:10DEF0001F93CF93DF93E091630450916204E51385
:10DF000073C0FB01483009F06CC0C081D0E049010A
:10DF1000742E6B015C0180915902882359F0609145
:10DF2000600480E00E945A6F0E946662AE01B501F3
:10DF30000E94326F80916104882309F455C090914A
:10DF4000630420911E0630911F069217130609F0F4
:10DF50004BC08091DF038730D8F4282F30E0F901DF
:10DF6000EE0FFF1FE20FF31FE95AFC4F209102044E
:10DF700030910304318320838F5F8093DF0392838A
:10DF800020E040E070E060E082E893E70E94B76242
:10DF9000B0929703A0929603D0929A03C0929903ED
:10DFA00070929803D0939C03C0939B0390929E031E
:10DFB00080929D031093A00300939F03F092A2030D
:10DFC000E092A103DF91CF911F910F91FF90EF900D
:10DFD000DF90CF90BF90AF909F908F907F900C94E8
:10DFE0007362C081D18193CF809163048F5F8093EE
:10DFF0006304DF91CF911F910F91FF90EF90DF901D
:10E00000CF90BF90AF909F908F907F900895CF93C7
:10E01000DF93EA010E945A6F62EF73E0CE01DF9155
:10E02000CF910D9478A2CF93C42F0E945A6F62EFC4
:10E0300073E08C2FCC0F990BCF910D9448A260E028
:10E0400080E00E945A6F10922F03089540E456E03A
:10E0500060E081E00E947A5D1092300310922F03FD
:10E0600048E050E06FE770E081E393E00D9412AA7E
:10E0700090915A02981709F180935A028823E9F087
:10E0800010921F0610921E061092A40583EE93E0D4
:10E090000F9447100F94F00D615071098109910997
:10E0A0006093C5037093C6038093C7039093C8031E
:10E0B0000E94267082E00C94F96E0895CF93C82FC9
:10E0C0001092300310922F0348E050E06FE770E0A9
:10E0D00081E393E00F9412AA44E951E162E080E306
:10E0E0000E947A5D46E950E062E080E30E947A5D3A
:10E0F00046E950E062E080E30E947A5D46E950E044
:10E1000062E080E20E947A5D8091000444E650E083
:10E1100060E080620E947A5D84E080932E0344E692
:10E1200050E060E08CE00E947A5DC1110E94267090
:10E1300044E650E060E086E0CF910C947A5D81E0A7
:10E140000C945E70CF92DF92FF920F931F93CF9348
:10E15000DF9300D000D01F921F92CDB7DEB78A3078
:10E16000D9F480913003843018F08FEF809330031E
:10E17000609130036F5F80E00E945A6F28960FB65F
:10E18000F894DEBF0FBECDBFDF91CF911F910F91ED
:10E19000FF90DF90CF90089590E8980F44E650E00C
:10E1A00061E09A3408F5482F4058550B9A0196E0E3
:10E1B000929FA001939F500D1124FA01EA56FB484B
:10E1C000F490E1E3F3E030E020E09FEF6191782FFD
:10E1D00076277F7789F4F901EF5CFC4F8083F22E7C
:10E1E00044E650E061E08F2D0E947A5D80912F031C
:10E1F0008F5F80932F03C2CF6F3709F03CC0F901C6
:10E20000EF5CFC4F8083922FF92EFA01EF56FB480A
:10E210008E010F5F1F4FD801959188E0182E10FED8
:10E2200005900294802D9795881F8D931A94B9F7C5
:10E23000BF2DE8E0BE02C001112444E650E060E0DA
:10E2400080640E947A5D6E01F9E0CF0ED11C44E635
:10E2500050E061E0D8018D918D010E947A5DC01679
:10E26000D106A9F780912F0344E650E060E0806872
:10E270000E947A5DB5CF67FF922F2F5F3F4F283006
:10E28000310509F0A3CF9F3F09F0BECFA9CFCF93AF
:10E2900024E1AC01249FC001259F900D11246091C1
:10E2A0006D0370916E030F94A9A4C62F653108F019
:10E2B000C4E180916C038C1748F48FEF0E94A27028
:10E2C00080916C038F5F80936C03F3CFCF9108959F
:10E2D00081E090E090936E0380936D030E944771FC
:10E2E0006CE271E080E090E00D94BD0D8F929F9202
:10E2F000AF92BF92EF92FF920F931F93CF93DF9352
:10E30000CDB7DEB7A0970FB6F894DEBF0FBECDBF76
:10E31000611571058105910599F480E3A0960FB60A
:10E32000F894DEBF0FBECDBFDF91CF911F910F914B
:10E33000FF90EF90BF90AF909F908F900C94A27041
:10E3400000E0842E912CB12CA12C9E012F5F3F4F19
:10E350007901A50194010F9453A4F701E00FF11D79
:10E360006083B901CA010F5F6115710581059105CF
:10E3700081F70E0D1F2D111DE016F10659F0F80161
:10E3800082918F018A3020F4805D0E94A270F4CFC8
:10E39000895CFBCFA0960FB6F894DEBF0FBECDBF51
:10E3A000DF91CF911F910F91FF90EF90BF90AF90B1
:10E3B0009F908F900895CF92DF92EF92FF926B0122
:10E3C0007C01F7FE0BC08DE20E94A270F094E094F5
:10E3D000D094C094C11CD11CE11CF11C4AE0C701BF
:10E3E000B601FF90EF90DF90CF900C9476710F9371
:10E3F0001F93CF938C01C62FCC2359F0F8012491A1
:10E40000222339F00F5F1F4F84910E94A270C150E8
:10E41000F3CF8C2F0E94286F8C2FCF911F910F91DB
:10E4200008950F931F93CF93DF938C01EB010E940C
:10E43000267010926C0310936E0300936D0361E0DD
:10E4400080E00E945A6F64E1CE010E94F77162E0A1
:10E4500080E0DF91CF911F910F910C945A6FEF9252
:10E46000FF920F931F93CF93DF93709163043091CA
:10E47000620473133FC0122FEA01062F7C018091C2
:10E4800059028823D1F00E946662482F609160048F
:10E4900080E00E94137061E1C7010E94F771402F74
:10E4A0006091600493E1981B892F0E94137040E2F1
:10E4B0006091600483E10E9413708091610488235D
:10E4C000C9F02091630480911E0690911F062817C1
:10E4D000190681F410925A02812FFE01199581E0EC
:10E4E00080935A02DF91CF911F910F91FF90EF908F
:10E4F0000C947362809163048F5F80936304DF9157
:10E50000CF911F910F91FF90EF9008950F931F935C
:10E51000CF93C82F8B010E946662482F60916004E0
:10E5200080E00E94137062E1C8010E94F7718C2F95
:10E53000CF911F910F910C94216FCF93DF93309166
:10E54000630420916204321321C0EB01BC0180916D
:10E550005902882319F080E20E948672809161043A
:10E560008823A1F02091630480911E0690911F06DC
:10E570002817190659F410925A02FE01199581E0E4
:10E5800080935A02DF91CF910C947362809163045F
:10E590008F5F80936304DF91CF910895309163047E
:10E5A00020916204321319C0BC0180915902882362
:10E5B00019F083E80E94867280916104882369F0D3
:10E5C0002091630480911E0690911F06281719065A
:10E5D00021F40E941B630C947362809163048F5F2B
:10E5E000809363040895CF93DF9330916304209167
:10E5F000620432131EC0EB01BC01809159028823D2
:10E6000019F08EE70E94867280916104882389F058
:10E610002091630480911E0690911F062817190609
:10E6200041F460E0CE010E94DD62DF91CF910C9455
:10E630007362809163048F5F80936304DF91CF9155
:10E6400008953091630420916204321319C0BC0113
:10E6500080915902882319F080E20E94867280918D
:10E660006104882369F02091630480911E069091D3
:10E670001F062817190621F40E94736281E008958D
:10E68000809163048F5F8093630480E008950F930B
:10E690001F93CF938C01C62FCC2349F0F8018191B1
:10E6A0008F01882321F00E94A270C150F5CF8C2FDA
:10E6B0000E94286F8C2FCF911F910F910895CF93B7
:10E6C000DF93EC018991882319F00E94A270FACFA0
:10E6D000DF91CF9108950E94A27090E080E00895AC
:10E6E000109295031092A7050895CF9380919503FA
:10E6F000C1E0811104C0C0E08C2FCF9108950E9429
:10E700007073FACF80915902882309F452C0209186
:10E71000A1033091A20380919D0390919E03211546
:10E720003105D9F040911E0650911F064115510543
:10E73000A1F07CF040919B0350919C03481759072E
:10E7400041F430939C0320939B0310921F06109278
:10E750001E061092A2031092A10320919B033091F8
:10E760009C0340911E0650911F06240F351F1092E6
:10E770001F0610921E062817390744F080919F0348
:10E780009091A003281739070CF4C90190939C03BA
:10E7900080939B0361E080E00E945A6F40919B034D
:10E7A00050919C03609196037091970380E20E94C0
:10E7B000326F0E947573882341F1E0919903F091C3
:10E7C0009A0380919B0390919C03209198038083EE
:10E7D0002830C9F48091DF038823B9F081508093F9
:10E7E000DF0390E0FC01EE0FFF1FE80FF91FE95A6D
:10E7F000FC4F6281062E000C770B20E040E0808108
:10E8000091810C94B7629183E5CF08950E9475734E
:10E8100081110C941B63089580911E0690911F0630
:10E8200097FF07C010921F0610921E0687E00F94F4
:10E83000AD2580911E0690911F0620919203281706
:10E84000190619F014F0809392038091920380933B
:10E8500062040E9475738093610408958EEF9FE0B7
:10E860000F94E0A38E3F39F091E020912D032813FF
:10E8700090E0892F089580E0089510922D036EEFA7
:10E880008EEF9FE00D9404A4853728E6920709F4E3
:10E8900059C0F8F48E3625E6920709F459C050F4B1
:10E8A000833723E69207B1F185369446B1F182EAC7
:10E8B00093E60895823726E6920791F1823728E69B
:10E8C000920709F442C08337954689F789EF93E6AA
:10E8D00008958C3620E7920731F170F48C362EE6DD
:10E8E000920721F18F362EE6920731F1843799464F
:10E8F000F1F687EE93E608958B3623E79207F9F059
:10E90000863723E79207A9F08F36924781F685EA8A
:10E9100093E6089589E094E6089581E094E60895E9
:10E9200080EF93E6089580EE93E6089585ED93E6F3
:10E9300008958DEC93E6089587EC93E608958CEBAB
:10E9400093E6089585EB93E608958CEA93E608959F
:10E9500081E194E60895EDE8F4E785919591A5911C
:10E96000B4918F3F9F4FAF4FBF4FB1F020E031E0E8
:10E9700081E0F9014591559165917491453A5A4567
:10E98000644B7B4409F00895F90134964591549104
:10E99000240F351F8F5FEDCF81E008950F931F93F4
:10E9A000811113C010922C0310922B0310922D038F
:10E9B00090912D0398135CC0682F8EEF9FE00F9409
:10E9C00004A481E01F910F910895813089F7E0E060
:10E9D000F1E04591559165917491453A5A45644BE2
:10E9E0007B4431F7E4E0F1E0A591B491E8E0F1E097
:10E9F0006591749150E040E030E020E0A417B50745
:10EA000029F5261B370B3227232732276217730776
:10EA100009F0CECFECE0F1E005911591259134910C
:10EA2000EDE8F4E745915591659174910417150748
:10EA30002607370709F0BCCF20E031E030932C03E4
:10EA400020932B0391E090932D03B2CFFA01E05075
:10EA5000FF4FE491F0E098E040FD90E002C0EE0F3F
:10EA6000FF1F9A95E2F72E0F3F1F4F5F5F4FC6CFF4
:10EA700080E0A8CF20912D03211104C0FC01329623
:10EA8000CF01089540912B0350912C03411551055E
:10EA9000A9F3FC01259134912F3F320779F3F90155
:10EAA0003896EE0FFF1FE40FF51F25913491FA0100
:10EAB000E20FF31F2491222309F3E2CF8F929F925A
:10EAC000AF92BF92CF92DF92EF92FF920F931F937C
:10EAD000CF93DF93E091630430916204E31373C03A
:10EAE000C22F6A017B015C01809159028823A1F148
:10EAF0000E94666201E08E3309F000E00C2B802F4B
:10EB00008270882EE114F10409F46FC0E70190E2ED
:10EB1000992E882009F441C0CE010F949EA114E0E3
:10EB2000180F4EE300FF40E26091600480E00E9415
:10EB3000137064E1611BC5010E94F7718BE50E94AF
:10EB4000216FCE01882089F10E941D6F8DE50E9402
:10EB5000216F892D0E94216F80916104882399F192
:10EB60002091630480911E0690911F0628171906B4
:10EB700051F5EF28E9F460E0C6010E94DD62DF9103
:10EB8000CF911F910F91FF90EF90DF90CF90BF90AA
:10EB9000AF909F908F900C947362FE0101900020C3
:10EBA000E9F7EC1B13E01E0FBCCF0E945F73CECFC2
:10EBB00010925A02C114D10411F0F601199581E0A6
:10EBC00080935A02DCCF809163048F5F809363044B
:10EBD000DF91CF911F910F91FF90EF90DF90CF9039
:10EBE000BF90AF909F908F90089583E798E40E9424
:10EBF0003A75EC018EE7982E8CCF0F931F93CF932D
:10EC0000DF938C01EB0188E79EE40E943A759F93A5
:10EC10008F938CE591E89F938F93DF93CF930F941D
:10EC2000F7A2C80FD11D47E050E0B801CE010F9404
:10EC3000D0A31F820F900F900F900F900F900F9006
:10EC4000DF91CF911F910F9108950F931F93CF9351
:10EC5000DF93CDB7DEB763970FB6F894DEBF0FBE74
:10EC6000CDBF3091630420916204321338C08B0110
:10EC7000209159022223A9F0BE016F5F7F4F0E94AD
:10EC8000FD750E946662482F6091600480E00E94DA
:10EC9000137062E1CE0101960E9447738EE70E94D5
:10ECA000216F809161048823D1F0209163048091C9
:10ECB0001E0690911F062817190689F460E0C80106
:10ECC0000E94DD620E94736263960FB6F894DEBF05
:10ECD0000FBECDBFDF91CF911F910F91089580910D
:10ECE00063048F5F80936304EFCFCF93DF93EC01D6
:10ECF00020E030E04CE852E460916D1270916E12A9
:10ED000080916F12909170120F9408A560936D120C
:10ED100070936E1280936F129093701260E070E0A7
:10ED200080EA91E40F94814C0E94ED630E9426706A
:10ED30008DEE91E60E943A75AC0160E080E00E94A1
:10ED400007708881882339F061E080E00E945A6F63
:10ED5000CE010E945F7385E699E30E943A75AC018B
:10ED600062E080E00E94077083E49BE20F94B20BA4
:10ED7000DF91CF910D94FB1A0F94A7658F3F11F18E
:10ED800080E00E9438700E94267089EA99E50E940E
:10ED90003A75AC0161E080E00E94077080E20E9459
:10EDA000A2700F94A765682F70E06F5F7F4F072EEA
:10EDB000000C880B990B0E94DB710F94719D81E010
:10EDC0000C94387008951F920F920FB60F92112471
:10EDD0000BB60F922F938F939F93EF93FF93E09136
:10EDE0002603E830E8F4F0E08827E650F9488F4F32
:10EDF0000D94F0A402771C77277735774B775477FB
:10EE0000777789778091280681110AC08091EE0575
:10EE1000880F80932503882319F081E080932603CF
:10EE2000FF91EF919F918F912F910F900BBE0F90BB
:10EE30000FBE0F901F901895809124038F5F8093D1
:10EE4000240390912503981758F382E0E7CF83E0DD
:10EE5000809326038FE0809323038FEF86BD81E0AC
:10EE600085BD84B58F7E84BDDBCF809123038295E1
:10EE7000807F819588BD80912303882321F0815074
:10EE800080932303CDCF84E0809326038FEF88BD4A
:10EE90008EEF86BDC5CF85E0809326038FEF88BDBA
:10EEA00086BD82E085BDBCCF2FEF28BD80912806AE
:10EEB0008111B6CF809124038F5F809324039091BA
:10EEC0002503891708F4ACCF8091EE0590E08F37C9
:10EED00091050CF0A5CF86E0809326038FE0809308
:10EEE000230326BD81E085BD84B58061BCCF8091C0
:10EEF00023038295807F819588BD809123038111B2
:10EF0000BECF87E08093260380E886BD8FEF88BD63
:10EF100087CF1092260380E886BD8FEF88BDC1CFD2
:10EF2000CF93C82F682F87E69FE00F9404A4CC23CB
:10EF300019F0CF910D94DC6D1092F1161092FD1620
:10EF4000CF9108951092B6030F94F00D60930717B8
:10EF5000709308178093091790930A170895809368
:10EF6000220380FD1CC010923E0320913E038FEFD0
:10EF7000820F8E3FE8F08091A000877F8093A000F1
:10EF80001092AD001092AC009FB7222361F0F8946C
:10EF9000809102018062809302019FBF08958FEFEC
:10EFA00080933E03E2CFF894809102018F7DF3CFEE
:10EFB000EFB7F8948091A00088608093A00030E0C3
:10EFC000809172004FEF50E081FF04C04091A80093
:10EFD0005091A900249FC001259F900D349F900D52
:10EFE00011246FEF70E00F94A9A47093AD006093AB
:10EFF000AC00EFBF08951F93CF93DF93D09122030E
:10F00000D1FD1DC01091CC03C1E020E030E048E408
:10F0100052E460915A0D70915B0D80915C0D90915E
:10F020005D0D0F9491A718160CF0C0E0DE7FCD2B7C
:10F0300081E0111101C080E0C82BC09322038091B0
:10F040002203DF91CF911F910C94AF77EF92FF9243
:10F050000F931F93CF93DF93EC018B017A010E94F2
:10F06000DA5581110BC0A801BE01C701DF91CF9114
:10F070001F910F91FF90EF900D94F4A3DF91CF912A
:10F080001F910F91FF90EF9008950F931F93CF93CF
:10F09000DF938C01D62FC72F0F94EEA38F3F9807D5
:10F0A00039F46D2F7C2FC8010F943EA48D2F9C2F17
:10F0B000DF91CF911F910F9108950F931F93CF93DD
:10F0C0008C01C62F0F94E0A38F3F29F46C2FC80149
:10F0D0000F9428A48C2FCF911F910F910895CF9357
:10F0E000DF93EC010F94EEA3BC016F5F7F4FCE0165
:10F0F000DF91CF910D943EA4CF93DF93EC010F9459
:10F10000E0A361E0680FCE01DF91CF910D9428A4B8
:10F110002BE0829FC0011124805B924F0F94EEA3DD
:10F1200021E0019609F420E0822F0895CF93DF9328
:10F13000C82FD8E0CF5FC8300CF0C0E08C2F0E9401
:10F140008878811103C0D150A9F7CFEF8C2FDF91C0
:10F15000CF91089581EA9DE00F94E0A30E949678F4
:10F1600087FD05C0682F81EA9DE00D9404A40895F1
:10F170000F931F93CF93C82F8B0160E474E7823005
:10F1800070F069E374E7843050F061E374E7843031
:10F1900031F069E274E7853011F062E274E7C8018A
:10F1A0000F9497A18CEF8C0F823028F0C170CF5C48
:10F1B000F801C6831782CF911F910F91089561E0E6
:10F1C00080EC9FE00F9404A460E08FEB9FE00F942D
:10F1D00004A460E08EEB9FE00F9404A460E08DEB4C
:10F1E0009FE00F9404A460E08CEB9FE00D9404A4D6
:10F1F000CF93C82F82958F700E94485D8C2F8F709F
:10F20000CF910C94485D40913C1250913D1290E09A
:10F2100080E041155105B1F1209138123091391239
:10F2200090E080E0F901E55BFF4EA081A23021F47F
:10F2300061817281860F971F4150510919F1F901BF
:10F24000E25BFF4EA1919F012B543041A111FACFF7
:10F25000F901E55BFF4E2D3EA1E03A0730F4A191A4
:10F26000A111E0CF2F5F3F4FF6CF2D3EE1E03E07EB
:10F27000C9F6EBE4F0E19F012B543041A191AA23A0
:10F28000D1F3D0CF089580913C1290913D12181681
:10F2900019060CF043C0019790933D1280933C12E5
:10F2A000892BA1F48091471090914810892B21F46B
:10F2B00010924A10109249108091491090914A1072
:10F2C000909339128093381281E00895809138121A
:10F2D000909139120396FC01E55BFF4E2081019667
:10F2E0002111F9CFFC01E55BFF4E8D3E21E0920735
:10F2F00040F441919C012F5F3F4F4111E1CFC90183
:10F30000F4CFEBE4F0E18D3E21E09207C9F6CF01A6
:10F310008B54904121912223D1F3D2CF80E00895E4
:10F32000FC0120E03EE2DB014D91BD01403249F09D
:10F33000283011F430833196DB0111974C914083D2
:10F3400031962F5F2B3079F71082089540E050E01E
:10F35000BA010D940B2DFC01238121110D94E92E8E
:10F36000089590911C06911107C09091C00095FFDF
:10F37000FCCF8093C6000895913031F49091C8007D
:10F3800095FFFCCF8093CE0008958F929F92AF920D
:10F39000BF92EF92FF920F931F93CF93DF93CDB75E
:10F3A000DEB7A0970FB6F894DEBF0FBECDBF6115D4
:10F3B00071058105910599F480E3A0960FB6F89444
:10F3C000DEBF0FBECDBFDF91CF911F910F91FF9098
:10F3D000EF90BF90AF909F908F900C94B17900E028
:10F3E000842E912CB12CA12C9E012F5F3F4F7901CF
:10F3F000A50194010F9453A4F701E00FF11D608360
:10F40000B901CA010F5F611571058105910581F789
:10F410000E0D1F2D111DE016F10659F0F801829115
:10F420008F018A3020F4805D0E94B179F4CF895C2D
:10F43000FBCFA0960FB6F894DEBF0FBECDBFDF9115
:10F44000CF911F910F91FF90EF90BF90AF909F9041
:10F450008F900895CF92DF92EF92FF926B017C0123
:10F46000F7FE0BC08DE20E94B179F094E094D09445
:10F47000C094C11CD11CE11CF11C4AE0C701B601BB
:10F48000FF90EF90DF90CF900C94C5798F929F9270
:10F49000AF92BF92CF92DF92EF92FF92CF936B0128
:10F4A0007C01B42E20E030E0A9010F94FDA587FF78
:10F4B00007C08DE20E94B179F7FAF094F7F8F09462
:10F4C000C0E060E070E080E09FE3CB1541F020E019
:10F4D00030E040E251E40F9407A6CF5FF6CF9B01E6
:10F4E000AC01C701B6010F9408A56B017C010F9414
:10F4F00080A64B015C014AE00E94C579CC2391F1C2
:10F50000C501B4010F946C9E9B01AC01C701B6010B
:10F510000F9407A56B017C018EE20E94B179C15066
:10F5200008F120E030E040E251E4C701B6010F9459
:10F53000AD9E4B015C010F9479A66B01770FEE082D
:10F54000FF08C701B6010E942A7AC701B6010F94CD
:10F550006E9E9B01AC01C501B4010F9407A56B0120
:10F560007C01DDCFCF91FF90EF90DF90CF90BF90E7
:10F57000AF909F908F9008958AE00C94B1790E948B
:10F58000B17990E080E00895CF93DF93EC01FE0124
:10F590008491882321F00E94B1792196F8CFDF91E0
:10F5A000CF910895CF92DF92EF92FF92C0905A0DC3
:10F5B000D0905B0DE0905C0DF0905D0D83E998E7D5
:10F5C0000E94C47A42E0C701B6010E94467A8BE8E5
:10F5D00098E70E94C47A6091BC037091BD0380914A
:10F5E000BE039091BF0341E00E94467AFF90EF90E6
:10F5F000DF90CF900C94BC7A4F925F926F927F9283
:10F600008F929F92AF92BF92CF92DF92EF92FF9232
:10F610000F931F93CF93DF93CC24CA94DC2C7601F5
:10F620000EEA1FE093E2892E912CA12CB12C412CE3
:10F63000512C3201D0E0C0E08FEFC81609F45DC054
:10F64000C8010F94EEA3EC01BC01990F880B990B34
:10F650000F946E9E2091730D3091740D4091750D35
:10F660005091760D0F9407A62B013C01C701B601FE
:10F670000E942A7A87EE97E70E94C47AC501B401F6
:10F680000E942A7A87EE97E70E94C47ABE010D2E67
:10F69000000C880B990B0E942A7A87EE97E70E944C
:10F6A000C47A20E030E04AE754E4C301B2010F9489
:10F6B000AD9E0F94A26585E0880E911CA11CB11C23
:10F6C0000E5F1F4F8FEFC81AD80AE80AF80A0A3BE4
:10F6D0008FE0180709F0B0CFDF91CF911F910F9104
:10F6E000FF90EF90DF90CF90BF90AF909F908F9062
:10F6F0007F906F905F904F90089583E798E40E9409
:10F70000C47AB8CF882371F18BED97E70E94C47A51
:10F710006091901270E090E080E00E942A7A8091DF
:10F7200090128430D8F01092901286ED97E70E94E4
:10F73000C47A8091901290E00F94BF6580919012EE
:10F7400020915B1230915C1230935E1220935D1217
:10F750000E9437FE0E94ED630D94FB1A8F5F809329
:10F760009012E3CF86E19DE30E943A7570E060E07D
:10F770000E94C8D1E5CFCF93DF9383ED97E70E9436
:10F78000C47AC1E6D2E1688179818A819B8142E0B5
:10F790000E94467A8FEC97E70E94C47A6C817D8143
:10F7A0008E819F8142E00E94467A8BEC97E70E940F
:10F7B000C47A688579858A859B8542E00E94467A6D
:10F7C00087EC97E70E94C47A6C857D858E859F853E
:10F7D00042E00E94467A89E194E60E94C47A80E081
:10F7E0000F94D91A0F946E9EC7E6DDE02C813D81FF
:10F7F0004E815F810F9407A642E00E94467A83EC17
:10F8000097E70E94C47A81E00F94D91A0F946E9EF4
:10F81000288539854A855B850F9407A642E00E94BA
:10F82000467A8FEB97E70E94C47A82E00F94D91A48
:10F830000F946E9E2C853D854E855F850F9407A69F
:10F8400042E00E94467A8BEB97E70E94C47A83E0FD
:10F850000F94D91A0F946E9E288939894A895B8939
:10F860000F9407A6DF91CF910D94A2658AEC96E7DD
:10F870000E94C47A60915A0D70915B0D80915C0D6D
:10F8800090915D0D41E00E94467A87EC96E70E94D8
:10F89000C47A60915D1270915E12072E000C880B85
:10F8A000990B0F946E9E41E00E94467A83EC96E796
:10F8B0000E94C47A6091BC037091BD038091BE0325
:10F8C0009091BF0341E00E94467A80EC96E70E9447
:10F8D000C47A6091591270915A12072E000C880B4D
:10F8E000990B0F946E9E41E00E94467A8BEB96E74F
:10F8F0000E94C47A60915A0D70915B0D80915C0DED
:10F9000090915D0D41E00E94467A88EB96E70E9457
:10F91000C47A60915D1270915E12072E000C880B04
:10F92000990B0F946E9E41E00E94467A84EB96E715
:10F930000E94C47A6091F50570E090E080E00E943A
:10F940002A7A8FEA96E70E94C47A6091EE0570E009
:10F9500090E080E00E942A7A8BEA96E70E94C47ABF
:10F96000609185037091860380918703909188034D
:10F9700041E00E94467A0C94BC7A0E94C47A0C94AE
:10F98000BC7A8F929F92AF92BF92CF92DF92EF920A
:10F99000FF920F94F00D6B017C0120913202222323
:10F9A00009F1409178024130E9F080911402909180
:10F9B0001502A0911602B091170246015701881A4C
:10F9C000990AAA0ABB0A30E0A8EEB3E00F9480A41B
:10F9D00086169706A806B9066CF0443031F19CF4FF
:10F9E0004230D4F4C0921402D0921502E092160272
:10F9F000F0921702FF90EF90DF90CF90BF90AF9002
:10FA00009F908F900895453069F78EEC91EA0E949F
:10FA1000C47A86E998E706C08EEC91EA0E94C47A1F
:10FA200083EC98E70E94BD7CDDCF8EEC91EA0E94CA
:10FA3000C47A8DEA98E7F6CFCF9381EA9DE00F94E0
:10FA4000E0A3CBE08C9FC0011124805B924F0F9408
:10FA5000EEA38156904F803A9F40C8F082E698E727
:10FA60000E94BD7C81EA9DE00F94E0A38C9FC001C1
:10FA7000112470E060E0805B924F0F943EA485E219
:10FA800098E70E9494EA81E0CF910C943870CF916E
:10FA900008952F923F924F925F926F927F928F9232
:10FAA0009F92AF92BF92CF92DF92EF92FF920F930D
:10FAB0001F93CF93DF93CDB7DEB7A4970FB6F8941B
:10FAC000DEBF0FBECDBF0F94FB1A8091420D811196
:10FAD00017C081E08093721280913906882349F023
:10FAE00080913A06882329F020913B062F8321112B
:10FAF00020C081E08093531281ED98E60F947867DF
:10FB0000A4960FB6F894DEBF0FBECDBFDF91CF91A4
:10FB10001F910F91FF90EF90DF90CF90BF90AF902B
:10FB20009F908F907F906F905F904F903F902F901D
:10FB300008958BEA9DE00F94E0A3182F8EE40E94B5
:10FB4000F555082F0E940A568E83002329F087302E
:10FB500009F4C9C0833029F0133009F0C3C063E051
:10FB60006E8380E090E0A0E8BFE38A839B83AC8350
:10FB7000BD838AEA9DE00F94E0A3888F83E40E940E
:10FB8000F555182F0E940A56112329F0882319F0E1
:10FB90008B3008F4888F88E50E94F555882309F496
:10FBA000ABC00E94855A20E030E048E052E40F9458
:10FBB00007A520E030E048EB51E40F9407A56A87E1
:10FBC0007B878C879D8789E50E94F555882309F4FA
:10FBD0009CC00E94855A20E030E048E052E40F9437
:10FBE00007A520E030E040EA50E40F9407A56C8BB5
:10FBF0007D8B8E8B9F8B87E50E94F555882309F4BA
:10FC000089C00E94855A2A853B854C855D850F9465
:10FC100008A520E030E048E852E40F9408A5698F79
:10FC20007A8F8B8F9C8F88E40E94F555882309F486
:10FC30007AC00E94855A2C893D894E895F890F942C
:10FC400008A520E030E048E852E40F9408A56D8F45
:10FC50007E8F8F8F98A30F94E37B80912C029091DD
:10FC60002D02A0912E02B0912F0280930A1390933F
:10FC70000B13A0930C13B0930D130F94AA5405EC1F
:10FC80001FE0C8010F94EEA3019609F051C00E5F6A
:10FC90001F4F053D8FE01807A1F7212CA9E0B3E124
:10FCA000BAA3A9A3B987A887512C412C312C042DC4
:10FCB000842D63E00F948FA4988B6884798410E07E
:10FCC000F889F11137C0812F63E00F948FA491114F
:10FCD00031C021103FC17E81733009F470C08F8123
:10FCE0008E8737C01E836AE979E989E19FE36A83D9
:10FCF0007B838C839D833DCF80E090E0A0E8BFEFC5
:10FD00008A879B87AC87BD875ECF60E070E080E824
:10FD10009FEF6DCF80E090E0A0E8BFE7898F9A8FDA
:10FD2000AB8FBC8F80CF60E070E080E89FE78FCF23
:10FD30002F80B4CF60E070E080EC9FE7D301119694
:10FD40006D937D938D939C931497BE81B330C1F1D5
:10FD50001E86812F0E94E05E4B015C01802F0E9475
:10FD6000E05E6B017C01A50194016A857B858C8531
:10FD70009D850F9491A718160CF41CC1298D3A8DFE
:10FD80004B8D5C8DC501B4010F9491A718160CF42E
:10FD900011C1A70196016C897D898E899F890F9475
:10FDA00091A718160CF406C12D8D3E8D4F8D58A1CC
:10FDB000C701B6010F9491A718160CF4FBC0339439
:10FDC0001F5F24E0620E711C173009F079CF6FEFCE
:10FDD000461A560A888599854C969987888797E0B0
:10FDE0004916510409F063CF0F94BD92A0915D06AE
:10FDF000AF83B091DE03B88781E080935D068AE02F
:10FE0000830D8093DE0381E00E94F96E80E090E034
:10FE1000A0EAB0E48093691290936A12A0936B12E7
:10FE2000B0936C1265E575E585E591E40F94814C1E
:10FE300080E00E9466659CA38BA3312C832D67E034
:10FE40000F948FA4F82E092F682F70E07F876E879C
:10FE500080FF03C076E0791B072F802F63E00F94AB
:10FE60008FA4911105C08F2D0F948FA411E09111D3
:10FE700010E0802F0E94E05E688B798B8A8B9B8BD1
:10FE80008F2D0E94E05E4B015C018E81833009F072
:10FE900099C01111C8C027E0AE85BF852A9FF00127
:10FEA0002B9FF00D1124E00FF11DEE0FFF1FEE0F41
:10FEB000FF1FE75FFC4E60E070E080EC9FE761832E
:10FEC0007283838394833394E1E33E12B7CF80E05F
:10FED00090E0A0EAB0E48093691290936A12A09334
:10FEE0006B12B0936C1265E575E585E591E40F94AE
:10FEF000814C0F94FB1AB1E33B1609F43CC280918C
:10FF00003D0391E0980F90933D03882309F4D3C1FA
:10FF100060E080E00E94F9DE84E396E30E943A7597
:10FF20000E9494EA80E00E94F2E981E080937802E6
:10FF300086EE9BE60E9494DE2F8120935D06688505
:10FF40006093DE0382E00E94F96E0F94FB1A109218
:10FF50007212D6CD011103C0112309F4BCCE812F3A
:10FF600063E00F949BA4840D952D911D880F991F1C
:10FF70008D53904F0F94EEA3BC01990F880B990BF2
:10FF80000F946E9E2AE037ED43E25CE30F94AD9E42
:10FF90009B01AC0160910A1370910B1380910C13BB
:10FFA00090910D130F9408A5F301618372838383ED
:10FFB000948391CEFE85FF2309F402CF222009F419
:10FFC000FECEFECE288939894A895B896A857B8580
:10FFD0008C859D850F9491A7181604F1288939897D
:10FFE0004A895B89698D7A8D8B8D9C8D0F94FDA5D7
:10FFF00087FD14C0A50194016C897D898E899F8934
:020000021000EC
:100000000F9491A7181654F0A50194016D8D7E8D63
:100010008F8D98A10F94FDA587FF05C0112309F4CA
:1000200052CF211050CF10E0A7E08E859F85A89F6A
:10003000F001A99FF00D1124E00FF11FEE0FFF1F3B
:10004000EE0FFF1FE75FFC4E41805280638074809B
:10005000C12CD12CE0EAEE2EE0E4FE2E222051F05D
:1000600023E333E343EB5EE3C301B2010F9408A53E
:100070006B017C01A70196016091691270916A126F
:1000800080916B1290916C120F94FDA587FF10C0A8
:10009000C0926912D0926A12E0926B12F0926C12C6
:1000A00065E575E585E591E40F94814C0F94FB1AA5
:1000B000688979898A899B89609361127093621239
:1000C00080936312909364128092651290926612EC
:1000D000A0926712B092681265E672E181E692E141
:1000E0000E941E6960E070E086E193E40F94814C09
:1000F0000F94FB1A8091420D882339F07F81709311
:100100005D0688858093DE03FBCC812C912C70E208
:10011000A72E71ECB72E222051F02A813B814C8111
:100120005D81C301B2010F9407A54B015C01488DAD
:10013000C501B4010F94ED7B81110BC08EEF99E3E3
:100140000E943A759F938F930F94A2A20F900F90E5
:10015000BECE2091691230916A1240916B1250917B
:100160006C12C701B6010F9407A520E030E0A90189
:100170000F94FDA587FF36C060E070E080EA90E450
:100180006093691270936A1280936B1290936C1251
:1001900065E575E585E591E40F94814C0F94FB1AB4
:1001A000488DC501B4010F94ED7B882339F220916D
:1001B000691230916A1240916B1250916C1260E09A
:1001C00070E080EA90E40F9407A52DEC3CEC4CEC39
:1001D0005DE30F94FDA587FF05C087E397E70F94C4
:1001E000C9A275CEC0906912D0906A12E0906B12CD
:1001F000F0906C122220A1F0A7019601C301B20178
:100200000F9407A59B01AC015F776A817B818C818C
:100210009D810F94FDA587FF03C08EEF96E7DFCF8A
:100220008FEA9FE00F94E0A3882309F440C086EA98
:100230009FE00F94E0A38823D1F160918503709132
:10024000860380918703909188030E9486562091AF
:10025000730D3091740D4091750D5091760D0F9482
:1002600007A69B01AC01E7E0AE85BF85EA9FC00110
:10027000EB9F900D1124080F191F000F111F000F85
:10028000111F075F1C4EC701B6010F9407A5D801C7
:1002900011966D937D938D939C9314978091DE03BB
:1002A00081508093DE0381E00E94F96E0CCE20E045
:1002B00030E0A901D8CF85E00F94AD25C12CD12C19
:1002C00090EAE92E90E4F92E80E096E30E943A75D8
:1002D0000E94A9E090E080E00E94C2DF81E00E94DD
:1002E00011FC80E00F948825182F60E070E080E812
:1002F0009FEB0E94946C81E00F948825C092691254
:10030000D0926A12E0926B12F0926C1265E575E57C
:1003100085E591E40F94814C0F94FB1A812F0F9483
:10032000882582E00F94E71A20E030E040EA50E4AC
:100330000F9491A7181644F2EF81E0935D06F885BB
:10034000F093DE0381E00E943870DD24D394DF92C5
:10035000812C912C5401CC24C394E12CF12C8701E5
:1003600021E040E050E0BA0181E00E942A6DD09285
:1003700053120F90C5CB10923D038BA19CA10E94FC
:100380004C65109227061092260680E10E945BD7EA
:10039000882391F00E941C7D81EA9DE00F94E0A3E8
:1003A0002BE0829FC0011124805B924F0F94EEA33B
:1003B0009093270680932606609126067091270663
:1003C000072E000C880B990B0F946E9E905820916D
:1003D000730D3091740D4091750D5091760D0F9401
:1003E00007A60E94A65E80EC9FE00F94E0A391E038
:1003F000813009F090E099834FEB5FE06CE4CE012F
:1004000001960E942456F82E4EEB5FE062E5CE0185
:1004100001960E942456082F4DEB5FE066E4CE0162
:1004200001960E942456182F4CEB5FE062E4CE0147
:1004300001960E942456212F110F330B082E000C19
:10044000990B5C01A21AB30A8F2DFF0C990B280F90
:10045000391F46E0429F6001439FD00C1124F12CCC
:10046000E12C002E000C110B081B190BB701665F65
:100470007C4E3B01460177E07A83D3012D903D907D
:100480004D905D903D01FD013497FB87EA87B401F3
:10049000092C000C880B990B0F946E9E2FE333EC04
:1004A0004EE259E30F94AD9EA20191010F9408A56D
:1004B000AA85BB856D937D938D939C931397BA8189
:1004C000B150BA83800E911EB111D7CFCA0CDB1C7C
:1004D000ECE1EE0EF11CF4ECEF16F10439F60F949A
:1004E000BD928DE40E94F555882309F484C00E94D2
:1004F0000A562E81273009F094C0882309F491C050
:10050000BB24B394AA24AA94AB0C09A11AA1612C10
:100510008EEF882E8B0C6A2D862D0F94755499249E
:100520009394960C81116EC06B2D862D0F9475548B
:10053000C12CD12C7601712C882381F020E030E091
:10054000A901D8015D966D917D918D919C919097B7
:100550000F9408A56B017C0177247394682D862D78
:100560000F947554882369F0F8017B9720813181BD
:1005700042815381C701B6010F9408A56B017C012C
:1005800073946A2D892D0F947554882361F0F801B6
:100590002581368147815085C701B6010F9408A592
:1005A0006B017C0173946A2D8FEF860D0F94755447
:1005B000882331F1F80133972081318142815381C1
:1005C000C701B6010F9408A56B017C017394672DD8
:1005D00070E090E080E00F946E9E9B01AC01C7013B
:1005E000B6010F9407A6D80111966D937D938D9354
:1005F0009C93149707C08CEA9DE00F94E0A379CFF9
:100600007110E5CF692C0C5F1F4FB7E09B1283CFB1
:10061000B394E9A1FAA17C96FAA3E9A3F8E0BF128A
:1006200071CF81E0809309138FE40E94F555811109
:1006300003C00E943D6A79CC0E940A568111F9CF0D
:100640000E94416572CCEC01F8940F940511179A41
:1006500010923906169A10923A06149A81EB91EA92
:100660000E94C47A86E098E70E94BD7C209779F0CA
:10067000CE010E94BD7CBE0185E99CE00F943EA4A2
:1006800062E484E99CE00F9428A40E941F66CEEFE8
:10069000D7E7F1CF2F923F924F925F926F927F9266
:1006A0008F929F92AF92BF92CF92DF92EF92FF9282
:1006B0000F931F93CF93DF9300D000D0CDB7DEB759
:1006C000809177028C831092770280E00F948825C6
:1006D0008B830E94416583E591E60E943A750E94F2
:1006E000A9E04DE457E663E080E00E94077081E0F6
:1006F0008093770280E090E0A0EAB0E480936912F2
:1007000090936A12A0936B12B0936C1265E575E535
:1007100085E591E40F94F6501092770280E090E026
:10072000A0E8BFE38093611290936212A0936312DA
:10073000B09364128093651290936612A09367122F
:10074000B093681265E672E181E692E10E941E694B
:1007500060E070E088E492E40F94F6500E94AE6688
:1007600082E00F94AE7943E060E070E080E291ECCB
:100770000F94ED7B811106C08EEF99E30E943A75CC
:100780000E9423838091691290916A12A0916B124A
:10079000B0916C1280930A1390930B13A0930C13D7
:1007A000B0930D13E2E0F0E0FA83E983C12CD12C81
:1007B00030EAE32E30E4F32E43E0B42E52E0952EDF
:1007C00004E811E867E0A62E0E944165C092691214
:1007D000D0926A12E0926B12F0926C1265E575E5A8
:1007E00085E591E40F94F65029812150822F6B2DDD
:1007F0000F948FA4892E822F0F949BA4782E80FFB4
:1008000003C0F92DF8198F2E882D880F880D0E94AE
:10081000E05E609361127093621280936312909312
:100820006412872D880F870D0E94E05E6093651229
:1008300070936612809367129093681265E672E176
:1008400081E692E10E941E6960E070E088E492E433
:100850000F94F65063E080E00E945A6F8A818F9374
:1008600099819F931F930F930E940B6F43E060E069
:1008700070E080E291EC0F94ED7B582E0F900F907A
:100880000F900F90882309F477CFA79CF0011124D3
:10089000E80DF11DEE0FFF1FEE0FFF1FE75FFC4E8F
:1008A0008091691290916A12A0916B12B0916C12B2
:1008B00081839283A383B483E981FA813196FA8399
:1008C000E9833A9709F080CF60900A1370900B1378
:1008D00080900C1390900D13462CA72CB82C292C2B
:1008E0001E821D8209E013E18D819E81865F9C4EF0
:1008F0009A83898393E0392EE981FA81C190D1905E
:10090000E190F190FA83E9839301A401C701B60154
:100910000F9491A7181614F036014701242D3A2D93
:100920004B2D522DC701B6010F94FDA587FD04C0C4
:100930004C2CAD2CBE2C2F2C3A943110DDCF8D8158
:100940009E814C969E838D838435910559F6930143
:10095000A401642D7A2D8B2D922D0F9407A520E0F4
:1009600030E040E450E40F9491A718162CF587E688
:1009700091E80E94BD7C512CFC81F09377028B8121
:100980000F948825852D26960FB6F894DEBF0FBEEE
:10099000CDBFDF91CF911F910F91FF90EF90DF902E
:1009A000CF90BF90AF909F908F907F906F905F900F
:1009B0004F903F902F900895198285ECE82E8FE09C
:1009C000F82E68011D829D81911103C0E981EE23FB
:1009D00029F120910A1330910B1340910C1350917F
:1009E0000D13F60161817281838194810F9407A5B3
:1009F00020E030E048EC52E40F94AD9E20E030E07F
:100A000040E05FE30F9408A50F94AFA60F9479A67A
:100A1000C7010F9422A4F2E0EF0EF11C84E0C80E8F
:100A2000D11C9D819F5F9D83933069F6045E1F4FAB
:100A3000E981EF5FE983E33021F60F94E37B0E94C5
:100A40003D6A9ACF88E493E00F94471080913C125E
:100A500090913D12892B79F0E0913812F091391282
:100A6000E55BFF4E8081813011F0863021F480EF0C
:100A700099E60C94BD7C089580913C1290913D12B2
:100A8000892B29F00E9422850E944379F5CF10928C
:100A900039121092381210924A101092491081E0C7
:100AA000809353120895EF92FF920F931F93CF9369
:100AB000DF9380910913882389F180E997E70E94E9
:100AC000BD7C8AE797E70E94BD7C89E697E70E9494
:100AD000BD7CC7E0DCE1C15058F1CD9F700111240D
:100AE00001E010E086E697E70E94C47AF801EE0F75
:100AF000FF1FEE0FFF1FEE0DFF1DEA5FFC4E608132
:100B000071818281938145E00E94467A0F5F1F4F79
:100B10000830110539F70E94BC7ADDCF8DE997E7DF
:100B2000DF91CF911F910F91FF90EF900C94BD7CBE
:100B3000DF91CF911F910F91FF90EF900895CF9289
:100B4000DF92EF92FF926B017C01C0922703D0925B
:100B50002803E0922903F0922A0380914303823014
:100B6000B1F420E030E040E950E4C7010F94FDA566
:100B700087FF14C08091970D9091980DA091990DC9
:100B8000B0919A0D803D9740A105B10520F5C701B0
:100B9000B601FF90EF90DF90CF9008952AE939E9F0
:100BA00049E95EE3C701B6010F94FDA587FF0AC0BE
:100BB00020E030E048E351E4C701B6010F94AD9E58
:100BC0006B017C0184E794E70E94C47AC701B601F7
:100BD0000F94A265DCCF2AE939E949E95EE3C70150
:100BE000B6010F94FDA587FDE3CF20E030E040E89B
:100BF0005EE3C701B6010F94AD9E20E030E048E50A
:100C000050E40F9408A5DCCFCF92DF92EF92FF92D1
:100C1000CF93909143039817B9F1C82FC090270341
:100C2000D0902803E0902903F0902A0320E030E0E0
:100C3000A901C701B6010F94FDA5882341F0C09218
:100C4000BB0DD092BC0DE092BD0DF092BE0D87E5BC
:100C500094E70E94C47AC13011F1E0F0C23011F182
:100C6000C09343036091BB0D7091BC0D8091BD0D8D
:100C70009091BE0D0E949F856093BB0D7093BC0D3B
:100C80008093BD0D9093BE0DCF91FF90EF90DF90BC
:100C9000CF9008958FE494E70E94BD7CE1CF8BE470
:100CA00094E7FACF87E494E7F7CF0F94FB1A179AEB
:100CB000E9E3F6E01082169A1182149A80E00E940D
:100CC00004868FEF9FEF90937302809372022FEF51
:100CD00020936F0290933E0280933D0220933F0247
:100CE000909371028093700290933C0280933B0238
:100CF0000895182FF894CDB7DEB700D0CF90DF90CD
:100D0000EF9088E199E20FB6F894A895809360007F
:100D10000FBE909360009FB7F894E2E0F1E080810D
:100D2000886080839FBF0F94051186E094E70E943E
:100D3000BD7C8EEF93E70E94C47A612F70E090E053
:100D400080E04AE00E94C5798AEF93E70E94C47A66
:100D50008E2DB60190E040E10E94C57986EF93E7C1
:100D60000E94C47ABE0190E080E040E10E94C57913
:100D70000E94BC7A40E060E072E290E080E00F9474
:100D8000D27880EF99E60E94BD7C0E941F66C82F32
:100D90009FB7F894809102018460809302019FBF05
:100DA0006C2F83E09DE00F9404A480910F068823AC
:100DB00019F08C2F0E9479860E941F661F920F9255
:100DC0000FB60F92112483E00E94C7861F920F92E4
:100DD0000FB60F92112482E00E94C78641ED50E0C9
:100DE00065E273E787E69DE00F947AA10F94A63C35
:100DF0000F9440170E944A648EEC91EA0E94C47AD4
:100E000083E093E70C94BD7C44E050E064E170E043
:100E100087E69DE00F94D0A343E050E065E273E7DE
:100E200087E69DE00F94BFA1892B09F05DC0E9EE34
:100E3000F3E7459155916591749188ED90E00E949A
:100E40009A5DEDEEF3E745915591659174918CEDC6
:100E500090E00E949A5DE1EFF3E7649180EE90E00C
:100E60000E945D78E2EFF3E76591749181EE90E086
:100E70000E944578E4EFF3E76591749183EE90E08A
:100E80000E944578E5EEF3E745915591659174919F
:100E900084ED90E00E949A5D41EC53E760E170E0E0
:100EA00080EB90E00E94267841ED53E760E170E02E
:100EB00080EC90E00E94267841ED50E064E170E023
:100EC00087E69DE00F94D0A30E944A640F94A63C4D
:100ED0000F9440178EEC91EA0E94C47A89EE92E753
:100EE0000E94BD7C81E008950E94EE8664E070E07F
:100EF00084E190E00E94DA5591E08927089565E247
:100F000073E787E69DE00F9497A141ED50E064E11F
:100F100070E087E69DE00F94F4A38EEC91EA0E94C6
:100F2000C47A89ED92E70C94BD7CCF93DF93EC01FA
:100F30008991882319F00E94B179FACFDF91CF917E
:100F400008950E9495870C94BC7A2F923F924F92FD
:100F50005F926F927F928F929F92AF92BF92CF9249
:100F6000DF92EF92FF920F931F93CF93DF93CDB752
:100F7000DEB7A0970FB6F894DEBF0FBECDBF8FE5EA
:100F800090E00E946455882309F4A1C00E94FC549B
:100F90008F37910561F480914405909145059093B8
:100FA0004305809342058AEC92E70E94BD7C6E0166
:100FB0004FE1C40ED11C992493940E94FC5418163E
:100FC00019060CF078C080917312882329F00E94D2
:100FD0003566882309F46FC08091930381116BC03B
:100FE000209144053091450580914205909143053B
:100FF0008217930711F3F901EE53FB4F80812F5FA6
:101000003F4F2F77332730934505209344058F3F7B
:1010100009F079C080911903882309F471C0909276
:101020001803109219031F8E18A280901C038820A9
:1010300021F280911A038F8FF1E0F81518F4809156
:101040001B0388A310921C031601822D8C1988158E
:1010500008F0B3CFF10111911F018FE193E00F94DC
:101060004E0E17FDF2CF80914710909148101A3024
:1010700009F44BC11D3009F448C18F3591050CF0BE
:1010800049C11B3311F490921E0320911E032111BC
:10109000DCCF9C012F5F3F4F3093481020934710C7
:1010A0002091491030914A10255B3F4E820F931FCB
:1010B000FC011383CACF80914710909148101816F5
:1010C00019060CF451C28091D713811167C2A09602
:1010D0000FB6F894DEBF0FBECDBFDF91CF911F9149
:1010E0000F91FF90EF90DF90CF90BF90AF909F90C7
:1010F0008F907F906F905F904F903F902F900895CA
:101100009092190390CF90911803992309F458C035
:10111000893FE9F170F5863F09F44AC0873F09F439
:1011200043C085E992E70E94C47A80E992E70E9471
:10113000C47A109117038CE892E710FD02C087E88B
:1011400092E70E94C47A012F027082E892E711FDB3
:1011500002C08DE792E70E94C47A8CE792E70E9472
:10116000BD7C002349F185E480930B0210921803A3
:101170005ACF8A3F41F08B3FA1F6809117038160DF
:1011800080931703CECF809117038E7FF9CF1092F3
:101190001C0310921803109217031092160310925A
:1011A000190310921503BDCF809117038260E8CF19
:1011B000809117038D7FE4CF90E290930B02D6CFFE
:1011C0009091190330911703992331F1E0911C0399
:1011D00030FF49C020911503222309F440C091E05B
:1011E0009E0F90931C03AE2FB0E0A65EBC4FFFEFA6
:1011F000FC9340911603442351F0EE5FE0931C03EF
:10120000E92FF0E0E65EFC4F408310921603215078
:101210002093150310921903E0911C0330FF6CC05A
:1012200090911503992349F121E02E0F20931C037F
:10123000AE2FB0E0A65EBC4F8C938091160388233E
:1012400051F0EE5FE0931C03E22FF0E0E65EFC4F0E
:10125000808310921603915090931503E4CE42E0E0
:1012600040931503D7CF91E09E0F90931C03F0E0BD
:10127000E65EFC4F9FEF9083CDCFA82FAF7030E09C
:1012800021E0AF3029F0B0E0A050BE4F3C9120E00B
:10129000482F407F403F59F4226020FF13C09092B6
:1012A000150321FF0CC0E2E0E0931503BCCE82954C
:1012B0008F70A82FB0E0A050BE4F9C91EECF9093BE
:1012C0001603B1CE81E08E0F80931C03AE2FB0E0E9
:1012D000A65EBC4F3C933A3009F4A5CE21FF03C073
:1012E00090921503A0CEEE5FE0931C03E82FF0E090
:1012F000E65EFC4F908397CE91E09E0F90931C0387
:10130000F0E0E65EFC4F80838ECE009719F41092D9
:101310001E03DDCE0091491010914A10025B1F4E52
:10132000800F911FFC0110821A83098380911E0394
:101330008111FDC0F80180818E3409F084C04AE03B
:1013400050E0BE016F5F7F4FC80101960F946B9F05
:101350002B013C01E980FA80F7018081803231F471
:10136000FFEFEF1AFF0AFA82E982F4CF80913E1272
:1013700090913F12A0914012B09141120196A11D8F
:10138000B11D84159505A605B70549F044E050E068
:1013900065EC72E7C7010F94BFA1892BA1F46AE243
:1013A00070E0C7010F9437AA9093BC048093BB04EC
:1013B000009709F441C0F801F12C8E179F07F1F056
:1013C0002191F226FACF81EB91EA0E94C47A80E360
:1013D00093E60E94C47A60913E1270913F12809110
:1013E0004012909141120E942A7A0E94BC7A0E9477
:1013F000AC55109248101092471069CE0E941756B3
:10140000F816190639F081EB91EA0E94C47A81E15D
:1014100093E6DFCFE091BB04F091BC041082E98039
:10142000FA8060EC72E7C7010F948EA1892B39F521
:1014300087E795E60E94238381EB91EA0E94C47AB4
:1014400087EE92E6C6CF89819A81FC012081203205
:1014500021F401969A838983F6CF6AE270E00F94B3
:1014600037AA892B39F081EB91EA0E94C47A8DEB7F
:1014700092E6AFCF44244A94542C3201D0CF44E0BA
:1014800050E06BEB72E7C7010F94BFA15C01F7015D
:101490008081873481F48091610D853061F082E430
:1014A00092E10F944E0EF6E0F093610D60E085EA54
:1014B0009FE00F9404A4AB2821F080913B1281118E
:1014C00098CF26E077FC21E08091491090914A1056
:1014D000FC01E55BFF4E208349815A81F801DA0166
:1014E00040175107A1F501900020E9F79F01201B4B
:1014F000310B0396280F391F2D3EF1E03F0779F19C
:1015000030934A102093491080913C1290913D12E3
:10151000019690933D1280933C1277FC08C0409254
:101520003E1250923F1260924012709241121092FD
:101530004810109247100E94FC54892B09F4C7CD23
:101540008FE590E00E94645581117FCDC0CD6D91F3
:1015500061939D01241B350B6111F9CFCACF109205
:101560004A1010924910D0CF8091600D60E273E074
:10157000811102C060ED77E08FE193E00F941F0EC0
:10158000882309F4A0CD10921E03109248101092E7
:10159000471080EB92E70E94BD7C99CD80916A163E
:1015A000882309F494CD8091471090914810892B9D
:1015B00009F08DCD80913C1290913D12892B11F450
:1015C00010921D0312E001E04091EB165091EC16D1
:1015D0006091ED167091EE168091E4169091E516EB
:1015E000A091E616B091E716481759076A077B07DE
:1015F00008F0C1C080911D038111BDC00F94EF6C34
:1016000040916F165091701660917116709172161C
:101610004093EB165093EC166093ED167093EE1614
:1016200020914710309148108A3061F08D3051F090
:10163000833209F487C02F35310524F48F3F980792
:1016400009F087C02115310509F441CD80916A1652
:10165000811103C040E050E0BA018091491290919D
:101660004A12481B590BA0914910B0914A10FD0134
:10167000E55BFF4E1083418352831396255B3F4EFB
:10168000F901EA0FFB1F1082A55BBF4EFD0101901F
:101690000020E9F73197EA1BFB0BF89480913C128C
:1016A00090913D12019690933D1280933C12EC5F15
:1016B0008091491090914A10E80FF92FF11DF09395
:1016C0004A10E093491080916A16882309F43DC0BE
:1016D0008091EB169091EC16A091ED16B091EE165C
:1016E0008093491290934A12A0934B12B0934C12DC
:1016F000ED3EF14021F410924A1010924910789476
:1017000010921E0310924810109247104091EB1651
:101710005091EC166091ED167091EE168091E416E2
:101720009091E516A091E616B091E7164817590773
:101730006A077B0700F58FE590E00E9464558111F0
:1017400043CFC5CC00931D037DCF80E090E0DC014A
:10175000C7CFA9014F5F5F4F509348104093471088
:101760004091491050914A10455B5F4E240F351F40
:10177000F901838329CF4091EB165091EC166091CB
:10178000ED167091EE168091E4169091E516A091F9
:10179000E616B091E716481759076A077B0708F461
:1017A00096CC0E940379892B09F091CC0F94F965AE
:1017B0008AEA92E60E94BD7C0F946D176B017C0152
:1017C0000E94B0648CE3882E912CA12CB12CC7010F
:1017D000B601A50194010F9453A4CA01B901A50152
:1017E00094010F9453A47F936F93C701B60120E136
:1017F0003EE040E050E00F9453A43F932F938CE9D8
:1018000092E79F938F938E010F5F1F4F1F930F934C
:101810000F94F7A28EEC91EA0E94C47AC8010E944C
:10182000A187C8010E94E8DE0F942B731092560224
:101830000FB6F894DEBF0FBECDBF8091D8138823BA
:1018400059F00F9432688091600D882309F43FCCE1
:1018500086E00F9479323BCC81E00F946A738091DB
:10186000D8138111EECFEFCF0F931F93CF93DF9358
:10187000C82F8091F116813009F449C0823009F4F3
:101880005FC00E9491668111FFC080915D129091AE
:101890005E12009739F42091591230915A12232B7D
:1018A00009F4F2C040913302509134026091350244
:1018B00070913602411551056105710509F4E4C0C6
:1018C000892B31F48091591290915A12892B29F069
:1018D0008091AD05882309F43FC18091600D882374
:1018E00021F040EE52E369E270E08DEA95E00F945A
:1018F000880E882309F4CAC00F94051180E696E388
:101900000E943A750E9494EA0F94D507BFC00F94C5
:101910008A6E882309F4B5CF81E09091FE1691116B
:1019200001C080E08093F4168091380E9091390EBA
:10193000909301178093001782E08093F116A1CF56
:101940000F948A6E1092F5168091F116823009F08C
:1019500098CF8091F616811140C0D091FE1681E09B
:10196000D11101C080E09091F416891709F489CF54
:101970008093F41686EF96E10F944E0EDD23B1F1BD
:101980008091F216882311F18091940381111EC079
:10199000809101138130D1F080913E0D90913F0DE7
:1019A000891B8F7099F40E94406681110FC080914D
:1019B0005E0D843059F08FE59FE00F94E0A3811114
:1019C00005C061E080E398E30E94DD6281E08093DE
:1019D000F51681E08093590254CF64E670E086EFFB
:1019E00096E10F941F0E8111B8CF4BCF8091F31663
:1019F000882379F3809194038111EBCF80913E0D80
:101A000090913F0D891B8F7021F40E9440668823BE
:101A100001F3809173128111DCCF80910113813029
:101A2000C1F280915E0D8430A1F28FE59FE00F94AA
:101A3000E0A38111CECF88E794E69F938F938EE544
:101A400094E69F938F930F94A2A21092F316109294
:101A5000F21660E070E0CB010F94066660E070E083
:101A6000CB010E94B86685E69FE00E947C7881E009
:101A70009FE00E946F788EE59CE60F9478670F9048
:101A80000F900F900F90A5CF1092AD0580913C1252
:101A900090913D12039714F40E94A58790913E0DFA
:101AA00080913F0D981781F08091610D863061F42F
:101AB00068E873E182E492E10F941F0E882321F01D
:101AC00082E492E10F944E0E4091440350914503FD
:101AD00060914603709147034115510561057105F9
:101AE00009F03FC0409137025091380260913902AD
:101AF00070913A024115510561057105A9F088E41C
:101B000093E00F94880E882379F090913E0D809198
:101B10003F0D981309C0C11107C0179A10923906DA
:101B2000169A10923A06149AC091551290913F0D50
:101B300080913E0D981701F180913F0D9EE6899F9F
:101B4000F0011124EC55F94FC08190913E0D98178A
:101B500099F08F5F8F70F9CF8DEA95E00F94471061
:101B600095CF88E493E00F94880E882309F4BACFC8
:101B70008AEE97E70E942383CC2309F4BEC08091AC
:101B80003F0390914003A0914103B0914203892B00
:101B90008A2B8B2B81F40F94F00D605E7C4F8F4F5E
:101BA0009F4F60933F037093400380934103909352
:101BB0004203CFEF0FC00F94F00D00913F0310913F
:101BC000400320914103309142036017710782075F
:101BD000930778F38091B603882309F497C0C093E4
:101BE000650280915F04811107C081E080935F04EA
:101BF0000F94389710925F048091A6058823C9F14D
:101C00001092A6054FB7F8948091A405282F082EAE
:101C1000000C330B37FF03C0319521953109243077
:101C200031050CF476C0982F87FF02C093E0980F1F
:101C30009595959520911E0630911F06290F311D0F
:101C400097FD3A9530931F0620931E06837887FFF1
:101C500003C081508C6F8F5F8093A4054FBF86E0D7
:101C60000F94AD2580915902811103C081E08093CA
:101C700059028091A705882361F00E947073E0915A
:101C80000604F0910704309721F080915A028111E7
:101C900019952091CF1330E0A8EEB3E00F9480A403
:101CA000AB01BC0180ED93E10F94880E882399F07D
:101CB0008091CE1380FD0E94367C8091CE1382FDF0
:101CC0000E94BB7B8091CE1381FD0E94156580ED43
:101CD00093E10F9447108091600D811102C00E9422
:101CE000C17C40E355E760E070E08CE893E0DF9171
:101CF000CF911F910F910D94880E10923F03109277
:101D00004003109241031092420364CFC0931D061A
:101D100068CF1092A4054FBF80E0A2CFCF93DF938E
:101D2000EC010F941C3A81E00E94348C80E00E9408
:101D3000F96E209799F0C233D10540F062E370E06C
:101D400080E090E00F94BD0DE297EBCFBE0190E0F4
:101D500080E00F94BD0DD0E0C0E0E3CFDF91CF91E4
:101D60000895CF93DF93C82FDFEF0F941C3A81E0E3
:101D70000E94348C8091FF128F3FD9F4809194128D
:101D8000843021F4809197128111EFCF8091D2128B
:101D90009091D312019749F78091F9129091FA121C
:101DA0008932904811F360E089E290E80F949775CA
:101DB000DCCFD093FF12853039F4CF3FF9F261E0E8
:101DC0008C2F0F94CC9DD1CF8430C1F6DF91CF9171
:101DD0000895FF920F931F93CF93DF93EC01F62E9C
:101DE000662309F44BC00F949EA18C01C8010E9488
:101DF0006455882309F453C08091491090914A108A
:101E0000FC01E55BFF4E23E02083825B9F4EBE0119
:101E1000FF20E9F10F9497A18EEC91EA0E94C47A19
:101E20008FE992E60E94C47A8091491090914A10FD
:101E3000825B9F4E0E9495878AE792E70E94BD7C55
:101E40008091491090914A100496080F191F0D3E79
:101E500081E01807F9F010934A100093491080911F
:101E60003C1290913D12019690933D1280933C124A
:101E7000DF91CF911F910F91FF900895FC01019088
:101E80000020E9F731978F01081B190BAFCF0F9492
:101E90004BAAC2CF10924A1010924910E0CF81EBAA
:101EA00091EA0E94C47A8FE992E60E94C47ACE0138
:101EB000FF2059F00E94C47A8FE791EADF91CF9119
:101EC0001F910F91FF900C94BD7C0E949587F4CFD9
:101ED000CF93DF933091630420916204321320C0CA
:101EE000EB01BC0180915902882319F080E20E9425
:101EF000867280916104882399F020916304809117
:101F00001E0690911F062817190651F4209721F0FC
:101F100061E0CE010E94E98EDF91CF910C94736253
:101F2000809163048F5F80936304DF91CF91089564
:101F30000F931F93CF93DF93D62F8C01C0E0F8014E
:101F40008591949128E68C3C920721F4209101130D
:101F5000213019F461E00E94E98ECF5F0E5F1F4FC0
:101F6000DC13EDCFDF91CF911F910F910895CF93A7
:101F7000DF93CDB7DEB76E970FB6F894DEBF0FBE16
:101F8000CDBF9E012C5D3F4FF901419151919F01C1
:101F90006EE170E0CE0101960F9436A360E0CE01B1
:101FA00001960E94E98E6E960FB6F894DEBF0FBEC2
:101FB000CDBFDF91CF9108952F923F924F925F92C4
:101FC0006F927F928F929F92AF92BF92CF92DF9249
:101FD000EF92FF920F931F93CF93DF93CDB7DEB7AE
:101FE000C356D1090FB6F894DEBF0FBECDBF82E055
:101FF000809378020091381210913912025B1F4EC3
:1020000045E050E066E571E8C8010F94BFA1892B57
:1020100009F09BC18091600D882309F44DC085E6CD
:102020009EE70F94623C882379F08091BD041F9253
:102030008F9382E095E69F938F930F94A2A20F90C7
:102040000F900F900F9008C081E69EE70F94623CBE
:10205000882341F01092080481E0809378020E9466
:1020600022853AC28EE59EE70F94623C882321F1D7
:102070008091BB049091BC0461E003960F94F371CE
:102080000F94EF6C8C0180916F1690917016A09157
